:1000000000800020BD010000A19E0000599E00005C
:10001000599E0000599E0000599E0000599E000004
:10002000599E0000599E0000599E0000A19E0000AC
:10003000A19E0000599E0000B9BE0000BDBF000097
:10004000A19E0000A19E0000A19E0000A19E0000B4
:10005000A19E0000A19E0000A19E0000A19E0000A4
:10006000A19E0000A19E0000A19E0000A19E000094
:10007000A19E0000A19E0000A19E0000A19E000084
:10008000A19E0000A19E0000A19E0000A19E000074
:10009000A19E0000A19E0000A19E0000A19E000064
:1000A000957E0000A17E0000A19E0000A19E0000A0
:1000B000A19E0000A19E0000A19E0000A19E000044
:1000C000A19E0000A19E0000A19E0000A19E000034
:1000D000A19E0000A19E0000A19E0000A19E000024
:1000E000A19E0000A19E0000A19E0000A19E000014
:1000F000A19E0000F1C20000A19E00001DC40000EE
:10010000A19E00002DA80000A19E0000A19E00005D
:10011000A19E0000A19E0000A19E0000A19E0000E3
:10012000A19E0000A19E0000A19E0000A19E0000D3
:10013000A19E0000A19E0000A19E0000A19E0000C3
:10014000A19E0000A19E0000A19E0000A19E0000B3
:10015000A9C00000BDC00000D1C00000E5C0000083
:10016000A19E000049AB0000A19E0000A19E0000DE
:10017000A19E0000A19E0000A19E0000A19E000083
:10018000A19E0000A19E0000A19E0000A19E000073
:10019000A19E0000A19E0000A19E0000A19E000063
:1001A000A19E0000A19E0000A19E0000A19E000053
:1001B000A19E0000A19E0000A19E0000564B4CF2A3
:1001C000205210B51A804DF628121A8000BF00BFC9
:1001D00009F06AFE514B4FF010621A60504A9A6063
:1001E000504ADA60504A136813F4807304D14F49BF
:1001F0000B604FF4A85313604D4B1A78110703D5C9
:100200001A7842F008021A704A4B4B492A221A7097
:100210004A4A4B4B8B4204D252F8040F43F8040B6A
:10022000F8E7484B484900228B4202D243F8042B9E
:10023000FAE74649464A002352F8230041F82300D2
:1002400001336F2BF8D1434B434A802103F8011B44
:100250009342FBD1414B3D4A1A60414B8A221A70AE
:10026000A3F5805324225A70A0221A709A7992071B
:10027000FCD59A79D406FCD43A4A937903F00C035E
:10028000082B384BF9D103221A7140225A719A79FE
:100290009006FCD5334A9179324B4906FBD5324A58
:1002A000324911600221516020221A709A7902F0BD
:1002B0000C020C2AFAD12E4B2E4A1A602E4B2F4AD2
:1002C0001A6000225A60072243F8042C2C4AC3F813
:1002D0000C2D62B60AF072F9144B1B68DA0705D5CB
:1002E000284809F03FFF284B284A1A60284B1B7802
:1002F0005B0609D5244C254B22689A4204D121483B
:1003000009F030FF002323600DF046FB09F0D2FD19
:100310000BF060FFFEE700BF0E2005403080044078
:10032000823F04000100002B10D0034014D0034092
:1003300002D0074000E00740CC9AFF1FB40701003D
:100340004088FF1FCC9AFF1F90A2FF1F0082FF1F53
:100350000000000000E400E05FE400E008ED00E0E1
:100360000050064000400640448004400000030165
:1003700004800440C010050014E000E0FF76010096
:100380000000202089BBA65E1CE00340A5C3945A50
:1003900000F00740FFFFFFFFFFFFFFFFFFFFFFFF32
:1003A000FFFFFFFFFFFFFFFFFFFFFFFFFFFFFFFF5D
:1003B000FFFFFFFFFFFFFFFFFFFFFFFFFFFFFFFF4D
:1003C000FFFFFFFFFFFFFFFFFFFFFFFFFFFFFFFF3D
:1003D000FFFFFFFFFFFFFFFFFFFFFFFFFFFFFFFF2D
:1003E000FFFFFFFFFFFFFFFFFFFFFFFFFFFFFFFF1D
:1003F000FFFFFFFFFFFFFFFFFFFFFFFFFFFFFFFF0D
:10040000FFFFFFFFFFFFFFFFFFFFFFFFDEF9FFFF23
:1004100010B5054C237833B9044B13B10448AFF33E
:1004200000800123237010BDCC9AFF1F0000000044
:10043000B8070100084B10B51BB108490848AFF3D5
:1004400000800848036803B910BD074B002BFBD0A0
:10045000BDE81040184700BF00000000D09AFF1F01
:10046000B8070100CC9AFF1F0000000038B5044611
:10047000104621700A491D460DF070F801464FF0F4
:100480007E500DF01FF907490DF068F8E5606060D7
:10049000256165610AF022F8E061204638BD00BFA1
:1004A000DB0FC9400024744938B50446104621705A
:1004B00009491D460DF052F801464FF07E500DF0EF
:1004C00001F906490DF04AF8E56060602561656153
:1004D0000AF004F8E06138BDDB0FC940002474491C
:1004E00038B503780446032B20D8DFE803F01A1848
:1004F0001002C16840690CF027FF0D49054660688D
:100500000DF0E0F8014628460DF0DCF838BD08494A
:1005100040680DF0D7F8E1680DF020F838BDC068EC
:1005200038BDC16840690CF00FFF38BD002038BDF0
:100530000024744970B504460E4609F0CFFF054605
:10054000E069281A0CF0B6FFE3682361E561666193
:10055000A061014660680DF0B5F80146A060104842
:100560000DF0B0F80CF086FB0CF026F80CF098FEBD
:10057000054601464FF07E500CF0E6FE61690CF036
:10058000EDFF2169064628460CF0E8FF014630469B
:100590000CF0DCFEE0602046BDE87040FFF7A0BF35
:1005A000000080BF08B50E2009F030FB114B1B88FE
:1005B000012B19D0104B1B88984213DB40F6FF71BA
:1005C0008842D4BFC3EB0001C3EB0101C1EB013191
:1005D000C3F57F630F33282091FBF3F1BDE808409A
:1005E00009F0D2BD0021F3E70146BDE80840142020
:1005F00009F0CABDA29CFF1F329CFF1F10B5044624
:100600000BF030FD204610BD70B44C88A04220D9BC
:1006100001230133DBB21CB2660031F8144084427E
:100620001D46F6D3A04211D005F10045013D965B71
:1006300031F8151032F81530401AF21A00FB02F0AA
:10064000641A90FBF4F4E01870BC7047905B70BCC7
:10065000704702260125E5E700280CDA064A4342E6
:1006600082FB0320DA17C2EB600000EB4000A3EB33
:100670008000C0F10C007047ABAAAA2A2DE9F04710
:100680000C2009F08FFA0C2009F07CFE9C49142004
:1006900009F088FE9B499C4807F002F902210320DB
:1006A00009F016FF0221042009F012FF02210520A3
:1006B00009F00EFF0221062009F00AFF01210A209D
:1006C00009F006FF0121092009F002FF01210D2098
:1006D00009F0FEFE0121282009F0FAFE0121142074
:1006E00009F0F6FE02210B2009F0F2FE01210C2098
:1006F00009F0EEFE0C20002109F0D6FE042009F0DE
:10070000D9FE70B3052009F0D5FE044680B300245D
:1007100020467E4D287004F06FFC2B78EBB9204604
:1007200006F08AF87A4B7B491B887B4C09887B4A08
:100730002170A3F5AF7140F23A7303FB01F382FB22
:100740000312DB17764D7748A3EB621332335A213D
:100750002B6007F04FFC90B9FEE7BDE8F04706F0CC
:10076000B3BF062009F0A6FE0028CBD10124D0E7B4
:10077000032009F09FFEB0FA80F04009C9E76A4AF9
:100780006A481268DFF8F8A100230121FFF78CFE08
:100790000B2009F08FFE011E0CBF012300238AF8F5
:1007A000003002D1112009F093FEDFF89081604EF5
:1007B000604F614D0023C8F8003033603B604FF05C
:1007C000040914E009F022FA33681844306009F093
:1007D000010080F0010003F00BFB2B88002B14BFFD
:1007E0004B20FA2009F09CFEB9F1010919D00F2025
:1007F0000AF088F83B6803440E203B6009F006FAD3
:10080000D8F800309AF800200344C8F800301520CA
:10081000002AD7D111200AF075F8336818443060E7
:10082000D5E73B68D8F8002044493068DFF854E148
:100830002D88002BB8BF0333002AB8BF03329210B3
:100840000A603F493F4A0988128800284FEAA303FB
:10085000B8BF03303B6080103B4F30605E1A1944D4
:100860003E60CEF80010394F394E3A49C2EB000EC7
:100870000244C7F800E032600B605DB94FF4FA70D3
:1008800003F0C6FA03F0B0FA04F0B8FE4FF4AF601C
:1008900009F046FE304B012504201D6009F00AFED8
:1008A00010B92E4B20701D702D4B1B881C2B1CD09B
:1008B0002C4C04F1C805232009F0A8F944F8040FD2
:1008C000012009F02DFEA542F5D1274A274B1078CB
:1008D000187005F0BBFE03F083FA45F6BF522449B9
:1008E0002448BDE8F0470BF073BB234B1888002861
:1008F000DED0224BC0B2197805F0F0FDD8E700BF7A
:10090000001B3746801A0600D48FFF1FF69CFF1F7E
:10091000A49CFF1FEC9BFF1F159DFF1FB5814E1B65
:10092000B889FF1F789CFF1FC089FF1F389CFF1FDD
:10093000049CFF1FF49BFF1F469DFF1F9C9CFF1FF5
:10094000B489FF1FBC89FF1FB89CFF1F6C9CFF1F51
:10095000E09CFF1F849CFF1FDC9BFF1F5E9CFF1F12
:10096000349CFF1FE49AFF1F7E9CFF1FCC9CFF1F3F
:10097000A5050000709CFF1FE69BFF1F109CFF1F3A
:100980003C9DFF1F109DFF1FF0B40E8886420DD2C4
:1009900003F10043013B31F81350854202D9F0BC0A
:1009A000FFF732BE32F81300F0BC70471088F0BC7D
:1009B000704700BF094B1B880C2B09D8084A80B22E
:1009C00052F8232028B143F6FE73984203D9108CC5
:1009D0007047108870470349FFF716BEA69CFF1F9B
:1009E000C8EB000060EA0000374A38491088384AEE
:1009F000F8B5384B12881B68834248DB9342A8BF86
:100A0000134698420B60C8BF002342DD101AB0F5B0
:100A1000804FAABF9B03C3EB8333013093FBF0F0FD
:100A2000FFF7C8FF2C4B2D4F1C883B68C0F3C61541
:100A300005FB04F47F2CA8BF7F249D42064608D006
:100A4000274B1B88002B38D1264B1B88002B30D11D
:100A50003D60254D2B689E4205D0214B1B885A1FB7
:100A6000032A1DD92E60214D2B689C420ED0204BAD
:100A7000188848B11A4B1F4A1B88D35C834203D0A5
:100A8000C0B2E1B205F02AFD2C60F8BDF8BD034606
:100A900008609A42D4BFC0EB0203C0EB0303B5E782
:100AA000144AD05C2030C0B206F07F0105F016FD7C
:100AB000D8E7284605F086FDCAE70E4A2946D05CED
:100AC00005F00CFDC0E700BF329CFF1F289CFF1FF4
:100AD000549DFF1FCC9BFF1FD69BFF1FB89BFF1F82
:100AE000C89BFF1FBC9CFF1FD89CFF1FB09BFF1F14
:100AF000CA9CFF1F3C89FF1F2DE9F04F172089B0CA
:100B000009F000FFAF4B1860162009F0FBFEAE4B5A
:100B1000AE4A1B8810600C2B00F03B81AC4BAD4AF9
:100B200019880093AC4B52F8214000221A70AB4B4D
:100B3000AB4D1B88AB4A2E88013B32F91370002E57
:100B40005CD0A94BA94A1B88A9491278013B31F90D
:100B50001380002A40F0DF80112009F0D3FEA54B5E
:100B60000193D3F800A00646B24540F3DF80A24BC4
:100B7000DFF8A4921B88A14A012BD9F80030B2F803
:100B800000B09F4A02922046C8EB030800F09A8208
:100B90000CF090FC029A52F82B100CF0DFFC01468E
:100BA00000200CF0D1FB0CF09FFECAEB0802B04510
:100BB000B8BFB0469042CAEB080880F2968200FBAC
:100BC0000888013298FBF2F08E4BDFF850820293D6
:100BD000D8F80030034403EBD3735B10C8F800303F
:100BE0002B88012B12D1884BDFF834B20393874B4B
:100BF000DBF8005004934FF0000A47E07D4B01936F
:100C0000DFF814927F4BDFF8148202937E4B03933C
:100C10001D460F2009F076FE2B689842824641DA85
:100C2000754A1288012A00F01D82744A05931288C1
:100C3000734D049220460CF03DFC049ADFF8E0B1BD
:100C400055F82210DBF800500CF088FC014600201B
:100C50000CF07AFB0CF048FEEF1B059B5745A7EB09
:100C60000302B8BF5746FF1A9042BABF013200FBD9
:100C70000777474397FBF2F7D8F80020634B0493BC
:100C8000BB1803EBD3735B10C8F80030604B1B88B4
:100C9000013B032B00F2B082DFE813F06301A901EE
:100CA000C4008601594B04931B68984240F3C281EB
:100CB000514A1288012A00F0A682504A07931188EF
:100CC0004F4A0691204605920CF0F4FB059A0699CE
:100CD000DFF84CB152F82110DBF800500CF03EFC6C
:100CE0000CF002FE079B2F445745A7EB0302A8BF59
:100CF0005746FF1AD8F800309042BABF00FB07777A
:100D00000132474397FBF2F73B4403EBD3735B108D
:100D1000C8F80030BAE7152008F078FF354B01938A
:100D2000D3F800A00646B2453FF721AF354B0293FA
:100D3000D3F800A0B24580F289812F4BDFF8D8901C
:100D40001B882E4A012BD9F80030B2F800B02C4A8B
:100D500003922046984400F070820CF0ABFB039A9B
:100D600052F82B100CF0FAFB0CF0BEFDB045CAEBAC
:100D70000802A8BFB046CAEB08089042B6BF00FB05
:100D8000088800FB08F8013298FBF2F0DFF88C804D
:100D90001EE7204B1B78002B3FF4C0AE0C4B0D4AD6
:100DA000198800930C4B52F8210001221A700CF0A4
:100DB00081FB4FF07C510CF0D1FB0CF095FD04460B
:100DC000B5E600BFC09BFF1F349CFF1F889CFF1F20
:100DD000CE9CFF1F5089FF1FFE9BFF1F8C89FF1FAA
:100DE000C69BFF1FD4EC00008E89FF1F3C9DFF1F98
:100DF000ECEC00006C9CFF1F509DFF1F7A9CFF1FB6
:100E000020EC0000E09CFF1FB89CFF1F109DFF1FFF
:100E1000C489FF1F449DFF1F049CFF1FE09BFF1F11
:100E2000F49BFF1F28460CF045FBB2490CF096FBE3
:100E3000054650460CF03EFBAF490CF08FFB0146D7
:100E400028460CF083FA0CF04FFD0546CBF8005015
:100E5000D9F800000CF02EFBA6490CF07FFB0746EA
:100E600030460CF027FBA4490CF078FB01463846CD
:100E70000CF06CFA0CF038FDC9F800009F4AA04B4A
:100E8000168819889F4AA04B12681B889F4FC6EB93
:100E9000050E3544039EC6F800E0461A084404993E
:100EA0000D6001990E6002993E8808609A4280F2B6
:100EB00089810025C3EB060E954974450F6880F2C1
:100EC0007681611C9F4205FB01F50EF1010E95FB39
:100ED000FEF5C0F2BE81BE42A8BF3E46F61A01FB37
:100EE00006F494FBFEF49A4200F33681BB42C0F252
:100EF0003381884C20680CF0DDFA87490CF02EFB1A
:100F000086490CF023FA0CF0EFFCA0F5FF531C3BD4
:100F1000082B98BF4FF40050D8F800301844002830
:100F20002060C0F24281B0F5804F80F252817C4B4C
:100F30001B781BB1B0F5005F40F05381794D2B78E1
:100F4000002B40F05481784D20682B68714C9842FA
:100F500004D080B205F0A0FB23682B6009B0BDE887
:100F6000F08F28460CF0A6FA70490CF0F7FA054607
:100F700050460CF09FFA6E490CF0F0FA01462846F4
:100F80000CF0E4F90CF0B0FC0546CBF80050D9F8B1
:100F900000000CF08FFA65490CF0E0FA0746304685
:100FA0000CF088FA62495FE728460CF083FA5A4948
:100FB0000CF0D4FA054650460CF07CFA5D490CF072
:100FC000CDFA014628460CF0C1F90CF08DFC05461F
:100FD000CBF80050D9F800000CF06CFA4E490CF038
:100FE000BDFA074630460CF065FA52493CE7284600
:100FF0000CF060FA50490CF0B1FA054650460CF07E
:1010000059FA4E490CF0AAFA014628460CF09EF90E
:101010000CF06AFC0546CBF80050D9F800000CF043
:1010200049FA45490CF09AFA074630460CF042FA64
:10103000424919E7D8F80030DFF810B103EBD37359
:101040005B10DBF80050C8F800301FE6DFF80081C5
:10105000DFF80091D8F8003003EBD3735B10C8F8C9
:101060000030BDE5364A06931188364A0591204680
:101070000492DFF8D8B00CF01DFA049A0599DBF859
:10108000005052F821100CF069FA0CF02DFCEF1B07
:10109000069B5745A7EB0302B8BF5746FF1AD8F87F
:1010A00000309042BABF013200FB0777474397FBFD
:1010B000F2F73B4403EBD373234A04925B10C8F866
:1010C0000030E3E50CF0F6F9029A52F82B100CF020
:1010D00045FA0CF009FCCAEB0802B045B8BFB046AF
:1010E0008242CAEB08083FF76AAD00FB08F898FB9C
:1010F000F2F069E5CDCC4C3FCDCC4C3EB489FF1F1E
:10110000BC89FF1FC09BFF1F3A9DFF1FA09CFF1FB4
:10111000889CFF1F8889FF1F9A99193FCDCC4C45A9
:10112000FF9DFF1FE59BFF1F3889FF1F3333733F70
:10113000CDCC4C3DCDCCCC3E6666663FCDCCCC3DD7
:101140007A9CFF1F20EC0000109DFF1FF49BFF1FE7
:10115000E09BFF1F049CFF1F009B1B88002B3FF49C
:10116000C8AE2B1B002BB8BF5B42092B47DD05F532
:1011700000500130001B0CF09DF93B493B4C0CF03A
:10118000EDF9054620680CF095F939490CF0E6F9BF
:10119000014628460CF0DAF80CF0A6FBD8F800302F
:1011A000184400282060BFF6BEAE002213E09F4224
:1011B00005FB04F5B8BF002195FBFEF54BDA91FB6A
:1011C000FEF490E6B242D4BFC3EB0205C3EB0605C2
:1011D00070E643F6FF72274B22601B78002B3FF42A
:1011E000ADAE02F001FE244B01221A70ABE602F014
:1011F000F7FD00232B70A6E6D9F800003EE64FF479
:1012000000501A4C88E61D491D4A069320460D8859
:1012100005920CF04FF9059ADFF868B052F82510E6
:10122000DBF800500CF09AF9014600200CF08CF825
:101230000CF05AFB2F44069B56E50CF03BF9039A41
:1012400052F82B100CF08AF9014600200CF07CF8C3
:101250008AE51E4642E6B742D4BFC3EB0701C3EBA3
:10126000060104FB01F1AAE7CDCCCC3E8889FF1F23
:101270009A99193FFF9DFF1FE59BFF1F7A9CFF1F57
:1012800020EC0000F49BFF1F08B5244B1B88FBB12A
:10129000234B1B78FBB1234B1B78E3B1224B1B780C
:1012A000CBB1224B1B78B3B1214B22481A78C2B97B
:1012B000214A22490088128809680244B1EB620F72
:1012C00009DD01221A706420BDE8084002F0A0BDCB
:1012D000174A117801B908BD1370BDE8084005F040
:1012E000A5B9154A16490088128809680244B1EB6D
:1012F000620FF0DD00221A7005F098F9642002F008
:1013000087FD642002F084FD642002F081FD4FF42B
:101310001670BDE8084009F003B900BF8C9CFF1FA0
:101320002C9CFF1FEF9BFF1FF09BFF1FF19BFF1FDC
:10133000D59BFF1FA09CFF1F3A9DFF1FC09BFF1F57
:10134000889CFF1F38B5114C2320257808F05EFCDF
:101350000F4A42F82500131F02F1C400002253F87F
:10136000041F83420A44FAD123780A4907480A4CE9
:101370000133DBB2322B81FB025108BF0023D217AD
:10138000C2EB21120370226038BD00BFC89CFF1F52
:10139000E89AFF1F1F85EB51D09CFF1F2DE9F047F6
:1013A0009F4CA04D206882B00CF084F89E490CF050
:1013B000D5F80646102009F0A5FA0CF07BF89B49F9
:1013C0000CF0CCF831460BF0C1FF0CF08DFA2B88F5
:1013D0002060192B00F0CA801A2B00F0F5801E2B1C
:1013E00000F0FB8001252E46914A1188002900F06B
:1013F0009180904B904A1B881288834240F3DD8095
:101400000020D31A8B42C6BF01FB000001334843C2
:1014100090FBF3F3894A1360894F388848B9894BA8
:101420001B8833B9884A117801B1137002B0BDE846
:10143000F087DFF800822168B8F80030784A8B42E4
:101440006EDCDFF804E29EF80090B9F1000F2FD1B6
:101450004FF0010C04288EF800C029D1002D40F077
:101460007181784B18880028E0D0002EDED02368E8
:10147000B8F80040704AA342128880F23E810023EF
:10148000141B7E2C714DD5BFC3EB8313C3EBC31369
:101490005B00013493FBF4F42B680134A34203D0C6
:1014A000C0B2E1B205F01AF82C6002B0BDE8F087D6
:1014B000012800F0D580022800F0A9800328D0D1AF
:1014C000634B1B88092BCCD0002DCAD02368B8F8F9
:1014D0000050594AAB42128880F25C810023551BB0
:1014E0007E2DDFF874A1D5BFC3EB8313C3EBC31309
:1014F0005B00013593FBF5F5DAF800300135AB42BE
:1015000003D0E9B24A2004F0E9FFCAF80050A8E786
:101510000D460E461E2B7FF47FAF00214D4F64E039
:10152000494B1A78002A81D0002401281C7062D00F
:10153000022840F0E980002D63D0474D2B68002B36
:101540005FD00420214604F0C9FF3E4B2C60188870
:1015500000283FF46BAF002E3FF468AFC0B200210B
:1015600004F0BCFF394B00221A605FE7394F3B4E55
:101570003A7872B13349098859B196F800E0964536
:1015800042D0C8B27F2104F0A9FF3A782B8832708C
:101590000AE03178914237D02A4B0021187804F0C4
:1015A0009DFF3A782B883270214A11880029AFD0EC
:1015B00000251E2B2E4618D01BE08242D4BFC3EB61
:1015C0000200C3EB00001CE7224F3A78002A0BBF51
:1015D000012500250026012606E71E4F144B3D7805
:1015E0001988B5FA85F56D0900263B78002B3FF484
:1015F00011AF2068FDE625B1174D2B68002B40F098
:101600009A80104B1888A3E700252E46ECE6002DA3
:101610003FF427AFDFF840A0074ADAF800304AE08D
:10162000189DFF1F349CFF1F9A99193FCDCCCC3ECB
:101630003E9DFF1FFE9CFF1F6A9CFF1FE89BFF1F34
:10164000F89CFF1FB49BFF1FEE9BFF1F249CFF1FF6
:10165000C89BFF1F449DFF1F009CFF1F5A9CFF1F3C
:10166000002D3FF4FEAE534A10888842D4BFC3EB2E
:101670000009C3EB0109C31A7E2B40F38280C9EB3A
:10168000C91103F1010991FBF9F909F10109DFF829
:101690002CA1DAF800304B4506D05FFA89F1012021
:1016A000019204F01BFF019A3888CAF800900228C2
:1016B0007FF404AF4B462168B8F800901088494584
:1016C00058DA0022C9EB0009B9F17E0FD3BFC2EB93
:1016D0008212C2EBC21209F10109520092FBF9F920
:1016E00009F10109994504D05FFA89F1042004F059
:1016F000F5FE3888CAF80090E0E69342D4BFC4EB08
:101700000303C4EB0203BBE6032828D12A4B1B8842
:10171000092B3FF476AF002D3FF473AF274D2B68B4
:10172000002B3FF46EAF4A20214604F0D7FE244B35
:101730002C6018880CE7214604F0D0FE204B2C606A
:10174000188805E740207F21019204F0C7FE388801
:10175000019A012825D002287FF4B0AE5AE7042868
:101760007FF44FAF002D3FF44CAF2146402004F0F2
:10177000B5FE46E78142D4BFC9EB0102C9EB0002C6
:10178000A0E7C9EB89194FEA490999FBF3F909F177
:1017900001097CE79342D4BFC5EB0303C5EB020309
:1017A0009DE61168B8F80030024A99421088FFF6A9
:1017B00062AF5AE76A9CFF1FC89BFF1F009CFF1F78
:1017C000B49BFF1F08B50F4B1B88022B0FD0032BB8
:1017D00012D0042B03D00C4B01221A7008BD7F21BC
:1017E000092004F07BFE084B01221A7008BD7F21FE
:1017F000412004F073FEEEE74021092004F06EFE64
:10180000E9E700BF689CFF1F029DFF1F38B51C4B16
:101810001B881D2B26D01B4B1B88012B25D01A4A59
:101820001A4B14881B681A4AA342128818DB934289
:10183000D4BFC4EB0303C4EB0203141B7F2CC6BF4D
:10184000DB010134C3EBC31393FBF4F4114D2B689C
:101850009C4203D0E1B2052004F040FE2C6038BD6C
:101860000023EAE70C4B1C88F0E70C4B0C4A0D49AF
:101870001B6812680C689B1A1C1B84F30704E5E7BD
:10188000349CFF1FC69BFF1FE49CFF1F0C9DFF1F86
:101890002E9CFF1FD49CFF1F109CFF1F849CFF1FCA
:1018A0004889FF1F049DFF1F10B50F4C23685BB9CB
:1018B0000E4B1B88022B11D0033B012B09D90C4A7C
:1018C00000231370236010BD0021052004F006FEE4
:1018D000EEE70021092004F001FEF0E7002141209D
:1018E00004F0FCFDEBE700BFD49CFF1F689CFF1FCA
:1018F000029DFF1F08B5274B1B78ABB1152008F0E0
:1019000085F9254A254B128818601D2A15D0244ACE
:101910001288EAB1012A25D0224B1B78002B34D043
:10192000BDE80840FFF7C0BF112008F0EBFF1A4ADE
:101930001A4B128818601D2AE9D11B4B1B78002B0B
:10194000EAD0184B1B780BB3BDE80840FFF75EBF29
:10195000164A1288002ADFD0154A1B6812889A425C
:10196000DADCEEE70F2008F0CDFF104B114A1B88A0
:10197000106033B1104B114A1B6812689B1A9842D1
:10198000DFDD084B1B78002BCAD108BDFFF71AFF1B
:10199000DAE700BF3C9DFF1F349CFF1F0C9DFF1F1B
:1019A000C69BFF1F029DFF1F449DFF1F689CFF1FDA
:1019B000E49CFF1F049DFF1F849CFF1F4889FF1F9D
:1019C0002DE9F04F87B003AD944F2C4606AE611B56
:1019D000C9B2934806F0D2FA3B88834294BF0020F4
:1019E000012004F8010BA642F1D18E488E4A9DF8E1
:1019F0000C508E4905709DF80E008D4E10709DF8AC
:101A000010209DF814308B4F8B4C0A709DF81210EB
:101A1000317000263B70267063B9002940F0DF80EA
:101A2000002A40F0E480854A002800F0E880022384
:101A3000237005E0002A40F0988005237F4A237038
:101A40007F4DDFF84CB29DF80DE09DF80F00DFF8F8
:101A500044A2DFF84492DFF844827A4F7A4E137042
:101A60009DF811109DF816209DF8133085F800E0C0
:101A70008BF800009DF815E09DF817C089F800204C
:101A8000012088F8003087F800E08AF8001086F816
:101A900000C008F037FF6D4A6D4BD2F800E070458A
:101AA000CCBF012200221A7063DD6A4B1988182905
:101AB0005FD80C39684B2D781A789BF800C09AF8DB
:101AC00000A099F8003098F80080DFF8D4913F78B2
:101AD00036782478A2EB4502AAEB8A0BCCEB020203
:101AE0005A44C3EB837BC3EB8B03134403EB4803E0
:101AF000B9F80020DFF8AC913B4406FB02334FF00D
:101B00000C0B1BFB0433C9F80030BAF1000F06D0F0
:101B10002EB1042A0CBF02330433C9F800304F4AF7
:101B20004F4E1288B6F800904E4C4F4E24883668BF
:101B3000033A02EB4202C9EBC90903EB82022244D9
:101B40004E444A4C0C3A54F826400A44224495B17B
:101B5000B8F1000F0FD0BCF1000F44D1BAF1000F63
:101B600051D1434901240C700EE006232370334AFF
:101B700066E700219EE73E4900240C70BCF1000F8F
:101B800000D027BB4FF0000C3A49704581F800C0E7
:101B9000C4BF39490B6039490B689A4213D0384B9E
:101BA000384C18680190019820601B680293364CED
:101BB000029B24880A601B1AA34284BF334B1A601D
:101BC00007B0BDE8F08F2F482D4B0068EDE7002DE2
:101BD000D8D1BAF1000FD5D14FF0010CD4E70423CE
:101BE0002370164A2CE7224900240C70CAE7134AD6
:101BF0001378002B3FF418AF0323237020E735B18F
:101C0000012323701CE71A4981F800C0BCE7137850
:101C1000012B8CBF23702B4612E700BFA49CFF1F33
:101C2000789CFF1FEF9BFF1FF09BFF1FF19BFF1F87
:101C3000F29BFF1FF39BFF1FBC9BFF1F969CFF1F88
:101C4000409DFF1F309CFF1F4C9DFF1FB889FF1F49
:101C5000449DFF1F349CFF1F8489FF1F5C9CFF1F56
:101C6000949CFF1F0A9DFF1FE89BFF1F48EC00008C
:101C70007C9CFF1F7D9CFF1F489DFF1FD09BFF1F6B
:101C80001C9EFF1FF89BFF1F529DFF1F089CFF1FFC
:101C9000419DFF1F439DFF1F2C9CFF1FD49BFF1FD7
:101CA0009A9CFF1F349DFF1F2DE9F04F3B4B1B7883
:101CB0008BB0002B6DD10E2007F0A8FF0BF0FAFBC4
:101CC00001463748374C384DFEF734FC3448FEF7B0
:101CD00007FC0BF009FE80F30C002060FFF770FE9C
:101CE0002E68012E7CD0022E00F0AA82032E00F076
:101CF000B9832E4C23682E4A2E4E0993099B1778E0
:101D000030682D4C07210122181A11FB072290423E
:101D1000236000F29082294E32689A1A0D2A00F24E
:101D20008382274E32689A1A132A00F27882254E4F
:101D300032689A1A252A1AD9234B1B88002B40F0A7
:101D40006781224B1B78002B40F06281FFF7FAFA83
:101D50001F4B1B881B3B9BB2022B04D81D4B1B78CF
:101D6000002B40F0588102F065F8236833601A4D6B
:101D70002A689B1A502B00F21182184B1B88012BEA
:101D800000F0298204F03EFC04F06CFA0BB0BDE8D0
:101D9000F08F05F025FB0BB0BDE8F08FF69CFF1F20
:101DA000389CFF1FCC9BFF1FDC9BFF1F1C9EFF1F4F
:101DB000149DFF1FEC9CFF1F149CFF1FC49CFF1F62
:101DC000909CFF1F2C9DFF1F8C9CFF1FD59BFF1F0E
:101DD000349CFF1F449DFF1F649CFF1FA29CFF1F9C
:101DE000DFF82883A34AB8F800001378834204D0B0
:101DF000C3B21846137004F041FBDFF80C939E4AFF
:101E0000B9F800301178994204D09C4F39780029F4
:101E100040F07E879A4A236812889A4C9A42C0F210
:101E2000FF80994A1278002A40F0FA80DFF8E0A299
:101E3000BAF8003023B9954B1B88002B00F01F85A2
:101E4000934A944B11881B88934A0B4412685B1089
:101E50009342924A126880F2C28400219342B4BF36
:101E600001230B4604910093ACBF4FF0010B8B464E
:101E700005910E2007F0CAFE894B8A4A1B68176835
:101E800003930133A7F25232002B8446029240F3AF
:101E90005087802BA8BF8023834A84491278019100
:101EA000002A00F0C7800978914200F0C380B9F899
:101EB0000010DFF854E2994201F047816F49AEF813
:101EC00000307B4B4FF0010E81F800E01978DFF80D
:101ED00044E2019B8EF800101A70009B002B00F06A
:101EE0001B81BAF80030002B00F01681714B1B6883
:101EF0005A1C002A40F32187802A00F31D876E4E6A
:101F00006E496F483688098800683144B0EB610F2C
:101F1000C1F2EF81A3F148020F2A02D8473BA8F88B
:101F200000300E2007F072FE6FF454731F44874296
:101F300002DC644B00221A70002008F0E3FC624AC5
:101F4000624B1168624E1B888842D4BF0022012276
:101F50003270002B00F03A845E4B1E78964240D0DF
:101F600088423EDD5C490E78002E00F0CB875B494D
:101F700091F800C0BCF1000F40F0C287584F0097A5
:101F8000584F59480297564F007887F800C0554F70
:101F90004FF0010E87F800C081F800E0002841F002
:101FA000668152490978002901F027805049039140
:101FB0000E460978002941F01D804E48494F0078AF
:101FC000397001210297317058B14548434900905A
:101FD000002008700099029F0870039901263E7046
:101FE00008701A70444B1B88A3F11B02012A40F2AF
:101FF0006A861D2B7FF47EAE3E4F3B78002B41F06E
:10200000E9803E4E3378002B40F06984337071E6EE
:10201000FFF73AF99AE62B68012B7FF4A4AEA4E609
:102020002168374A069106983649106002220B60F3
:102030002A60FBE61E49DFF8DCE0097800293FF45E
:1020400048AF9EF8000081423FF443AF03984B280D
:1020500041F327801833802BB9F80000A8BF8023F4
:1020600098423FF436AF28480380044801230370A8
:102070002FE700BFCC9CFF1F159DFF1F5E9CFF1F1D
:10208000329CFF1F1C9EFF1FD59BFF1F589CFF1FEC
:10209000A09CFF1F3A9DFF1FC09BFF1F889CFF1F36
:1020A000489DFF1F9C9CFF1F7C9CFF1F429DFF1FA4
:1020B0007D9CFF1F349DFF1FFE9CFF1F6A9CFF1F1E
:1020C000189DFF1F309DFF1FB889FF1FF49CFF1F45
:1020D0000D9CFF1F209CFF1F2C9CFF1F0C9CFF1FB3
:1020E000809CFF1FE49BFF1FD49BFF1F409DFF1F91
:1020F0000E9CFF1F449DFF1F349CFF1F5A9CFF1F17
:10210000D89BFF1F209DFF1FEC9BFF1F7E9CFF1F86
:10211000FA9CFF1F1C9DFF1F029B9C45BFF601AF51
:10212000AC4B1B88002B3FF4FCAEBBF1000F7FF4DF
:10213000DDAEA94B1B881BB1059B002B7FF4D6AEEF
:10214000049B002B3FF4EDAEA44B1A78002A7FF4D9
:10215000E8AEDFF8048398F8006001221A70002EC0
:1021600040F05A839E4B1B78002B01F004819D4B5D
:102170001B78002B01F015819B4B1B78002B7FF403
:10218000D0AE9A4B1B78002B3FF4CBAEB9F80030A1
:1021900097490A3BA9F800300A70C2E602F074FFC2
:1021A000944B1B7873B9944B1B785BB9934B1B789A
:1021B00043B9934B1B782BB9924B1B7813B901F0A1
:1021C0000FFE01E001F018FE23682B608E4B1B8888
:1021D000012B7FF4D7AD8D4A8D4B11688D481A784D
:1021E000A1F118032A2101FB03F10160002A00F08C
:1021F000D782894A1368994200F3458380F24F835E
:1022000086480068D0F17F0048BF0330801001305D
:102210001B1A994200F3438313601946C2E2FFF789
:1022200069FB2368336082E5FEF766FCFFF7B6F8CA
:102230002368336075E5FEF7D7FB236833606AE5F2
:10224000774A26681288B24204DB6E4B1B78002B5B
:1022500000F04083734C744823680793734B0799CD
:1022600000681B88091A994263D8002B61D0704B13
:10227000198800293FF43EAD6E4B6F481B680088FB
:10228000B342B8BF33469A4241F32C806B4B1A607D
:10229000DFF8C88188F800105C4FFEF7A5FB3868AE
:1022A0007F2840F32986664B7F3883FB0032C317B3
:1022B000C3EB620303EB4303A0EB83007330614B7A
:1022C00001931B883860002B40F031874B4B009303
:1022D0001B78002B00F05A845B4E3378002B00F003
:1022E0005584DFF87C91DFF858A14FF0000B0CE02B
:1022F00003F17300C0B298F8001004F017F93378B6
:102300000BF1010B5B4540F341843B6859F8040F26
:102310001844A0F17F038AFB0321DA17C2EB6102A4
:1023200002EB42027F28A3EB8203E1DCFEF794F983
:10233000E0E7404B40491B6808883D49B342B8BFBD
:1023400033469A4200F3AD823C4E09888342A8BFCF
:102350000346336000299BD19A42C8BF0B4640F325
:10236000A782801AB0F5804FAABF9B03C3EB8333CB
:10237000013093FBF0F0FEF71DFBC0F3C6100BF02D
:1023800099F8324B064618880BF094F83049074606
:1023900030460BF0E3F8014638460BF0DFF83146E3
:1023A0000AF0D4FF4FF07E5106460BF075FA002874
:1023B00040F08D87274930460BF08CFA002840F01A
:1023C0004A8730460BF0B6FAC0B2DFF8908088F842
:1023D000000061E7589CFF1FFC9CFF1F309DFF1F02
:1023E000409DFF1F419DFF1F439DFF1F2C9CFF1F12
:1023F0005E9CFF1FE49BFF1F0C9CFF1F809CFF1F28
:102400000E9CFF1FD59BFF1FA29CFF1F089CFF1F58
:10241000029DFF1FE89CFF1F1C9CFF1FD49CFF1FF9
:10242000329CFF1F1C9EFF1FD89BFF1FC09CFF1FDD
:102430004E9DFF1F209DFF1F549DFF1F289CFF1FC7
:10244000ABAAAA2A609CFF1F4C89FF1FC49BFF1FD9
:10245000CDCCCC3D0000FE42BC9BFF1F189CFF1F53
:102460008C89FF1FB94B26681988B14253DDB84BE0
:102470001B78002B4FD1DFF8209399F800007F28BC
:1024800040F3A486A3F155337F3803F1004383FB67
:102490000032C317C3EB620303EB4303A0EB8300DB
:1024A0007330AC4B01931B88C0B289F80000002B3D
:1024B00040F0ED86A84B00931B78002B00F04D8573
:1024C000A64E3378002B00F04885A54FDFF89882A0
:1024D0004FF0000A0AE003F17300C0B204F04EF8B6
:1024E00033780AF1010A534540F3378557F8043F22
:1024F00099F800001844A0F17F0388FB0321DA1744
:10250000C2EB610202EB42027F28A3EB8203E2DC12
:10251000FEF7A2F8E1E7934F38687F2840F3CF81B8
:10252000914B7F3883FB0032C317C3EB620303EB8D
:102530004303A0EB83007330DFF85C9299F800A0AE
:10254000824500F02682894B1B88002B43D1884AA4
:10255000884812680088914205DC8242D4BFC1EBF2
:102560000203C1EB0003411AB1F5804FA6BF9B03E4
:102570000131C3EB833393FBF1F0FEF71BFAC0F399
:10258000C6100AF097FF7C4B064618880AF092FFA7
:102590007A49804630460AF0E1FF014640460AF09B
:1025A000DDFF31460AF0D2FE4FF07E5106460BF0B9
:1025B00073F9002840F06886714930460BF08AF9BB
:1025C000002840F0378630460BF0B4F9C0B2DFF88F
:1025D000CC8188F80000BAF17F0F40F3888462480C
:1025E000AAF17F0A80FB0A304FEAEA73C3EB60006E
:1025F00000EB4000AAEB80007330574B00931B7830
:10260000C0B289F80000002B40F0E8835D4B0393D3
:102610001B78002B40F0B5855B4B02931B78002B99
:1026200040F058864B4B0193029B1B78002B3AD00D
:10263000564B1B88182B17D099F800201344A3F190
:1026400018007F2840F3F985474A973B82FB032116
:10265000DA17C2EB610202EB4202A3EB820303F141
:102660007300C0B203F08AFF494A4A4B127833F82C
:102670001230182B17D099F800201344A3F118003A
:102680007F2840F3E485384A973B82FB0321DA1721
:10269000C2EB610202EB4202A3EB820303F173007F
:1026A000C0B203F06BFF009B1B78002B00F0B584D9
:1026B000019B284E1988002900F05C8538687F2826
:1026C00040F35783284B7F3883FB0032C317C3EB9B
:1026D000620303EB4303A0EB8300733038600029EF
:1026E00040F0F084009B1B78002B00F05D811B4EB6
:1026F0003378002B00F05881DFF864A0DFF89C806D
:102700004FF0000B0CE003F17300C0B298F800101A
:1027100003F00CFF33780BF1010B5B4540F3448170
:102720003B685AF8040F104A1844A0F17F0382FB5B
:102730000321DA17C2EB610202EB42027F28A3EB0E
:102740008203E0DCFDF788FFDFE700BF329CFF1F5C
:10275000D59BFF1F609CFF1F809CFF1F4C89FF1FA4
:102760008C89FF1F089CFF1FABAAAA2A4E9DFF1F42
:10277000289CFF1F549DFF1FC49BFF1FCDCCCC3D49
:102780000000FE420E9CFF1FE49BFF1F009DFF1FE9
:10279000089DFF1F249DFF1FBE9CFF1F189CFF1F4D
:1027A000A84B1960A84B1B68A92202FB03F3002B5E
:1027B000BCBF03F57F533F339B13543B194481F354
:1027C0000C01282007F0E0FCFFF7DCBA9F4EA04880
:1027D000A049A14A337003700B70137002E4934256
:1027E0004FF0000B6EDA0123CDF800B0CDF814B035
:1027F0000493FFF73EBB994B1B78002B7FF491AB02
:10280000039B974A243B83F34703D9B25B201360B1
:1028100003F064FE98F80060032E30D1DFF8908258
:1028200098F80030002B40F03F868E4F3B78002B0D
:1028300040F02D86894E3378002B40F01B868A4B62
:102840001B78002B40F00986884A1380884B1B7840
:10285000002B40F0F585874B7F221A8098F80030D6
:102860006BB93B785BB933784BB9834A7F2107203A
:10287000138003F033FE7F210B2003F02FFE7F4BEC
:102880001F68FFF74EBB7E480068D0F17F0048BF4D
:10289000033003EBA00301339942BFF6BDAC1160D6
:1028A00080E7784B09881A6000297FF4F1AC134661
:1028B0009842D4BFC2EB0003C2EB030351E5FDF71E
:1028C000CBFE39E60123CDF810B0CDF800B005936A
:1028D000FFF7CFBA01232B606B4CFFF70BBA6B4BA2
:1028E0006A20198803F07EFF3B783370FFF702BA45
:1028F000564B1B78002B3AD0654B1B88182B17D0F2
:1029000099F800201344A3F118007F2840F3F684BF
:10291000604A973B82FB0321DA17C2EB610202EBAC
:102920004202A3EB820303F17300C0B203F026FE60
:10293000594A5A4B127833F81230182B17D099F89D
:1029400000201344A3F118007F2840F3DB84514A90
:10295000973B82FB0321DA17C2EB610202EB4202D2
:10296000A3EB820303F17300C0B203F007FE019BE7
:102970001B88002B00F09584354B1B78002B40F012
:102980008A84474B3F4A198826680020012310603B
:102990002B60B1423C4CBFF6ADA92268414B089276
:1029A000089A1A60FFF7A6B9039B1B78002B00F06A
:1029B00083803B68A3F10C007F2840F3FA833548FD
:1029C0008B3B80FB0320DA17C2EB600000EB40007A
:1029D000A3EB800303F17300DFF8D080C0B298F856
:1029E000001003F0A3FD009B1B78002B64D02E4E3B
:1029F0003378002B60D0DFF8BCA04FF0000B0BE069
:102A000003F17300C0B298F8001003F08FFD337823
:102A10000BF1010B5B454FDD3B685AF8040F1D4A73
:102A20001844A0F18B0382FB0321DA17C2EB610289
:102A30000C3802EB42027F28A3EB8203E0DCFDF7B7
:102A40000BFEDFE71C9CFF1F8889FF1FE49BFF1F15
:102A50000C9CFF1F809CFF1F0E9CFF1F2C9CFF1FC8
:102A6000DC9CFF1F439DFF1F419DFF1FBC9CFF1F60
:102A7000D49BFF1F4E9DFF1FC89BFF1F9C9CFF1FE9
:102A8000D49CFF1F289CFF1F1C9EFF1F109CFF1F34
:102A9000009DFF1FABAAAA2A089DFF1F249DFF1FB0
:102AA000329CFF1FE09DFF1F4C89FF1F189CFF1FDA
:102AB000409DFF1F8C89FF1F029B1B78002B3AD083
:102AC000AD4B1A88182A18D03B681344A3F118009C
:102AD0007F2840F3B683A94A973B82FB0321DA178C
:102AE000C2EB610202EB4202A3EB820303F173002B
:102AF000A34BC0B2197803F019FDA2490B78022B41
:102B000000F253830133DBB20B701A469E4830F853
:102B10001260182E40F090820422032B03F101066C
:102B2000F3B208BF002330F81360182E40F0838200
:102B3000013AF2D10B70019B1B88002B00F0CB8275
:102B4000009B1B783BB9039B1B7823B9029B1B7826
:102B5000002B00F0E0838D4B1B78002B00F0D6801B
:102B60008B490B78082B00F2D1808A483A680068BC
:102B7000894E0133DBB25F1E101A46F827000B7036
:102B8000864B2668198889F8002002E77F4B1B785E
:102B9000002B40F0C1823B68814A1278002A45D060
:102BA000A3F10C007F2840F30A83744A8B3B82FB1D
:102BB0000321DA17C2EB610202EB4202A3EB8203AC
:102BC00003F17300C0B298F8001003F0AFFC009B53
:102BD0001B7853B36E4E33783BB3DFF8FC91DFF8CC
:102BE0009CA14FF0000B0BE003F17300C0B298F80A
:102BF000001003F09BFC33780BF1010B5B4514DDF7
:102C00003B6859F8040F1844A0F18B038AFB032199
:102C1000DA17C2EB61020C3802EB42027F28A3EB09
:102C20008203E1DCFDF718FDE0E73B685D4A1278BE
:102C3000002A3DD0504A1288182A18D01344A3F114
:102C400018007F2840F30D834C4A973B82FB0321F9
:102C5000DA17C2EB610202EB4202A3EB820303F13B
:102C60007300C0B298F8001003F060FC3B6845495F
:102C70000A78022A00F2A6820132D2B20A701646FF
:102C8000414830F816E0BEF1180F40F0F0810426FC
:102C9000032A02F1010E5FFA8EF208BF002230F81B
:102CA00012E0BEF1180F40F0E181013EF0D10A7050
:102CB000019A1288002A00F041823B4903220B70DE
:102CC0002A60FFF717B8394F3B78002B3FF499A9DA
:102CD000374E307801F0FEF8364B1B78002B00F0B1
:102CE000918233887E2B00F28D82334A0133108823
:102CF00099B23180002800F09582C9B2C0B22F4E3F
:102D000003F0ECFB3B783370FEF7F4BF3A6837E72B
:102D1000DBB21846137003F0BFFB294B1B491A4660
:102D20001F4B184600230B703B7013700370FFF7A6
:102D300071B80123FFF7B0B880262249224B234AFD
:102D400009881B8812680B44B2EB630FBFF6E9A831
:102D5000164B1B78002B40F0FE81B9F800301C4A5E
:102D6000B3423FF4DEA81B4B168001221A70FFF716
:102D7000D8B8FDF771FCB1E4009DFF1FABAAAA2AE9
:102D8000189CFF1F089DFF1F249DFF1F0C9CFF1F09
:102D90004C89FF1FF09CFF1F9089FF1F329CFF1F73
:102DA0000E9CFF1FE49BFF1FBE9CFF1F449DFF1F47
:102DB000109CFF1F309CFF1FE69BFF1F5A9CFF1FAC
:102DC000809CFF1F6A9CFF1FFE9CFF1F189DFF1F1A
:102DD000EC9BFF1F5E9CFF1F8C89FF1FC14B019363
:102DE0001B88002B40F06C83BF4B0393BF4B0293B7
:102DF000BF4E33786BB3DFF81483DFF8F8A24FF0DF
:102E0000000B09E003F17300C0B203F0B7FB3378A5
:102E10000BF1010B5B451CDD58F8043F99F80000ED
:102E20001844A0F17F038AFB0321DA17C2EB610289
:102E300002EB42027F28A3EB8203E3DCFDF70CFCEC
:102E4000E2E7AA4B029303F099FB009B1B78002B4F
:102E5000CED1039B1B78002B3FF4E6AB99F80030F2
:102E6000A3F10C007F2840F3A781A2488B3B80FB95
:102E70000320DA17C2EB600000EB4000A3EB8003F5
:102E800003F17300C0B203F079FB009B1B78002BA9
:102E900000F08081964E3378002B00F06582DFF8D9
:102EA0006C82DFF850A24FF0000B0AE003F17300D0
:102EB000C0B203F063FB33780BF1010B5B457FF786
:102EC000B3AB58F8043F99F800001844A0F18B0305
:102ED0008AFB0321DA17C2EB61020C3802EB4202D3
:102EE0007F28A3EB8203E1DCFDF7B6FBE0E7504669
:102EF000FDF7B2FBFFF781BBFDF7AEFBFFF7DFB9D4
:102F0000002008707C49087840B17C49009109781C
:102F1000002900F0A981009F0021397078490978C3
:102F200000297FF443A8002E67D1002865D1754E93
:102F3000724F96F800E06C4E03966C4E02966A4E05
:102F400071493070694E0097087038703070BEF16A
:102F5000000F7FF43DA8FFF744B8634B1B78002BAC
:102F60003FF4C6AC99F80030A3F10C007F2840F381
:102F7000C281604A8B3B82FB0321DA17C2EB6102FC
:102F800002EB4202A3EB820303F17300C0B203F031
:102F9000F5FA009B1B78002B3FF4AAAC544E337813
:102FA000002B3FF4A5AC594FDFF848814FF0000AE1
:102FB0000AE003F17300C0B203F0E0FA33780AF1DB
:102FC000010A53457FF794AC57F8043F99F8000085
:102FD0001844A0F18B0388FB0321DA17C2EB6102CE
:102FE0000C3802EB42027F28A3EB8203E1DCFDF701
:102FF00033FBE0E70398002101704249097800297A
:103000003EF4EFAF394902910978002900F0888138
:10301000029800210170FEF7E4BF039B1B78002B90
:103020007FF446AB029B1B78002B7FF441AB019BE6
:103030001988FFF743BB0B703B681E44A6F11800CC
:103040007F2840F301812B4B973E83FB0632F31719
:10305000C3EB620303EB4303A6EB830606F17300A5
:103060002B4BC0B2197803F061FA64E50A7073441F
:10307000A3F118007F2840F3F1801E4A973B82FBA2
:103080000321DA17C2EB610202EB4202A3EB8203D7
:1030900003F17300C0B298F8001003F047FA3B68E0
:1030A00006E6243B002BB9F8000040F32F8198423C
:1030B0003EF40FAF9BB21748A9F80030012303700C
:1030C000FEF707BFDFF84880C0B298F8001003F0A1
:1030D0002DFAFFF707BB0E4B3878197803F026FA64
:1030E0002EE500BF609CFF1F0E9CFF1FE49BFF1F8F
:1030F0004C89FF1FABAAAA2AD49BFF1F809CFF1FED
:10310000409DFF1F449DFF1F0C9CFF1F8C89FF1FCC
:10311000189CFF1F5E9CFF1F7F21402003F0DEF9FB
:10312000B349B44A3B680B600021117034E5C0B26A
:1031300098F8001003F0FAF9FFF7C8B8D8B298F879
:10314000001003F0F3F93B68B7E5AB4BDFF8ECE2B6
:103150001978FEF7BEBE4B2E40F3A9801836802E9C
:10316000B9F80030A54AA8BF8026B3427FF4FBAD72
:10317000FEF7D7BE99F8000003F000FA3188FFF798
:103180009DBA9F4B01931B88002B7FF45AAE9D4B39
:10319000029363E6029B1B78002B7FF449AA039BF2
:1031A0001B78002B7FF484AA41E7002213460A70A3
:1031B000ACE4FDF751FA0FE4FDF74EFA62E6FDF7D5
:1031C0004BFAFFE4002216460A7059E5FDF744FA6F
:1031D000FFF767B98C4E307800F07CFE8B4B1B7884
:1031E0001BB133887E2B40F2A780894B1B7823B11B
:1031F0003388854A002B40F0AB80864E3B78337095
:10320000FEF778BD824B1B78002BF6D033887E4AC0
:10321000002BF2D08049013B088899B21180002828
:103220007FF46BADC8B27B4E03F0CCF93B783370C2
:10323000FEF760BD7F20FFF7CAB9FDF70DFAFFF773
:1032400010BAFDF709FA53E4FDF706FA08E7FDF7AF
:1032500003FAFFF725BA7F20FFF7B7B8FDF7FCF9AF
:1032600018E7FDF7F9F9FCE4664F6C4902974FF057
:10327000000C81F800C0009F02994FF0010E87F802
:1032800000E081F800C049E60120FFF7A0B903F093
:1032900075F9FFF70FB90021402003F01FF9FFF780
:1032A00070BB99F8000003F069F9FFF765BB243E95
:1032B000002EB9F800303ADDB3423EF432AEB6B279
:1032C000574BA9F8006001221A70FEF72ABE0120B0
:1032D000FFF77BB84A4B01931B88002B7FF4B3ADFB
:1032E000FFF7A2B94F4A8342A8BF03461360FEF717
:1032F000CFBF16462CE5FDF7AFF947E6FDF7ACF971
:10330000FFF713BBFDF7A8F9FFF72EBB01283EF42A
:10331000E0AD0123CFE699F8000003F02FF91AE49D
:103320004148009041483D490390FEF751BE012BB2
:103330003EF4F7AD0126C3E701339BB23380D9B227
:103340000520344E03F0CAF83B783370FEF7D2BC48
:10335000013B9BB2D9B205202E4E138003F0BEF87C
:103360003B783370FEF7C6BC029B1B78002B7FF4C2
:103370005FA9FFF79DB92E4B1B782BB32D4B1B7804
:10338000002B7EF4CEAD2C4B1B78002B3EF4C9AD48
:10339000B9F8003022490A33A9F800300A70FEF764
:1033A000C0BD244B1B78002B7EF4BBAD224B1B7899
:1033B000002B3EF4B6ADB9F800301949013BA9F82D
:1033C00000300A70FEF7ADBD1A4B1B78002B7FF45E
:1033D00012AA194B1B78002B3EF4A3ADB9F80030AC
:1033E0000F490133A9F800300A70FEF79ABD00BFFB
:1033F000F09CFF1F4C89FF1F7D9CFF1FEC9BFF1F54
:10340000609CFF1FE49BFF1F109CFF1F309CFF1F51
:10341000D49BFF1F5A9CFF1FE69BFF1F0C9CFF1FA6
:103420005E9CFF1F289CFF1F809CFF1F0E9CFF1FA0
:10343000419DFF1F439DFF1F2C9CFF1F1C9DFF1FD5
:10344000224B00227F2107201A8003F047F87F21BA
:103450000B2003F043F8FFF701BA1D4B01227F2137
:1034600007201A8003F03AF87F210B2003F036F88A
:10347000FFF7ECB9174B04227F2107201A8003F0D5
:103480002DF800210B2003F029F8FFF7D8B9114BD4
:1034900002227F2107201A8003F020F87F210B20D1
:1034A00003F01CF8FFF7C6B90A4B002107201E8065
:1034B00003F014F87F210B2003F010F8FFF7B5B9E3
:1034C000054B0393054B0293BDE400BF4E9DFF1FC8
:1034D000BC9CFF1FC89BFF1F0E9CFF1FE49BFF1F90
:1034E00038B506F02FFC0B4804F0E0FC00234FF049
:1034F0007E5201210848FCF7B9FF084B084A0949E8
:10350000802400251C7118461D60BDE838400AF073
:1035100031BA00BF789CFF1F389CFF1F709CFF1FB3
:103520001C89FF1FFD05000043682A20198803F04D
:1035300059B900BF10B5044622206368198803F00A
:1035400051F9E36824201988BDE8104003F04AB916
:1035500010B504460A206368198803F043F9E3684C
:103560000C201988BDE8104003F03CB910B50446A2
:1035700006206368198803F035F9E3680820198884
:10358000BDE8104003F02EB910B504460220636870
:10359000198803F027F9E36804201988BDE8104072
:1035A00003F020B970B50E4C84B01225042201231B
:1035B00006460390029320468DE824001423102130
:1035C00005F06CFE0622092302930396019520461E
:1035D00000921423102105F061FE04B070BD00BFFD
:1035E000789DFF1F2DE9F041224D82B0012602B2E5
:1035F00084B20092284601967823192105F094FDA3
:1036000004F10C0212B28DE844002846A719782371
:10361000192104F1020805F087FD3FB20FFA88F87E
:1036200019233A46284619460196CDF8008005F040
:103630007BFD78233A4628461946CDF8008001964E
:1036400004F10A070B3405F06FFD3FB224B2782372
:103650003A46284619468DE8500005F065FD1923C5
:1036600000943A4601962846194605F05DFD02B0E1
:10367000BDE8F081789DFF1F2DE9F0411E4682B024
:103680001446002A6AD0099B4D4A00EBC305012C61
:103690006F8929896868A7EB010382FB03E21A445A
:1036A0004FEAE373C3EBA21302887BD0042C38D11A
:1036B00012FA83F3994203DC9F423946A8BF1946A8
:1036C000089A0180B6F90030BDF920803D48971D69
:1036D0004FF0000E3FB2194642460097CDF804E085
:1036E00005F022FD29896A896B68521A1B885C2AB9
:1036F000A3EB010359DD03EB43030132C3EB431397
:1037000093FBF2F303F11B0213B20120328019463E
:103710004246019000972B4805F006FD2A4B0022F7
:103720001A702A4B022CB3F9001045D0082C31D165
:1037300000221A8091422DD0089AB6F90030214813
:103740000632012412B2009219460194BDF92020DC
:1037500005F0EAFC204602B0BDE8F0811C4D1D4A90
:103760002B681268CB1A93420F4617D9164A338832
:1037700011781448012918BF01241470089A0632E0
:103780001BB212B28DE814001946BDF9202005F0D5
:10379000CBFC2F60012002B0BDE8F081204602B0D2
:1037A000BDE8F0819BB2D31A84E75C2101FB03F3EF
:1037B00093FBF2F21B32A7E74A1C12B21A80B9E758
:1037C000C94216B2789DFF1FFE9DFF1F609DFF1F1F
:1037D000E09DFF1FCCF8000030B583B000230C46FD
:1037E00005B2009326225B231C210C4805F0ECF95E
:1037F000294601232622094804F002FD002C24B2A8
:1038000005DB214601232622044804F0F9FC044A82
:10381000044B15801C8003B030BD00BF789DFF1F96
:10382000C689FF1FC889FF1F70B5944C237882B0EA
:103830001BB1934B4FF6FF721A80924BB3F90030D5
:10384000C3B9914A8E4B1068B3F9002080F30C0085
:103850005B2303FB00F000131C3082425AD04FF070
:10386000FF31FFF7B9FF894805F012FA00232370F2
:1038700002B070BD012B32D0022B6AD0032B4FD087
:10388000042BF3D1272200258DE8240076231C2168
:103890007E487F4E05F048FC17E0B0F5AF7FA8BF2B
:1038A0004FF4AF70323803FB00F386FB0321DB17C4
:1038B000C3EB61111C3109B201231D442722734857
:1038C00004F09EFC0C2D00F08180E9B2714804F0F8
:1038D00055FB31284FF05B03DFDC1C21ECE76E4B1E
:1038E0001A68B2F52F7F32DB41F25C239342A8BF06
:1038F0001346A3F52F735B22684802FB03F380FB9A
:103900000320DB17C3EBA0201C305D4BB3F9003064
:103910008342A4D1624BB3F9003001339FD1A5E7B4
:10392000604B1B68B3F5FA7F11DBB3F57A6FA8BF64
:103930004FF47A63A3F5FA725B485B2303FB02F34F
:1039400080FB0320DB17C3EB20201C30DDE71C20AD
:10395000DBE7564B1B68B3F5FA7F33DBB3F57A6FC1
:10396000A8BF4FF47A63A3F5FA724F485B2303FBB9
:1039700002F380FB0320DB17C3EB20201C304C4BF1
:103980001B68B3F5FA7F1FDBB3F57A6FA8BF4FF45E
:103990007A63A3F5FA7244495B2303FB02F381FBCC
:1039A0000321DB17C3EB21211C31354BB3F9003068
:1039B00083427FF456AF3A4BB3F900308B427FF429
:1039C00050AF53E71C20DAE71C21EEE7012006F098
:1039D00099FF6FF495733238364A03FB00F082FB8F
:1039E0000023C017C0EB632303F5AF73312B3ADD1F
:1039F000B3F5AF7FA8BF4FF4AF735B22323B244DCA
:103A000002FB03F385FB0325DB17C3EB65151C35B0
:103A1000002006F077FF6FF495733238254A03FBD8
:103A200000F082FB0023C017C0EB632303F5AF73E4
:103A3000312B1ADDB3F5AF7FA8BF4FF4AF735B2214
:103A4000323B134902FB03F381FB0321DB17C3EB7A
:103A500061111C310A4BB3F90030AB4207D0284644
:103A6000FFF7BAFEFFE61C25D2E71C21F2E70C4B5C
:103A7000B3F900308B42F2D1F5E600BF569DFF1F2F
:103A8000C689FF1F5C9DFF1FCC9BFF1F789DFF1FFA
:103A90004B48371B789CFF1F0C9DFF1FD3058541AA
:103AA000C889FF1F189DFF1F011FB812C09BFF1F71
:103AB000889CFF1F67BBCF462DE9F04FDFF8F092DF
:103AC000B84CB9F900504E7854F8255087B00290A0
:103AD000039306B10E78DFF800B3002A35D19BF8C6
:103AE0000030002B31D1B04FB7F90000002800F0B2
:103AF000CE80012800F0248101203223324601903B
:103B000000930299A94B2846FFF7B6FD002604460C
:103B1000B7F90030022B40F3F48000233B80B9F961
:103B20000030A34A002BC0F2F880042BC4BF00234E
:103B30001380039B002B40F0F680002E0CBF204624
:103B40004FF0FF3007B0BDE8F08F9A4C964FEB680E
:103B50002A6804934FF0000820460592A7F80080D9
:103B60008BF8008004F088FF1120FFF73BFD4FF039
:103B7000010A192328212046CDF804A0009124220F
:103B8000194605F0D1FA782328212422CDF804A083
:103B900000912046194605F0C7FA5146204605F027
:103BA0004DFEDDF814A0022319222382E281504643
:103BB0000AF0A6FC51460246204608F09DFA20462F
:103BC00008F0B0FA142303227B4923822046A4F88C
:103BD0000E8008F091FA204608F0A4FA23232382ED
:103BE00003227649A4F80E80204608F085FA204684
:103BF00008F098FA049B002B73D10123704A1846F1
:103C00001370FFF7CFFC28896B896C68191A5C293F
:103C100022885CDC131A5C2202FB03F292FBF1F3B4
:103C20001B33684A6348138001241BB21A221946C9
:103C30008DE81400142205F077FA049BDBB1298A81
:103C40006B8AEC68581A5C2822886FDD521A02EBE6
:103C50004202C2EB4212431C92FBF3F31B33534A62
:103C600054481380012438221BB28DE814001946F1
:103C7000322205F059FA544A544BB7F90000012199
:103C800011704FF6FF721A8000287FF432AFDFF810
:103C90004C814F4AD8F8003002991268CB1A9342EF
:103CA0004CD9474B1A78012A18BF01201870FFF72A
:103CB00079FC029BC8F800300124012E4DD0042E5F
:103CC00058D0022E5FD0082E63D0002620E7121AAB
:103CD00002EB4202C2EB42124B1C92FBF3F31B338A
:103CE0009FE72F20FFF77EFC322303223949A4F8F7
:103CF0000E802046238208F0FFF9204608F012FAD1
:103D00007BE77FF40CAFEB68002B3FF406AFB9F90B
:103D10000030274A002BBFF608AF04231380039B13
:103D2000002B3FF40AAFFFF77FFD06E7511A5C2234
:103D300002FB01F292FBF0F31B3390E70446BCE771
:103D4000002414238DE81800324602991D4B2846A2
:103D5000FFF792FC26460446DAE6B9F800308BF805
:103D600000600133A9F800306B6983B10026284652
:103D70009847CDE6B9F800300122013BA9F80030A0
:103D80008BF80020F0E701233B800026C7E61E46A3
:103D9000BEE66B6900223A804FF0FF36002BE6D179
:103DA000BDE600BFCC89FF1F609DFF1F5A9DFF1F0E
:103DB0005C9DFF1F789DFF1F64ED000068ED000013
:103DC000FE9DFF1F589DFF1F569DFF1FC689FF1FA9
:103DD000CCF800006CED00005E9DFF1FE09DFF1F12
:103DE00001210D2006F060BB00210D2006F05CBB18
:103DF00001460D2006F058BB08B50D2006F05AFB11
:103E0000B0FA80F149090D20BDE8084006F04CBB2E
:103E100010B5002144080D2006F046FB204606F0B0
:103E20007FFB0D20012106F03FFB2046BDE810403E
:103E300006F076BB08B5214A214B128818688242E9
:103E400034DA204B1B88991A8342A8BF0346B1F588
:103E5000F87FA3EB020321DAC3EB031303EB431355
:103E600093FBF1F105310A2006F08EF9164B197813
:103E7000F1B1164B16491B6883F30703C3EB031319
:103E800003EB431381FB03211944DB17C3EBA1119F
:103E900005310920BDE8084006F076B9C3EB4313AD
:103EA0001B01013193FBF1F10531DCE70021DAE779
:103EB0000920BDE8084006F067B900BF329CFF1F2B
:103EC000289CFF1F549DFF1F029DFF1FD49CFF1FB6
:103ED000090402817F2838B5A8BF7F200D4D4FF41B
:103EE000FA7303FB00F485FB04232344E117C1EBC1
:103EF000A3110A2006F048F9A4F578400C3885FB98
:103F000000310144C017A0EBA111BDE838400920E1
:103F100006F03AB909040281024B4E20198802F0DA
:103F200061BC00BF609CFF1F024B4420198802F057
:103F300059BC00BF009DFF1F024B1020198802F0E2
:103F400051BC00BF7E9CFF1F024B2C20198802F041
:103F500049BC00BFA69CFF1F024B1E20198802F01F
:103F600041BC00BF7A9CFF1FC3680E20198802F075
:103F700039BC00BF024B2820198802F033BC00BFB7
:103F80005C9CFF1F024B6220198802F02BBC00BF13
:103F90009A9CFF1F024B6420198802F023BC00BFCB
:103FA000A29CFF1F024B5A20198802F01BBC00BFC5
:103FB000D69BFF1F024B1620198802F013BC00BFCE
:103FC0004E9DFF1F024B2E20198802F00BBC00BF34
:103FD000C09CFF1F024B3020198802F003BC00BFB9
:103FE000C49BFF1F024B1820198802F0FBBB00BFC7
:103FF000689CFF1F024B1A20198802F0F3BB00BF18
:10400000CE9CFF1F024B1C20198802F0EBBB00BFA7
:10401000F89CFF1F024B6620198802F0E3BB00BF2B
:10402000B49BFF1F024B7220198802F0DBBB00BF5C
:104030003E9DFF1F024B2020198802F0D3BB00BF1A
:10404000529DFF1F024B3220198802F0CBBB00BFEC
:10405000349CFF1F024B6820198802F0C3BB00BFCD
:10406000E69BFF1F024B5220198802F0BBBB00BF2A
:10407000C489FF1F024B5020198802F0B3BB00BF58
:104080008C89FF1F024B5420198802F0ABBB00BF84
:10409000B489FF1F024B5C20198802F0A3BB00BF4C
:1040A0008E89FF1F024B5E20198802F09BBB00BF68
:1040B000BC89FF1F024B6020198802F093BB00BF30
:1040C000C69BFF1F024B5620198802F08BBB00BF16
:1040D000509DFF1F38B5094D4624204602F09CFB39
:1040E00035F8021B00B28842204601D002F07AFB6C
:1040F0000234A4B24E2CF0D138BD00BF249DFF1F66
:10410000064B074A10B41C88064B0846002C14BF07
:1041100011461946042210BC0AF0B0BAFA9CFF1FDF
:1041200058F400005CF40000064B074A10B41C88E9
:10413000064B0846002C14BF11461946042210BC39
:104140000AF09CBA589CFF1F58F400005CF4000071
:10415000064B074A10B41C88064B0846002C14BFB7
:1041600011461946042210BC0AF088BA8C9CFF1F25
:1041700058F400005CF40000064B074A10B41C8899
:10418000064B0846002C14BF11461946042210BCE9
:104190000AF074BAF49CFF1F58F400005CF40000AD
:1041A000064B074A10B41C88064B0846002C14BF67
:1041B00011461946042210BC0AF060BAFC9CFF1F8D
:1041C00058F400005CF40000064B074A10B41C8849
:1041D000064B0846002C14BF11461946042210BC99
:1041E0000AF04CBA469DFF1F58F400005CF4000032
:1041F000064B074A10B41C88064B0846002C14BF17
:1042000011461946042210BC0AF038BABC9CFF1FA4
:1042100058F400005CF40000F0B52B4E2B4FDFF893
:10422000C4E005460FCE87B06C460FC496E8030085
:104230003B68274A274F44F8040B40F6CC308342B2
:10424000C8BF3A46BEF800602180012E11889278DE
:10425000ADF80D108DF80F202AD032D340F6CA02E7
:10426000022E18BF00229A4226DCA3F698031A49B0
:104270001A4AC3EB031381FB03011944DB17C3EB99
:104280006123243382FB0321DA17C2EBA10202EB84
:104290008201A3EB4103303330328DF813308DF8B7
:1042A00011206946284616220AF0E8F907B0F0BD49
:1042B00040F698029A42D8DD094B1868CDF81100F3
:1042C000EFE740F6FC02CEE770F40000D09CFF1F41
:1042D00064F4000060F400003B773B986766666614
:1042E00068F40000389DFF1FF8B5174C174E227870
:1042F000174D33782F888E46003218BF01220146B1
:104300007046FFF7D9FB002398423370237015DB0A
:1043100014BF012000202B889F420ED040F23A7239
:10432000A3F5AF730B490C4C02FB03F381FB0312A3
:10433000DB17A3EB621332332360F8BD0749012278
:1043400018460A702270E6E7708AFF1F719DFF1FF2
:10435000A49CFF1FB5814E1BB889FF1F6A9DFF1FDC
:10436000014B187802F0D6B9DC9DFF1F014B18787D
:1043700002F0EAB9AC8FFF1F134BB3F9003030B530
:1043800083EAE374A4EBE374002BA0B218DB0123EF
:1043900000E0134603EB830252009442F9DA0B4D1E
:1043A00090FBF3F285FB03E403FB1200DB173032D2
:1043B000D3EBA40380B201F8012BF1D10B7030BD17
:1043C0002D230B700131E2E7AC8FFF1F6766666635
:1043D000144BB3F9003070B583EAE375A5EBE375D0
:1043E000002BACB21ADB012300E0034603EB830091
:1043F00040008542F9DA0C4E94FBF3F086FB03E5AE
:1044000003FB1044DB173030D3EBA503A4B201F853
:10441000010BF1D105480B70106070BD2D230B709E
:104420000131E0E7D69BFF1F6766666688F40000EF
:10443000134BB3F9003030B583EAE374A4EBE374B3
:10444000002BA0B218DB012300E0134603EB83022C
:1044500052009442F9DA0B4D90FBF3F285FB03E432
:1044600003FB1200DB173032D3EBA40380B201F858
:10447000012BF1D10B7030BD2D230B700131E2E720
:10448000C489FF1F67666666134BB3F9003030B509
:1044900083EAE374A4EBE374002BA0B218DB0123DE
:1044A00000E0134603EB830252009442F9DA0B4D0D
:1044B00090FBF3F285FB03E403FB1200DB173032C1
:1044C000D3EBA40380B201F8012BF1D10B7030BD06
:1044D0002D230B700131E2E78C89FF1F676666664A
:1044E000134BB3F9003030B583EAE374A4EBE37403
:1044F000002BA0B218DB012300E0134603EB83027C
:1045000052009442F9DA0B4D90FBF3F285FB03E481
:1045100003FB1200DB173032D3EBA40380B201F8A7
:10452000012BF1D10B7030BD2D230B700131E2E76F
:10453000B489FF1F67666666134BB3F9003030B568
:1045400083EAE374A4EBE374002BA0B218DB01232D
:1045500000E0134603EB830252009442F9DA0B4D5C
:1045600090FBF3F285FB03E403FB1200DB17303210
:10457000D3EBA40380B201F8012BF1D10B7030BD55
:104580002D230B700131E2E78E89FF1F6766666697
:10459000134BB3F9003030B583EAE374A4EBE37452
:1045A000002BA0B218DB012300E0134603EB8302CB
:1045B00052009442F9DA0B4D90FBF3F285FB03E4D1
:1045C00003FB1200DB173032D3EBA40380B201F8F7
:1045D000012BF1D10B7030BD2D230B700131E2E7BF
:1045E000BC89FF1F67666666054B1B881BB9054BB8
:1045F000186808607047044B18680860704700BF6F
:10460000609CFF1F90F400008CF40000164B1B8888
:104610000BB31BB230B583EAE374A4EBE374002B55
:10462000A0B21CDB012300E0134603EB830252001F
:104630009442F9DA0D4D90FBF3F285FB03E403FBA2
:104640001200DB173032D3EBA40380B201F8012B48
:10465000F1D10B7030BD064B1868086070472D23F0
:104660000B700131DEE700BF7A9CFF1F676666664C
:104670005CF40000164B1B880BB31BB230B583EA09
:10468000E374A4EBE374002BA0B21CDB012300E075
:10469000134603EB830252009442F9DA0D4D90FB6E
:1046A000F3F285FB03E403FB1200DB173032D3EB9C
:1046B000A40380B201F8012BF1D10B7030BD064B81
:1046C0001868086070472D230B700131DEE700BFCA
:1046D000CA9CFF1F676666665CF40000164B1B8869
:1046E0000BB31BB230B583EAE374A4EBE374002B85
:1046F000A0B21CDB012300E0134603EB830252004F
:104700009442F9DA0D4D90FBF3F285FB03E403FBD1
:104710001200DB173032D3EBA40380B201F8012B77
:10472000F1D10B7030BD064B1868086070472D231F
:104730000B700131DEE700BF4E9DFF1F67666666A6
:1047400094F40000174B1B881BB31BB270B583EAAF
:10475000E375A5EBE375002BACB21EDB012300E093
:10476000034603EB830040008542F9DA0E4E94FBCA
:10477000F3F086FB03E503FB1044DB173030D3EB8B
:10478000A503A4B201F8010BF1D108480B70106029
:1047900070BD074B1868086070472D230B700131FE
:1047A000DCE700BFC09CFF1F676666666CF4000014
:1047B0005CF40000164B1B880BB31BB230B583EAC8
:1047C000E374A4EBE374002BA0B21CDB012300E034
:1047D000134603EB830252009442F9DA0D4D90FB2D
:1047E000F3F285FB03E403FB1200DB173032D3EB5B
:1047F000A40380B201F8012BF1D10B7030BD064B40
:104800001868086070472D230B700131DEE700BF88
:10481000C49BFF1F676666665CF40000164B1B882E
:104820000BB31BB230B583EAE374A4EBE374002B43
:10483000A0B21CDB012300E0134603EB830252000D
:104840009442F9DA0D4D90FBF3F285FB03E403FB90
:104850001200DB173032D3EBA40380B201F8012B36
:10486000F1D10B7030BD064B1868086070472D23DE
:104870000B700131DEE700BFB49BFF1F6766666601
:104880005CF40000164B1B880BB31BB230B583EAF7
:10489000E374A4EBE374002BA0B21CDB012300E063
:1048A000134603EB830252009442F9DA0D4D90FB5C
:1048B000F3F285FB03E403FB1200DB173032D3EB8A
:1048C000A40380B201F8012BF1D10B7030BD064B6F
:1048D0001868086070472D230B700131DEE700BFB8
:1048E0003E9DFF1F676666665CF40000174B1B88E1
:1048F0001BB31BB270B583EAE375A5EBE375002B20
:10490000ACB21EDB012300E0034603EB8300400052
:104910008542F9DA0E4E94FBF3F086FB03E503FBC8
:104920001044DB173030D3EBA503A4B201F8010B20
:10493000F1D108480B70106070BD074B1868086013
:1049400070472D230B700131DCE700BF529DFF1F24
:104950006766666698F400005CF40000074B1B88ED
:10496000022B06D0012B0CBF054B064B18680860C4
:104970007047054B18680860704700BFC69BFF1F53
:10498000A0F40000A4F400009CF40000054B1B8878
:104990001BB1054B186808607047044B1868086025
:1049A000704700BF509DFF1FACF40000A8F400004A
:1049B00008B5702001F030FF044B1988884204D0FC
:1049C0007020BDE8084001F00DBF08BD389DFF1FF5
:1049D00008B5742001F020FF044B1988884204D0E8
:1049E0007420BDE8084001F0FDBE08BD949CFF1F87
:1049F00038B5FCF7E5FF0D4B1B7833B90C4B102095
:104A0000198801F0EFFE012038BD0A4D0A4C2B78C1
:104A10002288B3FA83F382F008025B091146422030
:104A20002B70228001F0DEFE002038BD449DFF1F68
:104A30007E9CFF1F149DFF1FFC9BFF1F184B1A88B5
:104A400052B3184A128830B50A80B3F90030002BEF
:104A500083EAE374A4EBE374BCBF2D238B70A0B294
:104A6000ACBF02310331012300E0134603EB8302A4
:104A700052009442F9DA0C4D90FBF3F285FB03E40B
:104A800003FB1200DB173032D3EBA40380B201F832
:104A9000012BF1D10B7030BD044B186808607047D2
:104AA000CE9CFF1FB0F40000676666665CF40000F1
:104AB00010B40A4B0A4C0A4693E8030083B02388DB
:104AC00002AC04E9030004EB8303104653F8081C0E
:104AD000052203B010BC09F0D1BD00BFF4ED000009
:104AE000A29CFF1F30B40A4B0A4D0C4693E8070006
:104AF00084B02B8804AD05E9070005EB830320464D
:104B000053F80C1C042204B030BC09F0B7BD00BF40
:104B1000FCED0000389DFF1FF0B40C4D0C4F0E460D
:104B20000FCD8CB001AC0FC40FCD0FC495E80700BA
:104B30003B8884E807000CAA02EB8303304653F855
:104B40002C1C04220CB0F0BC09F098BD08EE00004B
:104B5000C89BFF1FF0B40A4D0A4F0E460FCD86B01A
:104B600001AC0FC42A683B88226006AA02EB8303CB
:104B7000304653F8141C042206B0F0BC09F07EBD88
:104B800034EE0000689CFF1FF0B40A4D0A4F0E4639
:104B90000FCD86B001AC0FC42A683B88226006AAFC
:104BA00002EB8303304653F8141C0C2206B0F0BC11
:104BB00009F064BD48EE0000F89CFF1FF0B40A4DF8
:104BC0000A4F0E460FCD86B001AC0FC42A683B8851
:104BD000226006AA02EB8303304653F8141C042219
:104BE00006B0F0BC09F04ABD5CEE0000949CFF1FCB
:104BF000164B1B880BB31BB283EAE370A0EBE37088
:104C0000002B30B584B21DDB012300E0134603EB1B
:104C1000830252009042F9DA0D4894FBF3F280FBD4
:104C200003E503FB1244DB173032D3EBA503A4B238
:104C300001F8012BF1D10B7030BD08460422054963
:104C400009F01CBD2D230B700131DDE7E69BFF1F32
:104C500067666666B4F4000070B53C4D2B78064676
:104C6000002B35D11C4673780BB9204670BDFCF77C
:104C7000A7FE374A374B3848127831781B780078CE
:104C800002EB43034A1E03EB80030E2AEDD801A07A
:104C900050F822F0FD4C00001F4D00006B4C00004E
:104CA000FD4C00006B4C00006B4C00006B4C000096
:104CB000EB4C00006B4C00006B4C00006B4C000098
:104CC0006B4C00006B4C00006B4C0000E74C00008C
:104CD000AE21224803F084FC204803F0CDFE0023DF
:104CE0002B700124BFE705F02DFFAF211B4803F017
:104CF00077FC1B4A012313702B70B6E783B9194860
:104D0000038804294FF6FF7103F1FF320CBF012322
:104D10000B46134403F07F03013303800FE073B1AC
:104D2000013B114A32F813304BB10E4E0F48104977
:104D3000104A33800123002606700B701370084A56
:104D40000221012311702B70204670BD708AFF1F55
:104D5000D49BFF1F309CFF1F4C9DFF1F789DFF1FA2
:104D60006A9DFF1FEC9BFF1FA89CFF1F159DFF1F47
:104D70005E9CFF1F009EFF1F10B5064B064C1A8855
:104D80002046012101F01CFD21884220BDE8104091
:104D900001F028BDFA9CFF1FFC9BFF1F10B5064BBE
:104DA000064C1A882046022101F00AFD2188422083
:104DB000BDE8104001F016BD589CFF1FFC9BFF1F73
:104DC00010B5064B064C1A882046042101F0F8FC69
:104DD00021884220BDE8104001F004BD8C9CFF1FDB
:104DE000FC9BFF1F10B5064B064C1A882046052178
:104DF00001F0E6FC21884220BDE8104001F0F2BC41
:104E0000F49CFF1FFC9BFF1F10B5064B064C1A8835
:104E10002046062101F0D4FC21884220BDE8104044
:104E200001F0E0BCFC9CFF1FFC9BFF1F10B5064B74
:104E3000064C1A882046002101F0C2FC218842203D
:104E4000BDE8104001F0CEBC469DFF1FFC9BFF1F3C
:104E500008B5122001F0E0FC054B1988884206D005
:104E6000122001F0BFFCBDE8084001F0D3BB08BD33
:104E7000C89BFF1F08B5582001F0CEFC054B1988D0
:104E8000884206D0582001F0ADFCBDE8084001F092
:104E9000C1BB08BDCA9CFF1F08B5142001F0BCFCB3
:104EA000054B1988884206D0142001F09BFCBDE810
:104EB000084001F0AFBB08BDBC9CFF1FF0B480EA06
:104EC000E075A5EBE0750028ACB21FDB1DBF2B23FE
:104ED0000B704E1C0E46012300E0134603EB8302C9
:104EE00052009542F9DA0B4F94FBF3F287FB03056E
:104EF00003FB1244DB173032D3EBA503A4B206F850
:104F0000012BF1D133700846F0BC70472D230B7094
:104F10004E1CE0E767666666174B18880C2813D0AE
:104F2000192815D01A2817D01B2819D01C281BD0D7
:104F30001D281DD01E2803D00C3800B2FFF7BEBFBD
:104F40000E4A1068086070470D4A10680860704784
:104F50000C4A1068086070470B4A10680860704778
:104F60000A4A106808607047094A1068086070476C
:104F7000084A106808607047349CFF1FD4F4000092
:104F8000BCF40000C0F40000C4F40000C8F4000049
:104F9000CCF40000D0F40000034B1888A0EB800094
:104FA000400000B2FFF78ABFDC9DFF1F024BB3F940
:104FB0000000FFF783BF00BF9A9CFF1F024B1888B9
:104FC000033800B2FFF77ABF5C9CFF1F024B1888C2
:104FD0000C3800B2FFF772BF0A9DFF1F024B188802
:104FE000183800B2FFF76ABF009DFF1FC36818881A
:104FF000183800B2FFF762BF30B5134C85B00125F9
:105000002B463C2202212046009503F05FFB204600
:1050100003F032FD002240218023204601910093BD
:1050200011460A4B029504F0D5F9204603F030FEF4
:1050300007480849084A0023036083800B608B807F
:105040001360938005B030BD789DFF1FD0EE000047
:10505000649DFF1FF89DFF1FE89DFF1F10B500EB2B
:10506000C00000F10F02D2B293B284B09C1E981C13
:105070003D2303918DE819003921024804F00EF90F
:1050800004B010BD789DFF1F014B01221A707047BC
:10509000719DFF1FF0B585B0664C674B0293674A60
:1050A0000192042300932046654B664F664E674D80
:1050B0004022802103F012F92046654A6549664C7A
:1050C00008F058FC654B66489F61664FDF61664F8C
:1050D000B761664FF761664FAF61664FEF61664F2C
:1050E000A761664FE761664F87616649664FC76192
:1050F000664F8F61664A674FCF61674F9761674B15
:10510000674FD761674F9F61674E684FDF61684F98
:10511000B761684D684FF761684F694CAF61694F7F
:10512000EF61694F6948A761694FE761694F6A4953
:1051300087616A4FC7616A4F6A4A8F616A4FCF6160
:105140006A4F6B4B97616B4FD7616B4F6B4E9F6193
:105150006B4FDF616B4F6C4DB7616C4FF7616C4FFC
:10516000AF616C4C6C4FEF616C4FA7616C486D4F39
:10517000E7616D4F87616D496D4FC7616D4F8F61FD
:105180006D4A6E4FCF616E4F97616E4B6E4FD76118
:105190006E4F9F616E4E6F4FDF616F4FB7616F4D06
:1051A0006F4FF7616F4FAF616F4C704FEF61704F92
:1051B000A7617048704FE761704F87617049714F08
:1051C000C761714F714A8F61714FCF61714F724BDF
:1051D0009761724FD761724F724E9F61724FDF615C
:1051E000724F734DB761734FF761734F734CAF617B
:1051F000734F74487449EF61744F754DA761E56151
:10520000744F754D754CDFF8F8E1754A754B876141
:10521000754EC561754F8C61754D764CC1F81CE0BB
:10522000754876499761D5619C61D861B16005B0D8
:10523000F0BD00BF789DFF1FA0860100801A060008
:10524000D48FFF1FCD4F0000148EFF1F848DFF1FD2
:105250001C89FF1F35830000908BFF1FD48CFF1F1C
:10526000388EFF1F693F0000BD4F0000753F0000F2
:1052700001410000794D0000294100009D4D0000D2
:1052800051410000688CFF1FC14D000079410000B2
:10529000048AFF1FE54D0000AD4F0000208CFF1F6A
:1052A000853F0000A1410000B08FFF1F094E0000A4
:1052B000B14A0000FC8BFF1F953F0000C941000070
:1052C000B08CFF1F2D4E0000994F00008C8CFF1FEB
:1052D0006143000079430000F08DFF1F6D43000023
:1052E000E54A0000488BFF1FB1490000194B000040
:1052F000A08EFF1F514E000075460000D88BFF1F87
:10530000754E0000D1430000048BFF1FA53F000035
:10531000F14100000C8FFF1F994E0000DD46000098
:10532000B48BFF1FB53F000045470000F88CFF1FFE
:10533000C53F0000B5470000748AFF1FD53F00003D
:10534000554B0000448CFF1FE53F00003D4A000024
:10535000CC8DFF1FF53F0000894B0000888FFF1F99
:10536000054000001D480000608DFF1F1540000033
:1053700085480000988AFF1F25400000BD4B0000B3
:10538000C48EFF1FD1490000ED480000A88DFF1F0B
:1053900035400000194F0000BC8AFF1F4540000047
:1053A000F14B0000588FFF1F5540000031440000B2
:1053B0006C8BFF1F65400000894400004C8AFF1F72
:1053C00075400000E08AFF1F5C8EFF1FE144000073
:1053D00085400000394500009540000091450000DF
:1053E000288AFF1FE089FF1F7C8FFF1F5D49000097
:1053F000B54000008D490000C5400000B1590000D3
:10540000A5400000F0B5461C83B00D4601270323DC
:1054100036B22AB2044631468DE888002448ADB23F
:1054200003F0D2FE0C23AA1C12B2009301970523AD
:1054300021B21F4803F0C8FE1E4A1F4B12881B688A
:10544000BA422AD023D3022A10D11C4CA3F6CA0395
:1054500084FB03241C44DB17C3EB24140A2CA8BFD1
:105460000A2424EAE474A2B223B202E000231A461A
:105470001C460D35AA1A01200093019012B2314644
:1054800003230B4803F01EFE204603B0F0BD0C4C76
:10549000A3F6FC0384FB0324DDE7084CA3F6980382
:1054A00084FB03241C44DB17C3EBE404D6E700BFF2
:1054B000789DFF1F389DFF1FD09CFF1F898888881B
:1054C0001F85EB512DE9F0438FB283B0DFF84C809C
:1054D000BD1D461D2DB204B236B24FF001090AB20D
:1054E0002346314640460095CDF8049003F01CFE5B
:1054F0002A463346214640468DE8200203F014FE3A
:1055000007F10C020095334612B22146CDF8049003
:10551000404603F009FE03B0BDE8F083789DFF1F0D
:105520002DE9F04F804685B0002959D1012131483D
:1055300004F084F9304998F8062098F8083011F8FA
:105540000290994525DADFF8ACB04FEA89064D465E
:105550000C244FF0000AD8F80C309B595F68ABF868
:1055600010403846ABF80EA008F0CAFF3946024694
:10557000204806F0C1FD1F4806F0D4FD98F8083019
:1055800001350934AB42A4B206F1040601DD422C18
:10559000E1D1B9F1000F13D109F1060999450CDAEF
:1055A0003C2301213B220391029300930192392372
:1055B0003F223A210F4803F071FE05B0BDE8F08F9D
:1055C0000F2301213B22039102930093019239237F
:1055D0000C223A21074803F061FE98F80830DBE717
:1055E00000213423009301913F230C22014803F052
:1055F00069FD9BE7789DFF1FF89DFF1F38B50F4C95
:10560000012320461946A3826382552504F016F92A
:105610003423204602220A492382E58106F06CFDEC
:1056200020460522074906F067FD204606F07AFD70
:105630002046BDE8384003F02BBB00BF789DFF1F1C
:10564000D8F40000DCF40000F8B50F46064608F078
:1056500057FF00EB40008400AFB3384608F050FF1E
:1056600000EB4000400023185B10194D03F160026D
:10567000121A4FF0280E01212846C3F16004EA8176
:10568000A5F810E004F0DAF8384608F039FF39469A
:105690000246284606F030FD284606F043FD02216A
:1056A0000B4804F0CBF8212330462B82EC8108F024
:1056B00027FF31460246064806F01EFD0448BDE8B5
:1056C000F84006F02FBD6410C4F16004004DE6E719
:1056D000789DFF1F10B50D4B1B5C51F823402378BC
:1056E00084B013B1012004B010BD04AA01A942F88E
:1056F000103D2046A3699847A38A9B07F2D401A8CE
:105700000099FFF7A1FF012004B010BD649DFF1FA9
:105710002DE9F04F304DDFF8D0B0DFF8C8A00FCD45
:1057200091B003AC0FC40FCD0FC40FCD0FC42B68C5
:1057300023600025A8462F462E4600E09846BAF87A
:10574000003026495BF82320DFF8A090112328467B
:10575000FBF71AF900EBC00300EB8300204B83FB3F
:1057600000340444C017C0EB6434C4F13C00C6F1FB
:105770003C0207F14101012600B208F1410300900B
:105780001BB2019612B209B2484603F0CDFC08EBF9
:10579000060305F211153C2B2646ADB24746CDD186
:1057A0006B22342300214846A9F80E20A9F81030B6
:1057B00004F044F80B4B1B8810AA02EB830353F848
:1057C000344C204608F09CFE21460246484611B063
:1057D000BDE8F04F06F090BC84EE000060EA0000E7
:1057E00009000280A69CFF1FC8EB0000789DFF1FE8
:1057F000214B70B5B3F9003083EAE374A4EBE37492
:10580000002B82B0A1B22FDB68466D46012300E079
:10581000134603EB830252009442F9DA174E91FBD0
:10582000F3F286FB03E403FB1211DB173032D3EBF8
:10583000A40389B205F8012BF1D119462B70FFF7AB
:1058400003FF0F4B1B786BB10E4C0121204603F078
:10585000F5FF74253323204601220B49E58123827D
:1058600006F04AFC02B070BD2D238DF800300DF11A
:1058700001056846CAE700BF7E9CFF1F6766666633
:10588000149DFF1F789DFF1F7CF8000070B5404EEF
:10589000404D82B0304603F0EFF82B78D3B93C4C42
:1058A0000621204603F0CAFF2B78012B38D9022BA2
:1058B0004FF003024FF00A030CBF37493749E38129
:1058C0002046238206F018FC204602B0BDE8704056
:1058D00006F028BC324B1A7801210523002A33D167
:1058E000019100931146304603F06EFC2D4B1A785F
:1058F000002A34D0052301220192009300220A21BC
:10590000234803F0DFFB284B1A78002A33D101210A
:1059100005230191009314211D4803F055FCBEE7B7
:10592000224B1988092930D963298CBF0A221F22EA
:105930000A231748F281338206F044FC144802B06F
:10594000BDE8704006F0EEBB0022019100931146C5
:10595000304603F0B7FB134B1A78002ACAD105234F
:105960000121019100930A21094803F02DFC0E4BFF
:105970001A78002ACBD0012205230192009300223D
:105980001421034803F09EFB89E73022D0E700BFD3
:10599000789DFF1F009EFF1FE4F40000E8F4000064
:1059A000D49BFF1F309CFF1F4C9DFF1FEC9BFF1FD4
:1059B0002DE9F047714E307848B9714B1B68994218
:1059C0005FD3704A012313703370BDE8F0876E4DCA
:1059D0006B4F0C46284603F04FF804F6AC533124C5
:1059E0000022EC810124114628462A82AC826C8276
:1059F0003B60327003F022FF05226449644E284662
:105A000006F07AFB102728464FF00C0806F08AFBB8
:105A10000B226049EF812846A5F8108006F06CFB48
:105A20005D490522284606F067FB284606F07AFB0A
:105A30005A4BEF811A68A2F69803C3EB031386FB57
:105A400003161E44DB17C3EB662640F6CC33202139
:105A50009A42298206F124064FF022014FF00400F9
:105A600011DCFFF7CFFC4E4BB3F800908246B9F142
:105A7000000F30D0B9F1010F4DD0B9F1020F47D06E
:105A80002046BDE8F087FFF71DFD4649092228465C
:105A900006F032FB4449EF8181FB0637F317C3EB75
:105AA000A7072A23394628462B8206F08BFB22467D
:105AB0003E49284606F020FB07EB8701A6EB410193
:105AC000284606F07FFB22462846394906F014FB9B
:105AD0002046BDE8F08737493A46284606F00CFBD9
:105AE000284606F01FFB2A232B825146EF812846C9
:105AF0002D4F06F067FB07222F49284606F0FCFAD7
:105B0000F31787FB0627C3EBA70739462846CCE7E0
:105B100042462A49E1E742462949234C284606F0F5
:105B2000EBFA284606F0FEFA2A232B825146284635
:105B3000EF8106F047FB07221F49284606F0DCFAF2
:105B4000F31784FB0624C3EBA4042146284606F081
:105B500039FB4A461549284606F0CEFA04EB840183
:105B6000A6EB4101284606F02DFB4A46284610497F
:105B700006F0C2FA4846BDE8F08700BF708AFF1FF2
:105B8000E49DFF1F6A9DFF1F789DFF1FECF400003E
:105B90003B773B98F4F40000DCF40000D09CFF1F3E
:105BA000389DFF1F00F5000067666666F8F9000083
:105BB00070F900000CF5000020F5000038F5000039
:105BC00028F500002DE9F041744C2278002A0546A2
:105BD0000F4614BF4FF001084FF000084ED1704E31
:105BE0003368CB1AB3F5FA6F04D86B78A3B9404683
:105BF000BDE8F0816B4B6C486C49DFF8CCE11A7062
:105C0000012303700988237026208EF8002000F0FD
:105C1000E9FD6B78002BEAD03760FBF7D1FE644AD0
:105C2000644B6549127828781B78097802EB4303A6
:105C3000421E03EB81030E2AD9D801A151F822F0AC
:105C40002D5D0000F95C0000EF5B00002D5D0000A1
:105C5000EF5B0000EF5B0000EF5B0000E15C000029
:105C6000EF5B0000975C0000EF5B0000EF5B000063
:105C7000EF5B0000EF5B0000935C0000AF214F483A
:105C8000474E02F0ADFCFFF701FE002337602370A2
:105C9000ABE704F057FF494C204602F0EDFE2046EA
:105CA000022103F0CBFD23250F2323820522444943
:105CB000E581204606F020FA204606F033FA1E233E
:105CC0000522404923822046E58106F015FA204648
:105CD00006F028FA204602F0DBFF00F0A7FC86E77A
:105CE000394D2B78012B50D9304B2620198800F0E4
:105CF00079FD00232B707AE7002B3FF478AF013B4E
:105D0000324A32F81330002B3FF471AF274C304841
:105D100025492D4A23804FF001080023037081F8A4
:105D2000008082F80080FFF7B1FD60E793B1013B8E
:105D3000264A32F8131019B31C4B254D1A4C224A2F
:105D400019800026012326202E702370137000F086
:105D500049FD15E0154C1E4922880B7004284FF6AA
:105D6000FF7002F1FF310CBF012202460A440E4EC1
:105D7000154D02F07F0201320121228031702B701B
:105D8000FFF784FD4FF0010831E70649064A012379
:105D90000020087013702370A6E700BF708AFF1FF1
:105DA000F49DFF1F6A9DFF1F5E9CFF1FEC9BFF1F62
:105DB000D49BFF1F309CFF1F4C9DFF1F789DFF1F32
:105DC00048F5000050F50000009EFF1FA89CFF1F33
:105DD000159DFF1F2DE9F04FAE4E4FF00109A6F8BB
:105DE0001490A6F81290838813EA09048BB0054634
:105DF0000F46934640F0AB80DFF8C48298F800303D
:105E0000002B7BD1AA79A44CA35CA3B9DFF8B4A280
:105E100079781AF8029039B33B78013B072B00F2EE
:105E2000B280DFE813F0EF005101B0006B01B00069
:105E3000B000B000E7007E78002E00F0C580013B86
:105E4000E868397850F82360F0684B1E0788072B04
:105E500000F2A380DFE813F070015901A1006A018C
:105E6000A100A100A1009B008C4E3368C3EB0B0383
:105E7000B3F5967F72D98A4B187801281ABF012092
:105E800018701970874B18BF0146985CC0EB090069
:105E9000C0B2FFF7E3F80124C6F800B0AB889B0757
:105EA0006DD57B78002B6AD0FBF78AFD7E4B7F4A4D
:105EB0007F481B78127839780078022515FB023369
:105EC0000A2903EB800300F049810C2957D1002BEC
:105ED00055D003F11900774E774A013B002140006D
:105EE00080B226F813100123157088F8003000F0F6
:105EF00079FC724B032220461A702CE0304602F0E7
:105F0000BBFD3046494603F099FCF4813482AB88EE
:105F1000580725D42C68204608F0F2FA214602469C
:105F2000304606F0E9F8304606F0FCF80922012375
:105F30008DE80C0000217F23564803F0F5F800217E
:105F40002846FFF7EDFA002388F800305AE7836807
:105F50001146384698470BB0BDE8F08F0846FAE77F
:105F60002B6804A8984704A808F0CAFA04A90246B6
:105F7000304606F0C1F8304606F0D4F8D6E72046A1
:105F80000BB0BDE8F08F00240AF8029086E70023EA
:105F9000A3543046F3699847F0680780002425220F
:105FA0003C238DE81400412118223A4803F08AF876
:105FB000E968A879FFF78EFB394A384B1470C3F8AB
:105FC00000B00BB0BDE8F08F34490B68C3EB0B0396
:105FD000B3F5967F40F2E080314FC1F800B03C78D5
:105FE000012C00F0AF800123E9683B701046FFF7F9
:105FF00071FBB0E7304BE9791970012388F8003064
:106000000024C1E72B7A013B4B45BCDD09F10104BB
:10601000E4B2A145B7D0234E16F802B0CBEB09008D
:10602000C0B20021FFF71AF82B7A052BD9461BD9ED
:10603000CBEB0402042A40F3A980A4F1040BBBF1CA
:10604000000FC0F2AD80063B5B45A8BF5B465FFA20
:1060500083F9AA791348B15C994205D000F80290FF
:1060600001212846FFF75CFAC9EB0400C0B2012108
:106070000B4EFEF7F3FF00213423019100930B2216
:106080003170044840233F21A14603F01BF801244E
:10609000AA7979E7789DFF1FE89DFF1FE09DFF1F0C
:1060A000FE9DFF1FF89DFF1FD49BFF1F309CFF1F0D
:1060B0004C9DFF1FA89CFF1F6A9DFF1F009EFF1F96
:1060C000708AFF1F649DFF1F0FFA89F3E9685D481E
:1060D00051F823B0036804935B499BF8003004989F
:1060E0000860002B6CD0012B7FF44DAF57499BF813
:1060F000080088F800300870002445E7B9F1000F67
:106100004CD009F1FF34E4B283E7B38A03F004030F
:106110009BB2002B3FF43CAF336A984700283FF412
:106120003BAFAB79F0680022E25436E7738ABB429A
:1061300040D90137BFB230E7338ABB4234D2013F86
:10614000BFB22AE725238DE8480041483E703C2332
:106150001822412102F0B6FF2046FCE6002B3FF456
:106160000EAF3C4A3C4E1188384A03F11900013BFE
:10617000400080B226F81310012388F80030157013
:1061800000F030FB354B20461D70E4E6002A3FF757
:106190005AAF04F1FF3B52E73046DCE64C46F3E6EB
:1061A0004FF000094B4654E7B38AD9077FF5F5AEA7
:1061B000778AF2E6B38ADA077FF5EFAE378AECE644
:1061C00027490393885CC0EB090009F1010EC0B2B6
:1061D000012104F802E0FEF741FF039BDBF808B061
:1061E000019334231A4800930B2240233F2102F0ED
:1061F00069FF012434230B228DE818003F2140233E
:10620000134802F0E1FF2146114803F017FB5846FE
:1062100008F076F9A0EB800000F15F030F22F38114
:106220003282584608F06CF959460246084805F093
:1062300063FF074805F076FFE968A879FFF74AFA97
:10624000AA79A1E61C9EFF1FE09DFF1F6A9DFF1F0C
:10625000789DFF1FEC9BFF1FA89CFF1F009EFF1F48
:10626000F89DFF1F2DE9F047DFF808926D4B99F874
:1062700000601B68DFF800A282B0003601934FF087
:10628000030018BF0126019F9AF8008004F012F95C
:106290000546042004F00EF90446052004F00AF92E
:1062A000800040EA4404062004F004F92C4364B260
:1062B0005D4944EAC0000A7880F00F03DBB29A42DD
:1062C0005A4A3CD01760002259480B7003788DF869
:1062D00000808DF8012053B3564A12684EF66021B3
:1062E000BA1A8A4219D8022B59D0012B5FD0062B3B
:1062F00048D0032B63D0042B69D0052B77D0072B14
:106300007DD0082B00F08380092B68D016B14A4855
:1063100002F0BEFC02B0BDE8F087484A484C0023BA
:106320000121237003701360938089F800103A46AE
:1063300069464448FFF74EFD3043C6B2E6E71268AF
:10634000BA1A1E2A6BD99AF80020934222D0394CEF
:106350003D488AF80030012B276082EA030207607B
:106360009846B1D0042BAFD137480068381AB0F541
:10637000C87FA9D9354C2068381A3228A4D927609B
:106380001A46A1E73A4669463148FFF723FD3043F4
:10639000C6B2BBE7012B4FF00002E3D1E4E73A4677
:1063A00069462C48FFF716FD3043C6B2AEE73A46C1
:1063B00069462948FFF70EFD3043C6B2A6E73A46C4
:1063C00069462648FFF706FD3043C6B29EE73A46C7
:1063D00069462348FFF7FEFC3043C6B296E73A46CB
:1063E00069462048FFF7F6FC3043C6B28EE73A46CE
:1063F00069461D48FFF7EEFC3043C6B286E73A46D1
:1064000069461A48FFF7E6FC3043C6B27EE73A46D3
:1064100069461748FFF7DEFC3043C6B276E7002234
:1064200052E700BF1C9EFF1F019EFF1F6C9DFF1FB8
:106430006A9DFF1FF09DFF1F789DFF1FE89DFF1FB6
:10644000FF9DFF1FACF30000049EFF1F749DFF1F04
:1064500000F4000070F30000D0F20000C4EE000071
:1064600004F30000BCF8000014F3000054F3000033
:106470007C8FFF1F708AFF1F709DFF1F28B110289F
:10648000044BA8BF102018607047024B0120186011
:10649000704700BF089EFF1F38B50F4D2B78013B9A
:1064A00001381B02C4B203F47063200443F4404378
:1064B00043F00C0300F4FE00184305F061F928686E
:1064C000013860F03F00C0B204F08AF92046BDE810
:1064D000384004F085B900BF089EFF1F70B5124D0B
:1064E0002B78013B1B0203F47063064643F43043F0
:1064F0000806320400F0FE4043F00B03034302F4AD
:10650000FE0018430C4605F03BF92868013860F09E
:106510004F00C0B204F064F9304604F061F920463F
:10652000BDE8704004F05CB9089EFF1F70B5124DC5
:106530002B78013B1B0203F47063064643F41043BF
:106540000806320400F0FE4043F00903034302F45E
:10655000FE0018430C4605F013F92868013860F076
:106560006F00C0B204F03CF9304604F039F920461F
:10657000BDE8704004F034B9089EFF1F38B5104DD7
:106580002B78013B1B0203F47063044643F4104371
:10659000000443F0090300F4FE00184305F0F0F88E
:1065A0002868013860F06F00C0B204F019F9204685
:1065B00004F016F90020BDE8384004F011B900BF1E
:1065C000089EFF1F38B50E4D2B78013B1B0203F4CC
:1065D0007063044643F45043000443F00D0300F499
:1065E000FE00184305F0CCF82868013860F02F0051
:1065F000C0B204F0F5F82046BDE8384004F0F0B829
:10660000089EFF1F08B5002005F084F90028FAD184
:1066100008BD00BF08B564210720FFF75FFF7F2199
:106620000B20BDE80840FFF759BF00BF10B500219F
:106630007B20FFF753FF0024E0B2FFF79FFF0134F8
:10664000022003F06DFF802CF6D110BD10B504467A
:106650004FF4406004F074F804F0CCF82CB1102C26
:10666000044BA8BF10241C6010BD024B01241C6009
:1066700010BD00BF089EFF1F10B5044641F0E000AA
:1066800004F0AEF804F07F0004F0AAF8C4F3C610DA
:10669000BDE8104004F0A4B838B5134D2B7804467B
:1066A00041F6FF72A0F50050824203F1FF33A8BF0C
:1066B00002461B0202F5005203F47063100443F417
:1066C000604343F00E0300F4FE005204184302F04E
:1066D000FE42104305F054F8296801392046C9B23A
:1066E000BDE83840FFF7C8BF089EFF1F38B5044615
:1066F0000D46F02004F074F835B1254414F8010B70
:1067000004F06EF8AC42F9D1F720BDE8384004F04F
:1067100067B800BF00B50B4B83B002469988186874
:106720000090032AADF8041002D903B05DF804FB11
:10673000684606218DF80520FFF7D8FF03B05DF805
:1067400004FB00BF30F9000000B50B4B024683B0DC
:10675000186899880090131F4C2BADF8041002D9CB
:1067600003B05DF804FB684606218DF80520FFF7AD
:10677000BDFF03B05DF804FB38F90000030203F429
:10678000FE43C0F3C6101843704700BF037840783B
:10679000DB0103F47E5300F07F001843704700BF15
:1067A00082B002AA114642F8040D002012F8013B03
:1067B00003F07F03914243EA0020F7D102B0704713
:1067C000003210B403884FF0010404FA01F418BF3A
:1067D000012202FA01F123EA04020A43028010BCFA
:1067E000704700BF70B5CEB20C46054603F0F2FA12
:1067F000864203D03146284603F006FB0135284681
:1068000003F0E8FA240A844205D021462846BDE870
:10681000704003F0F9BA70BD38B5054603F0DAFAF6
:106820004FF0000460F30704681C03F0D3FA60F330
:106830000F24A0B238BD00BFF8B504460020FFF712
:10684000EBFF002C00F009814FF4AF610220FFF74D
:10685000C9FF04204FF47A61FFF7C4FF0B2003F057
:1068600029FE002840F0F8844FF496610620FFF7D7
:10687000B9FF4FF4FA610820FFF7B4FF4FF4AF619E
:106880000A20FFF7AFFF40F6FC010C20FFF7AAFF3C
:106890004FF496612220FFF7A5FF4FF416612420E4
:1068A000FFF7A0FF7D212A20FFF79CFF0C210E207F
:1068B000FFF798FF01211020FFF794FF022112201B
:1068C000FFF790FF00211420FFF78CFF0021162016
:1068D000FFF788FF02211820FFF784FF01211A200B
:1068E000FFF780FF02211C20FFF77CFF04211E2000
:1068F000FFF778FF14212020FFF774FF01212620E5
:10690000FFF770FF03212820FFF76CFF04212C20E4
:10691000FFF768FF0F212E20FFF764FF00213020D2
:10692000FFF760FF0C213220FFF75CFF00213420CD
:10693000FFF758FF00213620FFF754FF00213820D1
:10694000FFF750FF00213A20FFF74CFF00213C20C9
:10695000FFF748FF00213E20FFF744FF00214020C1
:10696000FFF740FF00214220FFF73CFF1F2144209A
:10697000FFF738FF13214620FFF734FF0E21482090
:10698000FFF730FF11214A20FFF72CFF0A214C208E
:10699000FFF728FF00214E20FFF724FF062150209B
:1069A000FFF720FF02215220FFF71CFF0C2154208B
:1069B000FFF718FF00215620FFF714FF0021582091
:1069C000FFF710FF01215A20FFF70CFF03215C2085
:1069D000FFF708FF0A215E20FFF704FF0021602077
:1069E000FFF700FF04216220FFF7FCFE0121642075
:1069F000FFF7F8FE00216620FFF7F4FE0B21682068
:106A0000FFF7F0FE7F216A20FFF7ECFE00216C20EB
:106A1000FFF7E8FE00216E20FFF7E4FE0021702062
:106A2000FFF7E0FE00217220FFF7DCFE002174205A
:106A3000FFF7D8FE23210020FFF7D4FE0220FFF746
:106A4000EBFEB0F5805F034616D34FF4AF61022032
:106A5000FFF7C8FE4FF4AF630EE04FF6FF739842A6
:106A60003FF4F2AE232840F003840220FFF7D4FE67
:106A7000B0F5805F0346E8D2D24A04201380FFF7C6
:106A8000CBFEB0F5805F034680F0D282CE4A06206E
:106A90001380FFF7C1FEA0F52F739BB2B3F57A6F99
:106AA000024606D940F628210620FFF79BFE40F655
:106AB0002822C64B08201A80FFF7AEFEA0F52F73E0
:106AC0009BB2B3F57A6F024606D940F6E44108203E
:106AD000FFF788FE40F6E442BD4B0A201A80FFF71C
:106AE0009BFEA0F5FA739BB240F6AC518B42024676
:106AF00006D94FF4AF610A20FFF774FE4FF4AF627E
:106B0000B44B0C201A80FFF787FEA0F5FA739BB2F6
:106B100040F6AC518B42024606D940F6FC010C20EF
:106B2000FFF760FE40F6FC02AB4B0E201A80FFF729
:106B300073FE1828034600F29582A84A102013809D
:106B4000FFF76AFE431E9BB20F2B024604D90121B8
:106B50001020FFF747FE0122A14B12201A80FFF7F9
:106B60005BFE0A28034600F277829E4A14201380B7
:106B7000FFF752FE0128034604D900211420FFF735
:106B800031FE0023984A16201380FFF745FE7F2828
:106B9000034600F25B82954A18201380FFF73CFE03
:106BA0000428034600F24C82914A1A201380FFF712
:106BB00033FE0C28034600F2E5828E4A1C20138027
:106BC000FFF72AFE0428034600F2D6828A4A1E20D6
:106BD0001380FFF721FE0928034600F2C782874A87
:106BE00020201380FFF718FE4628034600F2B882E3
:106BF000834A22201380FFF70FFEA0F5FA739BB2A1
:106C000040F6AC518B42024606D94FF496612220E1
:106C1000FFF7E8FD4FF496627A4B24201A80FFF7C5
:106C2000FBFDA0F5FA739BB240F6AC518B420246D5
:106C300006D94FF416612420FFF7D4FD4FF41662F5
:106C4000714B26201A80FFF7E7FD7F28034600F2EC
:106C500081826E4A28201380FFF7DEFD0628034656
:106C600000F272826A4A2A201380FFF7D5FDA0F154
:106C700032039BB2B3F5967F024604D97D212A20C8
:106C8000FFF7B0FD7D22634B2C201A80FFF7C4FD77
:106C90000C28034600F252825F4A2E201380FFF731
:106CA000BBFD1E28034600F243825C4A302013805D
:106CB000FFF7B2FD0928034600F23482584A322019
:106CC0001380FFF7A9FD1E28034600F22582554ACE
:106CD00034201380FFF7A0FD7F28034600F21682C0
:106CE000514C36202380FFF797FD7F28034600F2A2
:106CF000078238206380FFF78FFD7F28034600F26C
:106D0000F9813A20A380FFF787FD7F28034600F230
:106D1000EB813C20E380FFF77FFD7F28034600F2F4
:106D2000DD813E202381FFF777FD7F28034600F2B7
:106D3000CF8140206381FFF76FFD7F28034600F27B
:106D4000C1814220A381FFF767FD384D2880442090
:106D5000FFF762FD3028034600F2AE81344A462038
:106D60001380FFF759FD3028034600F29F81314C14
:106D700048202380FFF750FD3028034600F2908121
:106D80004A206380FFF748FD3028034600F28281E5
:106D90004C20A380FFF740FD3028034600F27481A9
:106DA0004E20E380FFF738FD0128034604D9002177
:106DB0004E20FFF717FD00231F4A50201380FFF7D6
:106DC0002BFD3BE0329CFF1F549DFF1FE49CFF1FE7
:106DD0002E9CFF1F3A9DFF1FA09CFF1F0A9DFF1FB7
:106DE0007E9CFF1FC89BFF1FBC9CFF1F4E9DFF1F6B
:106DF000689CFF1FCE9CFF1FF89CFF1F7A9CFF1F03
:106E0000529DFF1FFE9CFF1F6A9CFF1FEC9BFF1FF4
:106E10005C9CFF1FA49CFF1FA69CFF1FC09CFF1F24
:106E2000C49BFF1F349CFF1FA89CFF1FFC9BFF1FE0
:106E3000009DFF1F249DFF1F609CFF1F431E9BB2F0
:106E40000B2B024604D906215020FFF7CBFC06226B
:106E5000CF4B52201A80FFF7DFFC0428034600F2D4
:106E60000D81CC4A54201380FFF7D6FC431E9BB201
:106E70001D2B024604D90C215420FFF7B3FC0C2231
:106E8000C54B56201A80FFF7C7FC0128034604D9DA
:106E900000215620FFF7A6FC0023C04A582013808B
:106EA000FFF7BAFC7F28034600F2E280BC4A5A2072
:106EB0001380FFF7B1FC431E9BB2092B024604D995
:106EC00001215A20FFF78EFC0122B64B5C201A806C
:106ED000FFF7A2FC431E9BB2102B024604D90321EC
:106EE0005C20FFF77FFC0322AF4B5E201A80FFF788
:106EF00093FC431E9BB21D2B024604D90A215E203F
:106F0000FFF770FC0A22A94B60201A80FFF784FC6F
:106F10000228034600F28680A54A64201380FFF70A
:106F20007BFC0128034604D901216420FFF75AFCA9
:106F30000123A04A62201380FFF76EFCC31E9BB2A0
:106F4000012B024604D904216220FFF74BFC0422E6
:106F5000994B66201A80FFF75FFC7F28034600F2FA
:106F60007581964A68201380FFF756FC7F280346F8
:106F700000F26681924A6A201380FFF74DFC7F2859
:106F8000034600F257818F4A6C201380FFF744FCC0
:106F90000428034600F248818B4A6E201380FFF7D5
:106FA0003BFC1928034600F23981884A702013807F
:106FB000FFF732FC0228034600F22A81844A72203D
:106FC0001380FFF729FC0628034600F21B81814A43
:106FD00074201380FFF720FC042800F20D812B8819
:106FE000DFF810E27C4F7D4A7D4D7E4E7E4C7F491E
:106FF00003F0010CAEF800C0C3F3400EA7F800E0A8
:10700000C3F380071780C3F3C007794A2F70C3F317
:107010000017C3F34015C3F38013378025800B801E
:107020001080F8BD00216020FFF7DCFB002373E730
:107030004FF47A610420FFF7D5FB4FF47A6325E51E
:1070400002211820FFF7CEFB0223ADE50021162018
:10705000FFF7C8FB00239EE502211220FFF7C2FBC9
:10706000022382E50C210E20FFF7BCFB0C2364E514
:1070700000215820FFF7B6FB002317E7022152201A
:10708000FFF7B0FB0223ECE60A214C20FFF7AAFB36
:107090000A2385E611214A20FFF7A4FB112377E696
:1070A0000E214820FFF79EFB0E2369E613214620A0
:1070B000FFF798FB13235AE61F214420FFF792FBAA
:1070C0001F234BE600214020FFF78CFB002338E60E
:1070D00000213E20FFF786FB00232AE600213C200A
:1070E000FFF780FB00231CE600213A20FFF77AFB24
:1070F00000230EE600213820FFF774FB002300E692
:1071000000213620FFF76EFB0023F2E5002134203A
:10711000FFF768FB0023E3E50C213220FFF762FB59
:107120000C23D4E500213020FFF75CFB0023C5E5EC
:107130000F212E20FFF756FB0F23B6E504212C204C
:10714000FFF750FB0423A7E503212820FFF74AFBA4
:10715000032387E501212620FFF744FB012378E57F
:1071600014212020FFF73EFB142341E504211E20BB
:10717000FFF738FB042332E502211C20FFF732FB26
:10718000022323E501211A20FFF72CFB012314E53C
:107190008C89FF1FC489FF1FB489FF1F509DFF1FEB
:1071A000CA9CFF1FD69BFF1F8E89FF1FBC89FF1F34
:1071B000C69BFF1FA29CFF1F9A9CFF1FB49BFF1F33
:1071C000E69BFF1F109CFF1F989CFF1FE69CFF1F64
:1071D000389DFF1F3E9DFF1FFA9CFF1F589CFF1FFD
:1071E000149DFF1F8C9CFF1FF49CFF1FFC9CFF1F26
:1071F000949CFF1F469DFF1F74200021FFF7F2FAA9
:107200000020ECE600217220FFF7ECFA0023DEE616
:1072100000217020FFF7E6FA0023CFE600216E2060
:10722000FFF7E0FA0023C0E600216C20FFF7DAFA4E
:107230000023B1E67F216A20FFF7D4FA7F23A2E67C
:107240000B216820FFF7CEFA0B2393E6002166207E
:10725000FFF7C8FA002384E640F628210620FFF74E
:10726000C1FA40F6E4410820FFF7BCFAFFF706BB7D
:1072700017287FF6E9AA19287FF658AB1B287FF656
:1072800075AB1C283FF48AAB1E287FF68FAB1F28F6
:107290003FF494AB20283FF4ADAB21283FF4B6ABCC
:1072A00022287FF4C7ABFFF7B9BB00BFF8B5872032
:1072B00006F09AFB204B214A054603CB1368C5F81C
:1072C00003001A0C7620C5F807102B80AA70FFF770
:1072D00055FA2E46002426F80B0FA0B2FFF79CFAB1
:1072E000FFF74CFA0234762C26F8020FF5D16C1E0B
:1072F00005F182064FF0FF3014F8013F082758408F
:107300000F4B40F300017A1E0B4012F0FF0783EA97
:107310005000F5D1B442EFD1C043FFF741FA3A46ED
:10732000C5F883008721284604F078FA2846BDE88E
:10733000F84006F061BB00BF44F9000040F90000CE
:107340002083B8EDF0B50E4B0E4C054693E80700D0
:1073500085B024682E88AD7801AB83E80700270C40
:10736000184600220B21ADF804408DF80670ADF8E8
:107370000C608DF80E5004F051FA05B0F0BD00BF5E
:1073800050F9000040F90000F0B5124B124D1E6894
:10739000124F0FCD87B06C460FC495E8030044F838
:1073A000040B38683B79CDF80D00320C2320218086
:1073B0008DF802208DF81130ADF80060FFF7DEF98E
:1073C0000022ADF80B001221684604F027FA07B03E
:1073D000F0BD00BF40F900005CF90000DCF40000E3
:1073E000002004F097BA00BF02F0ACBC70B5104C9E
:1073F00082B0002540230646294620460093019589
:107400008023202201F05EFE0123202230462282CA
:10741000A3826382E58107F073F831460246204675
:1074200004F06AFE204602B0BDE8704001F030BCB6
:10743000789DFF1FF0B5862983B075D90546441E97
:1074400000F182064FF0FF3014F8012F082750405A
:10745000404A40F300017B1E0A4013F0FF0782EA16
:107460005000F5D1B442EFD1C043FFF799F901467E
:10747000D5F883000190019A914202D0B2F17F2F9A
:107480000BD105F10B00FFF781F976280BD03248BC
:10749000FFF7ACFF002003B0F0BD3048FFF7A6FFB8
:1074A000384603B0F0BD05F10D00FFF76FF9232852
:1074B00040D1002440F6AC5613E004281AD0062828
:1074C00021D008281FD00A2828D00C2822D1A1F5C5
:1074D000FA7292B2B24201D8FFF784F90234762CE4
:1074E0000ED004F10D002844FFF750F9022C01469C
:1074F000A0B2E2D1B1F5805FEED30234762CF0D1A8
:10750000012003B0F0BDA1F52F7292B2B2F57A6FEF
:10751000E4D8E1E7222801D0242811D1A1F5FA729C
:1075200092B2B242DAD8D7E70D48FFF75FFF0020EA
:1075300003B0F0BD0B48FFF759FF002003B0F0BDCA
:107540002A28C9D1A1F1320292B2B2F5967FC5D8EC
:10755000C2E700BF2083B8EDA0F900008CF900005D
:1075600074F90000B4F9000003290CD970B5461C69
:1075700082B005460C46304603222A4907F02EF811
:1075800010B102B070BD70470B2C05D905222649F9
:10759000281D07F023F840B12448FFF727FF2448AF
:1075A00002B0BDE87040FFF7CDBE05F1090103222E
:1075B00001A807F063F801A803221E4907F00EF89E
:1075C000D8B103221C4901A807F008F808B301A8A4
:1075D00003221A4907F002F8B0B91948FFF706FF6D
:1075E000A11E89B23046FFF725FF0028C9D01548F3
:1075F00002B0BDE87040FFF7F9BE1348FFF7F6FE92
:10760000FFF754FE1148F3E71148FFF7EFFE11486A
:10761000C6E71148FFF7EAFE02B0BDE87040FFF789
:10762000B3BE00BF40F90000ECF40000CCF900004C
:10763000E0F90000E4F900000CFA000024FA000070
:1076400028FA00003CFA0000E8F90000FCF900000C
:1076500050FA000064FA000010FA00002DE9F0432F
:10766000174D2B6883B081460F469046F3B1154EF7
:1076700034880A1992B218461146328006F032FD5B
:1076800028603A464946204402F0E0F8B8F1000F7D
:1076900009D031882868FFF767FF286806F0ACF941
:1076A00000232B60338003B0BDE8F083054E0193C7
:1076B0000846318006F098F9019B28601C46E0E7F7
:1076C000109EFF1F0C9EFF1F10B51D4C4FF4FA704B
:1076D000FCF79EFB204601F0CFF90023194601225A
:1076E0002046E3812382A282628202F0A7F80B2265
:1076F0001449204604F000FD204604F013FD0F223B
:107700001149204604F0F8FC204604F00BFD0F4917
:107710000722204604F0F0FC204604F003FD20463A
:1077200001F0B6FA0A4B0B4A1A604FF4FA70FCF7F4
:107730006FFBFFF729FE0848BDE81040FFF756BE73
:10774000789DFF1F68FA000074FA000084FA0000B8
:10775000A89FFF1F5D7600008CFA00000020704794
:1077600090F8392090F83800101A704790F83830A7
:1077700090F839209A4205D95A1C034480F83820E1
:10778000187E70474FF0FF30704700BF90F83830D8
:1077900090F839209A4286BF1B18187E4FF0FF30B0
:1077A000704700BF704700BF38B50546B0F85E00AF
:1077B00090B195F85D301446C3F1210294420CD883
:1077C00005F13B001844224602F040F895F85D3080
:1077D000234485F85D30204638BD012014462871C9
:1077E000EEE700BFB0F85E306BB190F85D30202B53
:1077F00007D8C218013380F85D30012082F83B10B1
:107800007047012303710020704700BF00234269C5
:1078100080F8383080F8393080F85C3080F85D309E
:1078200080F85E3080F85F3006CA30B40D680469B5
:1078300043662A4383660A60A370426990F8613008
:107840001649146813441D7A5B7B01EBC5051B02C6
:107850006D6803F4E06343F064032B6090F86230DA
:1078600013449D7CDB7D01EBC5011B02496803F4D9
:10787000E06343F064030B6021685368194205D04C
:10788000036927225A70036904229A71036920222E
:107890005A71036980229A7030BC7047B0050100AC
:1078A00043690CCB12681A420CD0094B99420AD991
:1078B000084B9942036994BF1A220D225A7003693A
:1078C00004229A717047036927225A70F7E700BFB4
:1078D0007F1A06003F420F0010B50269D378DBB271
:1078E000D90604463DD510215806D17038D503F08D
:1078F000040303F0FF02002B51D03D49626E0023C8
:107900000B7084F85D30002A5BD0904794F85D30AE
:10791000002B56D02369D0229A70236994F83B201B
:107920001A712369012284F85C200222DA7010BDEA
:10793000304B84F860009C424AD02F4B9C4252D07E
:1079400094F8391013791F29DBB207D8284800783A
:1079500020B16018013184F8391003760223D37006
:1079600010BD5906C3D4917801F0100101F0FF0059
:107970000029DDD013F001031ED194F85C1094F8B7
:107980005D00884281BF4B1C091984F85C3091F876
:107990003B3013712369D0229A702269DEE7236994
:1079A00084F83920C0229A702369114A197901217B
:1079B00011700222DA7010BDC0239370226913790E
:1079C000CCE70122002384F85D2084F83B30A1E756
:1079D000626994F86130094913440322187A02F06D
:1079E00001FB2269ACE7626994F861300449F3E76E
:1079F000149EFF1FD48FFF1F4090FF1F617A00006D
:107A00006D7A00000369DB7803F0200373B190F80E
:107A100060300133DBB2012B80F860301AD9426943
:107A200090F861301344187A02F058BB70B542697F
:107A300003F0FF0590F8613013440446187A02F011
:107A40004DFBA36E5BB184F8385094F83900BDE863
:107A50007040184790F85F30002BE0D0704770BD41
:107A60000148FFF7CFBF00BFD48FFF1F0148FFF7CA
:107A7000C9BF00BF4090FF1F2DE9F047374FDFF827
:107A8000E0903B68026982B006460093DDF8008012
:107A90000021A025D3789B065BD53B680193019B11
:107AA000C8EB03030F2BF5D949B1102BF2D00020FE
:107AB0009070336980229A7002B0BDE8F0877269D5
:107AC00096F8613013440521187A02F001FD7269BD
:107AD00096F861301344012193F812A0504602F049
:107AE000F7FC09240021504602F0DEFC2B46013B46
:107AF000FDD10121504602F0D7FC2B46013BFDD1C0
:107B0000013CEFD1706996F8611001444FF4A07206
:107B10000C7A4B7B09EBC4011B02496803F4E06358
:107B200043F064030B6096F862300344997CDB7D7C
:107B300009EBC1011B02496803F4E06343F06403ED
:107B40000B60013AFDD13269D3789B064FF00101F9
:107B5000A3D4012002B0BDE8F08700BF1C9EFF1F28
:107B6000B0050100F0B503691222DA70026993785A
:107B700003F0200385B004460D46002B5ED0B423ED
:107B800093703C4922690B680093009E05E00B68E6
:107B90000193019B9B1B042B42D8D37803F0200355
:107BA00003F0FF00002BF2D094F85D30002B31D0B1
:107BB0004FF0000E4FF0020C04EB0E0393F83B3035
:107BC00013710B680393039F206907E09B060DD593
:107BD0000B680293029BDB1B052B28D8C378DBB212
:107BE00003F0020202F0FF06002AEFD080F803C083
:107BF0002669F378DBB2DF0632462DD49F062BD5FB
:107C0000DB0731D40EF1010E94F85D305FFA8EFE81
:107C10007345D1D800201DBB002384F85E3004E0FA
:107C20009070236980229A70042005B0F0BD8670A0
:107C30002369802204209A7005B0F0BD03F0FF068E
:107C4000FFF71AFF10B9042005B0F0BD236984F8CE
:107C50005F60B0229A7094E78023B3700420DAE763
:107C600026698023B370D7E7BEF1000F0CBF022056
:107C70000320F6E71C9EFF1F2DE9F0410669002551
:107C8000122780F8385080F83950F770D0F810C0BB
:107C90009CF802E00EF0200E88B004468846154697
:107CA0001E46BEF1000F49D0B4238CF80230784B49
:107CB00021691A680092DDF800E006E01A68019276
:107CC0000198CEEB0000042830D8C87800F02000DE
:107CD00000F0FF070028F1D04FEA480242F001020D
:107CE000D2B20A711A680292DDF808E0206906E053
:107CF0001A6803920399CEEB010105292AD8C178AD
:107D000001F0020101F0FF070029F1D04FF0020C51
:107D100080F803C02269D17811F0110722D12DBB60
:107D2000002E0CBFA0238023937003E08F70236983
:107D300080229A70384608B0BDE8F0810EF0FF0747
:107D4000FFF79AFE0028F5D0236984F85F70B0220F
:107D50009A70ACE787702369802238469A7008B021
:107D6000BDE8F081802393700027E3E7012D75D0F3
:107D7000A021917021690A79BE4667464FF0A80C90
:107D80001A680492049805E01A680592059A121A76
:107D9000052A4AD8CA7802F0020202F0FF08002A37
:107DA000F2D0CF702169CA78D2B212F0100F084613
:107DB0005AD1920658D5013DEDB2012D49D0BEF100
:107DC0001F0F3BD90A79012DDAD11A680692069D58
:107DD00005E01A680792079A521B052A46D8C2780E
:107DE00002F0020202F0FF01002AF2D00223C37067
:107DF0002269D378DBB2D9063AD49B0634D5B023B6
:107E0000BEF11F0F93703FD8226904EB0E03127965
:107E10001A760EF1010E5FFA8EFE16B123698022EA
:107E20009A7084F839E0774684E781F80280236904
:107E300080229A70774684F839E07BE704EB0E02E3
:107E400091F8048082F818800EF1010E5FFA8EFE20
:107E5000B9E781F802C021690846B0E7A82191700E
:107E60002069BE460279B0E7774663E78170DEE7B6
:107E70001021A023D170013BFDD12269937803F03A
:107E8000F7037746937055E723691B79C5E700BF71
:107E90001C9EFF1F0148FFF71FBD00BFD48FFF1FAF
:107EA0000148FFF719BD00BF4090FF1F704700BF9A
:107EB00038B5144C037801225B000546204684F84F
:107EC0003B3084F85E2084F85D20FFF78BFC204671
:107ED0000021FFF747FE0B4C2978012320461A4664
:107EE000FFF7CAFE0128F6D194F8383094F839200B
:107EF0009A4205D9E218013384F83830107E38BD33
:107F0000FF2038BDD48FFF1F38B51B4C03780122EA
:107F10005B000546204684F83B3084F85E2084F8F8
:107F20005D20FFF75FFC20460021FFF71BFE124C8F
:107F30002978204601230222FFF79EFE0228F6D16F
:107F400094F8382094F839108A420FD2531CDBB2CF
:107F5000A018994284F83830007E0AD923440232AE
:107F60001B7E84F8382040EA032038BD4FF6FF70AE
:107F700038BD40F47F4038BDD48FFF1F0C2901D994
:107F8000002070470231490001F0FE01FFF7BCBF3D
:107F900070B50C4C0378164601255B00204684F82A
:107FA0003B3084F85E5084F85D50FFF71BFC31468F
:107FB0002046FFF717FC29462046BDE87040FFF732
:107FC000D1BD00BFD48FFF1FF8B505460F4616463A
:107FD000412421463A462846FFF7DAFF611C023465
:107FE000C9B232462846E4B2FFF7D2FF592CF0D18D
:107FF000F8BD00BF38B504460D463548FFF706FC0E
:108000006322802120462570FFF7C2FF012002F085
:1080100087FA204600225E21FFF7BAFF20465D2145
:10802000FFF746FF242801D0002038BD2046062255
:108030000C21FFF7C9FF204601222B21FFF7A8FFE3
:10804000204601222C21FFF7A3FF20460E222D21DE
:10805000FFF79EFF204600222E21FFF799FF2046C2
:1080600001222F21FFF794FF204605223021FFF740
:108070008FFF204601223121FFF78AFF2046002290
:108080003221FFF785FF204600223321FFF780FFD2
:10809000204600223421FFF77BFF204600223521B5
:1080A000FFF776FF204600225B21FFF771FF204695
:1080B00010225C21FFF76CFF204620225D21FFF794
:1080C00067FF20468F225E21FFF762FF012038BD47
:1080D000D48FFF1F10B4047F4160022CC26002D015
:1080E00010BC03F087BE836810BC184790E80C00F2
:1080F000F0B41C6859682568164F174E2943216053
:10810000164D17491760D66015611160417A154AFE
:108110005C180A3194F8244053F8215002EBC40152
:1081200049680D60017A5C1803EB8101247ECD69FA
:1081300002EBC40149680D60817A581803EB810392
:1081400090F83000596B02EBC002F0BC5368196024
:10815000704700BF01401F00011000380110007877
:1081600000001F80B0050100704700BFF0B50C1E75
:10817000BDF8146034DBB0F906701919B942C4BFF8
:108180003B1B1BB2002BA6461CDD002A1146B8BFC4
:10819000D11D02F00705CC10826A012007FB04E123
:1081A000A840012E0A44C0B21ED00CD3022E09D121
:1081B000013B12FA83F3013A12F8011F41409A423F
:1081C0001170F9D1F0BDC043013B12FA83F3C0B284
:1081D000013A12F8011F014093421170F9D1F0BD2C
:1081E00023441BB20024C6E7013B12FA83F3013A91
:1081F00012F8011F01439A421170F9D1F0BD00BF7E
:1082000000291EDB30B4B0F90A408C4218DD002A88
:1082100016DBB0F90C40944212DD047E022C54D0DF
:10822000032C4CD0012C06D15140C4884A40514007
:10823000013C611A09B2012B2DD017D3022B01D0BA
:1082400030BC7047002AB0F90630856A1446B8BFC2
:10825000D41D44F3CF0404FB031102F007026B5C4E
:10826000012000FA02F25A406A54E9E7002AB0F904
:108270000630856A1446B8BFD41D44F3CF0404FB0E
:10828000031102F007026B5C012000FA02F223EAFC
:1082900002026A54D4E7002AB0F90630856A14460F
:1082A000B8BFD41D44F3CF0404FB031102F007024E
:1082B0006B5C012000FA02F21A436A54C0E7048999
:1082C000013C641A114622B2B5E7C5880489013D14
:1082D000013C691AA21A09B212B2ACE72DE9F041C9
:1082E000079E9DF91880089D04461F4600F0BCFFBC
:1082F0000D4B0E480E4984F83380FF22002F08BF33
:108300001F4684F82F20002384F8302084F8312081
:1083100084F8322020606665A56567622166236265
:10832000A3622046BDE8F081D48FFF1F18FB000038
:108330000110013810B50446806A034B236008B170
:1083400005F05AFB204610BD18FB0000F8B5436A43
:10835000DBB190F82C200125AA4083F83B2083F85C
:108360005E5083F85D500446406A03680E461B6801
:1083700000219847606A036831461B689847294680
:10838000606ABDE8F840FFF7EDBBC26BC56C1368CF
:10839000046A23EA050313604CB122684FF00043DE
:1083A000D3625163D36A002BFCDA936BF8BD836B05
:1083B000466B0825802410E03768426C3A433260EF
:1083C0001F68826C3A431A601A68876C013D22EA82
:1083D00007024FEA54041A6007D02142ECD13268F8
:1083E000476C22EA07023260EAE7F8BD70B504463E
:1083F000406A0D4600282BD0616DFFF751FA002D21
:1084000020460CBFA621A721FFF7A0FF606A20B17C
:10841000A16DBDE87040FFF743BA216C226D08687A
:10842000236A02430A6093B1DA7A82B1D00703D596
:10843000224A99691160DA7A910703D5204AD969ED
:108440001160DA7A520702D51E4A1B6A136070BDAA
:10845000236A002B2BD0D97A226EE1B172B6D97A79
:10846000CE0706D51848D968066831409961016081
:10847000D97A880706D51548196906683140D96147
:108480000160D97A4E0705D511485969066831400F
:108490001962016062B61B68D968914207D00D4825
:1084A00018600D49DA6042F0804018611960226C52
:1084B000216D136823EA01031360A0E700E100E0E7
:1084C00004E100E008E100E080E100E084E100E098
:1084D00088E100E001403F0000003F80436A2DE951
:1084E000F04105460E469046002B3ED090F82C10E9
:1084F0000124A14083F83B1083F85E4083F85D407F
:10850000406A036800211B6808F1FF379847FFB2F3
:10851000B8F1000F23D03744A046013E686A16F830
:10852000011F03681B6898470134B742E4B216D0B4
:10853000202CF3D10121686AFFF714FB95F82C2059
:108540006B6A520083F83B2083F85E8083F85D807D
:10855000686A036800211B6898470124DEE7686A9F
:108560000121BDE8F041FFF7FDBAC26BC16C136891
:1085700023EA010306EB080413604FF00048A6420B
:108580000ED02B6A16F801EB63B11A68C2F82C8082
:10859000C2F834E0D36A002BFCDAA642936BF0D128
:1085A000BDE8F081AB6BD5F834C008208021DCF841
:1085B00000206F6C1EEA010F14BF3A43BA43CCF897
:1085C00000201A68AF6C3A431A601A68AF6C013821
:1085D00022EA07024FEA51011A60E8D1CFE700BF53
:1085E00070B50446406A0D46002828D0616DFFF73B
:1085F00057F920462946FFF7A9FE606A20B1A16D10
:10860000BDE87040FFF74CB9216C226D0868236A01
:1086100002430A6093B1DA7A82B1D00703D5234AC4
:1086200099691160DA7A910703D5214AD9691160F5
:10863000DA7A520702D51F4A1B6A136070BD236A9B
:10864000002B2BD0D97A226EE1B172B6D97ACE073F
:1086500006D51948D9680668314099610160D97A10
:10866000880706D51548196906683140D961016047
:10867000D97A4E0705D51248596906683140196202
:10868000016062B61B68D968914207D00D48186036
:108690000D49DA6042F0804018611960226C216D4A
:1086A000136823EA01031360A3E700BF00E100E0C1
:1086B00004E100E008E100E080E100E084E100E0A6
:1086C00088E100E001403F0000003F802DE9F041DB
:1086D000044686B0806A9DF830801E460F461546D7
:1086E000B4F90830002800F04B81DA1D48BF03F1CF
:1086F0000E02B4F90630D21003FB02F2002105F09D
:108700009FFCB4F90820202A00F3A780B4F90610D2
:10871000A74B0120203A733902EBD27201EBD171E1
:108720004FF0200E029073208DE8014042F34F027B
:1087300041F34F01204600F04DFE606A84F82D7031
:10874000002800F05181002D40F09F80B4F90830DE
:10875000202B14BF3D253C2584F82C50B8F1000F88
:1087600040F09A8006B394F93300002818DBC0B2B9
:10877000012101F0ADFE012194F8330001F094FED7
:10878000012001F0CDFE002194F8330001F08CFEB1
:108790000A2001F0C5FE012194F8330001F084FEA7
:1087A000606A002800F09880616DFFF779F8042274
:1087B00080492046FFF792FE217A0139C9B220464E
:1087C000FFF7C4FD7C4904222046FFF787FE94F999
:1087D0002D30012B14BF142110212046FFF7B6FDC8
:1087E000042276492046FFF779FEB4F906308F223D
:1087F000802B84F85C2000F0A580602B00F0B18015
:108800000225DA212046FFF7A1FD29462046FFF781
:108810009DFD81212046FFF799FD94F85C102046CC
:10882000FFF794FDD9212046FFF790FD94F92D30F4
:10883000012B14BFF12122212046FFF787FD20469E
:1088400006225F49FFF74AFE606A58B3A16DFFF741
:1088500027F8012006B0BDE8F081B4F90610594BA5
:108860000120403A52394FF0400E029002EBD27292
:10887000522001EBD1718DE8014042F34F0241F3E8
:108880004F01204600F0A6FD57E76DB284F82C504A
:10889000B8F1000F3FF466AFFEF7B8FF002E3FF4CB
:1088A0007FAF60E7216C226D0868236A02430A608B
:1088B00073B1DA7A62B1D00703D5434A996911607E
:1088C000DA7A91076FD4520702D5404A1B6A1360C7
:1088D000012006B0BDE8F081236A002B2BD0D97AA5
:1088E000226EE1B172B6D97ACF0706D53848D96879
:1088F0000568294099610160D97A8E0706D5354807
:10890000196905682940D9610160D97A4D0705D5F3
:1089100031485969056829401962016062B61B68CF
:10892000D968914207D02D4818602D49DA6042F08D
:10893000804018611960226C216D136823EA0103DD
:10894000136034E7B4F90830402B7FF459AF94F941
:108950002D30012B14BFCF239F2384F85C301225C8
:108960004FE7B4F90830102B7FF44AAF94F92D305B
:10897000012B14BFAF23102384F85C30022540E79D
:10898000DA1D48BF03F10E02B4F90630D21003FB22
:1089900002F21046059205F027F8A06200283FF485
:1089A00059AF059AAAE60F4AD9691160DA7A8AE7BF
:1089B00068FB000048FD00004CFD000050FD000079
:1089C00054FD00005CFD000000E100E008E100E073
:1089D00080E100E084E100E088E100E001403F0048
:1089E00000003F8004E100E0012194F83100214FB4
:1089F00001F06EFD94F83200012101F069FD94F957
:108A0000312094F9323057F83220E26357F833308E
:108A1000206A23640125E56425651A682A431A60E3
:108A200048B1B8F1000F3FF439AFFFF75FFB002EFC
:108A30003FF4B6AE97E6294694F82F0001F048FDC2
:108A4000294694F8300001F043FD94F92F2094F961
:108A5000303057F83220626357F833306564A564CC
:108A60001A68A36322F001021A60002E3FF498AE48
:108A700079E600BFB0050100B0F90820D31D48BF5A
:108A800002F10E03B0F90620806ADB1002FB03F24C
:108A9000002105F0D5BA00BFF0B50029BDF814508B
:108AA0002EDBB0F90660B1422ADA002A59DBB0F9B0
:108AB000087014461C44BC42C4BFBB1A1BB2002B36
:108AC0001EDDD2B2D408D0F828E016FB041112F053
:108AD0000702DBB20EEB010421D0C2F10807FAB2A3
:108AE000374F9342BF5C0CD2C3EB020CFF2646FA11
:108AF0000CF6012D07EA06073FD005D3022D36D02C
:108B0000F0BD012D39D030D21EF8016026EA0707EA
:108B10000EF801709342F3D3B0F906100C449A1A80
:108B2000D2B2072A10D9022D36D0002D14BFFF264D
:108B3000002613462670083BB0F90610DBB2072B5F
:108B40000C44F7D802F00702002AD9D01D4B012DA2
:108B50009B5C1DD017D3022DD2D1227853402370B5
:108B6000F0BD13441BB20022A1E7022D25D11EF84F
:108B7000016077400EF80170CCE71EF801603743C2
:108B80000EF80170C6E7227822EA03032370F0BDD5
:108B9000227813432370F0BD11462378DB43237002
:108BA0000839B0F90630C9B207291C44F5D812F0CB
:108BB0000702A5D0034B9B5CCFE73444AFE700BF6F
:108BC00008FB0000F8FA000070B4047EBDF80C50F9
:108BD000022C18D0032C1FD0012C0BD0002A03DB51
:108BE000B0F90840944201DC70BC7047039570BC3A
:108BF000FFF7BCBAC4880395013CA41A0A4621B207
:108C000070BCFFF749BF0689C488013E641AB21AD6
:108C1000E41A12B221B2E1E704890395E41A641A56
:108C2000114622B270BCFFF737BF00BF70B4057E9B
:108C3000BDF80C60022D1AD0032D12D0012D03D0E7
:108C4000039670BCFFF728BFC488E41AA41A0A462A
:108C500021B2002A03DBB0F90840944213DC70BC57
:108C600070470489013C641A114622B2F1E7C488B6
:108C700005890396013CAD1AED1A621A11B22AB2A7
:108C800070BCFFF709BF039670BCFFF76FBA00BF57
:108C90002DE9F8430446406A002863D0616DFEF771
:108CA000FFFD052274492046FFF718FCA179013920
:108CB000C9B22046FFF74AFBB4F90820E588A66A46
:108CC000D31D48BF02F10E03DB10626A15FB03F5EA
:108CD0001FFA85F8002A7BD094F82C300125AB4090
:108CE00082F83B3082F85E5082F85D50606A03681B
:108CF00040211B6808F1FF379847BFB2B8F1000F59
:108D000023D03744A846013E606A16F8011F036865
:108D10001B6898470135B742EDB216D0202DF3D12C
:108D20000121606AFEF71EFF94F82C20636A52004E
:108D300083F83B2083F85E8083F85D80606A036877
:108D400040211B6898470125DEE70121606AFEF794
:108D500009FF606A002800F08D80A16DBDE8F8432E
:108D6000FEF79EBD236A002B2BD0D97A226EE1B18B
:108D700072B6D97ACE0706D54048D9680568294029
:108D800099610160D97A8D0706D53D481969056852
:108D90002940D9610160D97A480705D53948596910
:108DA000056829401962016062B61B68D968914262
:108DB00007D0354818603549DA6042F080401861C4
:108DC0001960226C216D136823EA0103136068E7C0
:108DD000E26BE36C1168276A0B4306EB080913602A
:108DE0004FF0004E4E450DD016F801CB2FB33A6828
:108DF000C2F82CE0C2F834C0D36A002BFCDA4E452E
:108E0000936BF1D1226C236D11680B43136097B102
:108E1000FB7A83B1D90703D51D4BBA691A60FB7A77
:108E20009A0703D51B4BFA691A60FB7A5B0702D5D8
:108E3000194B3A6A1A60BDE8F883A36BD4F8348002
:108E400008208021D8F80020656C1CEA010F14BFAF
:108E50002A43AA43C8F800201A68A56C2A431A605E
:108E60001A68A56C013822EA05024FEA51011A601E
:108E7000E8D1B7E7276AC5E700FB000080E100E022
:108E800084E100E088E100E001403F0000003F8015
:108E900000E100E004E100E008E100E02DE9F04F2E
:108EA00085B09946BDF93870BDF83CA0BB1AC1EB3E
:108EB000090B002BB8BF5B42BBF1000FB8BFCBF171
:108EC000000B5B450D4616460093804648DC4D4539
:108ED0003A4633464CDC194613460A46C5EB0901AF
:108EE0009B1A89B2002B0CB2B8BF5B4204EBD4745E
:108EF000BE42ACBF4FF0FF3201224D4503910292BA
:108F00004FEA640429DC9BB201930DE0D8F80070AD
:108F1000BF69B847019BE41AA3B21CB20135002C0B
:108F20002DB211DBA94518DB009B5B452A46534651
:108F300031464046EADCD8F8002053469769294676
:108F400032464046B847E5E7029A1644039AA945D7
:108F500002EB030436B224B2E6DA05B0BDE8F08FC6
:108F60004A462B46B94635464D4517461E46B2DDA4
:108F7000304629463E464D4607468946AEE700BF85
:108F800010B404682469A44610BC604730B4046877
:108F9000BDF808500295A46BA44630BC604700BFE2
:108FA00030B40468BDF808500295E46BA44630BCA8
:108FB000604700BF70B40468BDF90C60BDF8105084
:108FC00003960495246CA44670BC6047704700BFAC
:108FD00010B582B0B0F90C20019101680092002216
:108FE0000C6CB0F90A301146A04702B010BD00BFAA
:108FF000704700BF01F003010129017606D0032963
:1090000004D0C28803894281838170470289C38862
:1090100042818381704700BF2DE9F0410568134EFE
:109020006F6986B0B7420446BDF8308010D1013B6D
:1090300013441BB20093CDF804800B46AD6A204662
:10904000A8472368DB6AB3420AD106B0BDE8F081C5
:10905000059304920391B84703A925680EC9E6E772
:10906000204606B0BDE8F041184700BFCD8F000094
:109070002DE9F0410568124E6F6986B0B74204468B
:10908000BDF830800FD1013BCDF804800B44009235
:109090001BB2AD6A2046A8472368DB6AB3420AD1F7
:1090A00006B0BDE8F081059304920391B84703A987
:1090B00025680EC9E7E7204606B0BDE8F04118472D
:1090C000CD8F00002DE9F04F0568DFF858B06F69CB
:1090D00085B05F450646BDF93890BDF83CA00C460A
:1090E000904615D11F19BC420CDACDF800A02146DC
:1090F00001342D6A4B464246304624B2A847BC4252
:109100003568F2DBEB6A5B4507D105B0BDE8F08F4F
:109110000393B8473568039BE4E7304605B0BDE8E4
:10912000F04F1847CD8F00002DE9F04387B09942EA
:109130000546BDF93840BDF83C6025D0A24212D0AA
:109140000768DFF88080D7F81490C14532D18DE8E8
:1091500050002846BC6AA0472B68DB6A434524D1EF
:1091600007B0BDE8F083994202DD08461946034680
:1091700028680E96C46B01335B1A1BB22846A446BE
:1091800007B0BDE8F0436047A24202DD1346224625
:109190001C4628680E96631C846B9B1A1BB22846DB
:1091A000A44607B0BDE8F0436047284607B0BDE8D5
:1091B000F0431847059304920391C84703A92F6809
:1091C0000EC9C4E7CD8F00002DE9F04FD0F800E0C4
:1091D000DFF89090DEF814B083B0CB450446BDF9BB
:1091E0003080BDF834A00D4617461E4631D1CDF86B
:1091F00000A0DEF824B0294633463A462046D84738
:109200002368CDF800A008F1FF323A44D3F824B027
:10921000294612B233462046D8472368CDF800A02D
:109220002946D3F820B03A4643462046D84720681E
:10923000CDF800A0711E29444346056A09B23A469A
:109240002046A8472368DB6A4B4506D103B0BDE83A
:10925000F08FD847D4F800E0C9E7204603B0BDE856
:10926000F04F1847CD8F0000F0B4002401254FF6D1
:10927000FF76094F076004710476C4810482847606
:10928000C461C5758575457686824682C180028136
:1092900041818281F0BC7047240001002DE9F04F2C
:1092A00085B00668BDF84450BDF93880CDF800801F
:1092B00004460195D6F848B00392BDF93C60BDF96B
:1092C000407089469A46D8472368019500974246E0
:1092D0005146D3F8488020463346C0472068039B58
:1092E0000E930F95856C4B463A4631462046AC4668
:1092F00005B0BDE8F04F60472DE9F04F87B0174645
:10930000BDF9404000912546E91D059344BF2B4619
:1093100003F10E010268BDF8486053690294C91058
:1093200003912B49BDF9444001968B42824645D1B9
:10933000002C3CDD029B3C445E1EB6B24FF000099F
:1093400023B2049301364D46029B002B28DD059B7A
:10935000002403EB090806E0EDB22B0604F101043A
:1093600011D4A6421CD0A1B211F0070F23B24FEACC
:109370004505F1D1002BB8BF0733DB10013418F8D5
:1093800003502B06EDD5009BD2F818B019443A468D
:1093900009B2019B5046D847A642DAF80020E2D134
:1093A000039B01379944049B3FB2BB42CCD1D36AA3
:1093B000074A934206D107B0BDE8F08F9847DAF824
:1093C0000020B5E7504607B0BDE8F04F184700BF92
:1093D000CD8F000070B4BDF90C60BDF91050BDF820
:1093E000144003960495059470BCFFF785BF00BF39
:1093F0002DE9F04F91B083460591C169BDF8680031
:1094000006909DF87400BDF86C709DF870A00390F4
:1094100002929946002900F0CC800B7A48680A68CD
:10942000C3EB0903DBB2154600EBC30230F833602F
:10943000D3780993BAF1010F92F9053092F80280BE
:109440000E9392F9064079D9BDF93830089323B2CA
:109450000B93A94BDBF800200F93194653698B42FD
:1094600040F0A280099B002B53D0BDF808300C932C
:109470000021234407910D930F460C46A946B8F1ED
:10948000000F3FD0BDF81C100B9BBDF80C000297DD
:10949000CB1813FB00F30C9803440D981BB2014446
:1094A00004930BB20A93002505E00135EBB264008A
:1094B0009845E4B223D9029B2B44590703D1731C6E
:1094C00019F806409EB22306EFD5089BE918059BC4
:1094D00011FB0AF1BAF1010F194402D1039B012BD0
:1094E0001ED0069B0193039B0093D369049A1F46E9
:1094F00009B253465846B847DBF80020D5E7029F2B
:109500004744FFB2079B099901330793DBB29942A5
:10951000B5D8D36A0F9A934241D111B0BDE8F08F0C
:109520000E9B0599591893690A9A29441F4609B256
:10953000069B5846B847DBF80020B6E7039B012B93
:1095400082D800230B93089383E70799099A013186
:10955000013A49B212F0FF020791099260D1069ACE
:109560004A454F4617D0BAF1010F03D1039A012A99
:1095700000F0B5800A9A089802EB8201039AD200A3
:109580008DE88400084401B2DC69029A53465846CB
:10959000A047DBF80030DB6A0F9A9342BDD05846F3
:1095A00011B0BDE8F04F184758469847DBF8002047
:1095B00058E7BBF90A3005998B42AEDDBBF90C3098
:1095C00002988342A9DD062313FB0A13002BA4DDB6
:1095D000039B00EBC303002B9FDD9BF81A3033B9CC
:1095E000B9F1AF0F84BF09F101035FFA83F9424A71
:1095F000DBF800300F9211465A698A426AD1BDF8F1
:109600001420089205220992002207921FFA8AF27A
:109610000A92CDF830900FFA8AF2B946039F05926C
:109620000799BDF83040089D0522104610FB041232
:109630000A98324C0646084601FB0651A65C15FA0C
:1096400080F209B212B204910B92082400251CE0AA
:10965000BAF1010F01D1012F24D0069A0192029A8A
:10966000009705FB0722D3F81C800499059B12B2D2
:109670005846C047DBF80030013C013514F0FF04C8
:109680006DB24FEA56063FF460AFF007E0D4069A99
:109690004A45F1D0BAF1010F01D1012F0ED0CDF81A
:1096A0000490DCE7029AD3F818800B99069BAA185D
:1096B00012B25846C047DBF80030DDE7029AD3F813
:1096C00018800B99AA184B4612B25846C047DBF8CF
:1096D0000030D1E758469047DBF800308FE7089913
:1096E000CDF8009005311C6A029A082309B2584649
:1096F000A047DBF800304EE7CD8F0000740001007A
:10970000F0B5C36985B004463BB30A296FD00D2973
:109710004FD01A7A91424CD3587A884249D38A1A48
:109720005D68D2B205EBC205AA78002A56D0E87867
:10973000002853D0607E00283ED095F905E0B4F9AA
:109740000E00A67DB4F90A70724406FB0202BA420A
:1097500069DCE77DB4F9102034E00A295CD00D29DA
:1097600027D0427E002A50D0B0F90E00A57DB4F972
:109770000A60062212FB0502B242E67D42DD228A21
:10978000E38102EBC60212B218462282B4F814E05A
:10979000678A03960B46029501468DE88040204675
:1097A000FFF726FEA37DE28903EB430302EB4303AD
:1097B000E381012005B0F0BDA67DE77DB4F90E0080
:1097C000B4F91020B4F814E00397678A02960B46A8
:1097D0008DE8804001462046FFF70AFE2979E3899B
:1097E000A27D012001FB0233E38105B0F0BD002220
:1097F000C2819A7AC17D038A01FB02330382012070
:1098000005B0F0BDB4F91020C0E7857DC67DB4F980
:109810001020B0F90E00B9E7028AC17DC38102EBC6
:10982000C1030382C5E70020E0819B7A228AE77D9D
:1098300003FB072212B22282C4E700BF11B1817577
:10984000C175704701218175C1757047844641EA31
:10985000000313F003036DD1403A41D351F8043BA8
:1098600040F8043B51F8043B40F8043B51F8043BFA
:1098700040F8043B51F8043B40F8043B51F8043BEA
:1098800040F8043B51F8043B40F8043B51F8043BDA
:1098900040F8043B51F8043B40F8043B51F8043BCA
:1098A00040F8043B51F8043B40F8043B51F8043BBA
:1098B00040F8043B51F8043B40F8043B51F8043BAA
:1098C00040F8043B51F8043B40F8043B51F8043B9A
:1098D00040F8043B51F8043B40F8043B403ABDD209
:1098E000303211D351F8043B40F8043B51F8043BAB
:1098F00040F8043B51F8043B40F8043B51F8043B6A
:1099000040F8043B103AEDD20C3205D351F8043B39
:1099100040F8043B043AF9D2043208D0D2071CBF05
:1099200011F8013B00F8013B01D30B88038060462E
:10993000704700BF082A13D38B078DD010F00303A4
:109940008AD0C3F10403D21ADB071CBF11F8013B14
:1099500000F8013B80D331F8023B20F8023B7BE763
:10996000043AD9D3013A11F8013B00F8013BF9D28E
:109970000B7803704B7843708B7883706046704728
:10998000374A384913681B06FCD40B6813F0800370
:10999000F8D172B634490A78002A5FD0334A344885
:1099A000F0B4344C176806682568D4680C303E441F
:1099B000143200681268304F35442C44204402446D
:1099C000C2F34E022D4E2E482E4D2F4C42F4004233
:1099D0003A60376806682D682C4A24680C303E448B
:1099E000006812682A4F35442C4420440244C2F3D4
:1099F0004E02284E2848294D294C42F400423A6034
:109A0000376806682D68274A24680C303E44006891
:109A10001268254F35442C4420440244C2F34E02C0
:109A2000224E2348234D244C42F400423A603768CA
:109A300006682D68214A24680C303E44006812688C
:109A400035442C4420440244C2F34E021C4842F4E4
:109A5000004202600B7062B6F0BC704762B670479D
:109A600024B0034024B00B40169EFF1F38B00340C3
:109A70003CB0034040B003402CB0034058B003401A
:109A80005CB0034060B0034064B003406CB003407E
:109A900030B0034038B00B403CB00B4040B00B40FE
:109AA00044B00B404CB00B402CB00B4058B00B40B6
:109AB0005CB00B4060B00B4064B00B406CB00B402E
:109AC00030B00B4030B42948294A2A4B2A4D602433
:109AD000E121047011701B78284C082B30D00A2B20
:109AE0002748284937D00C2B0CBF35223D221223A2
:109AF0002A60236002600B60234B24491B78244AB0
:109B0000BBB101230B601360224B23491B78234A0E
:109B1000012B26D9042B0FD9082B1ED9102B94BF4B
:109B2000862387230B6013601D4B01221A7030BC03
:109B300070470B601360E7E784230B601360F3E763
:109B400000F58E200F490830012213232A6023607C
:109B500002600B60D0E73922F7E785230B601360C2
:109B6000E2E780230B601360DEE700BF00400740A0
:109B700001400740AC90FF1F08B003400CB0034009
:109B800008B00B400CB00B40199EFF1F20B00340E3
:109B900020B00B40AD90FF1F24B0034024B00B4019
:109BA000169EFF1F0C2830B417D91023984228BFE7
:109BB00018461C46104A114D1178181A8C4228700C
:109BC00018D00F4913700B7823B10E490E4A0023A9
:109BD0000B60136030BCFFF775BF0A2802D90C2355
:109BE0001C46E7E7082802D90A231C46E2E70823B7
:109BF0001C46DFE730BC7047AC90FF1F159EFF1F6F
:109C0000169EFF1F24B0034024B00B4028282FD8F5
:109C1000334B2DE9F0411E5CFF2E2BD0314B1B78CE
:109C2000002B2AD132062CD472B62F4D2F4C2F4642
:109C3000012326602B7062B672B623681B060CD413
:109C40003B781BB9F4E72B78002BF1D062B602F019
:109C5000CBFA72B623681806F5D5254B1B6800228F
:109C60002A7062B6234A107843FA00F0BDE8F0810A
:109C7000002070470020BDE8F081FFF781FE32062A
:109C8000D2D572B61C4DDFF87C801C4C06F0400724
:109C9000FFB206F03F06D8F80030DFB123F0100322
:109CA000C8F8003001232660134A2B7062B672B6E2
:109CB000236819060CD413781BB9ECE72B78002B1A
:109CC000E9D062B602F090FA72B623681B06F5D5A9
:109CD0000B4BC3E743F01003C8F80030E2E700BFC6
:109CE00074050100169EFF1F189EFF1F00B0034061
:109CF00010B00340159EFF1F179EFF1F00B00B40C2
:109D000010B00B400CB00B400A4A0B49136843F4E7
:109D1000805313600B7843B9084BC0221A70084B6C
:109D200080F30C0000B218807047044B80221A7038
:109D3000F5E700BF2C800440199EFF1F21C00C4096
:109D400000C00C40F0B51B4B1B4E596818689A6850
:109D5000DB6885B06C460FC4337899071DD5174A68
:109D6000174C1378174913F0700318BF1370164A75
:109D7000164B8027177000263320032226706D466D
:109D800008701A7072B6043C45F001052046A847D9
:109D900062B6237813F0700309D10D4B064901E038
:109DA000013B02D00A78D207FAD505B0F0BD237086
:109DB00005B0F0BDA0050100010002400000024016
:109DC000040002400B000240070002400A0002406B
:109DD000410D0300B0F5006F0AD210B5094B1B7896
:109DE000DB07044606D504F1A0500078C0B210BDD0
:109DF00000207047FFF7A6FF04F1A0500078C0B222
:109E000010BD00BF01000240B0F5006F17D238B599
:109E10000F4B1B78DA070D46044611D504F1A0500C
:109E20000378AB420AD00B4A137813F0700318BFC3
:109E30001370074A05701378DB07FCD538BD7047EF
:109E4000FFF780FF04F1A0500378AB42EBD1F5E7B8
:109E5000010002400000024008B5104C08E02368F1
:109E600059050DD423681A050FD42368DB0411D4D7
:109E700023685803F3D500F067FE23685905F1D530
:109E800002F036FA23681A05EFD502F0C7FA236804
:109E9000DB04EDD500F0CAFCEAE700BF34800440E3
:109EA00008B5FFF7D9FF00BF014B10221A80704799
:109EB00000200540704700BF094908B50B6830B164
:109EC0006A461844A2F58052904202D208601846B1
:109ED00008BD03F05BFD0C2303604FF0FF3008BDAD
:109EE000B090FF1FFEE700BFEFF3138070B9EFF3F0
:109EF00010836BB9EFF305825AB94FF48070EFF31A
:109F000011832BB1984228BF184670474FF0FF309D
:109F100070470F2A01D81846F1E7014BD05CEEE7F5
:109F2000F0E300E0704700BF10B40F4B53F830204F
:109F300092F880422CB1012369B182F8803010BCC4
:109F4000704703EBC0035B681A6841B922F0020254
:109F50001A6010BC704782F8003110BC704742F0A4
:109F600003021A6010BC7047B00501001C4A02EBE6
:109F7000C00301295B6811D004291BD052F83000BE
:109F8000002280F8802229B1022920D0032922D082
:109F90001A6070474FF480721A60704752F83000B0
:109FA0004FF4A27280F880121A601A6822F0200220
:109FB0001A60704752F830104FF4A272012081F8F5
:109FC00080021A601A6842F020021A60704740F25C
:109FD00003121A6070474FF481721A60704700BF15
:109FE000B0050100212848D8F8B5042A44D8DFE894
:109FF00002F0484B4E0345004FF410262B4B03EB69
:10A00000C0030D465C68216811F4E06148D0284B1C
:10A01000284A2949C3F89C2104F140422748C3F843
:10A02000A411A2F59221264FC3F8A0017C2925484E
:10A03000C3F8A871C3F8AC012CD9A2F594237C2BEA
:10A040002AD9A2F596237C2B28D9A2F598237C2B1C
:10A0500029D9A2F59A227C2A27D81B4872B62368F0
:10A0600023F4702343F08072C4F384011643236009
:10A0700040F82150266062B6F8BD70474FF4302694
:10A08000BCE74FF40026B9E74FF44026B6E74FF49B
:10A090002026B3E70D48E1E70D48DFE70D48DDE78F
:10A0A000FFF764FFB3E70C48D8E7F8BDB00501003F
:10A0B0000082FF1FF188FF1F9988FF1FC588FF1FBF
:10A0C0006D88FF1F4188FF1F8C91FF1FB490FF1FF9
:10A0D000EC90FF1F3C91FF1F6C91FF1F1A4B03EB8D
:10A0E000C00010B4426802F14043A3F592217C29DC
:10A0F00023D9A3F594217C290DD9A3F596217C2998
:10A100001FD9A3F598217C2919D9A3F59A237C2B73
:10A1100011D80E4C00E00E4C72B613680D4823F0B7
:10A120008773C2F3840123F4803343F08073136098
:10A1300044F8210062B610BC7047074CECE7074CAE
:10A14000EAE7074CE8E700BFB00501008C91FF1F6C
:10A15000EC90FF1F259F0000B490FF1F6C91FF1F24
:10A160003C91FF1F30B4054B054D064C00221021D9
:10A170001A602A602060196030BC704714D0034018
:10A1800004D0034000D00340282838B52ED0002941
:10A1900004464FDD5F4B1B78012505FA03F28A4226
:10A1A00002D8212837D938BD0338C2B2012A3AD99A
:10A1B000202C4AD0192C48D0574A126802FB0112B1
:10A1C00022FA03F31D2800F29B80DFE800F0928B57
:10A1D000847D9999766F999999999999999999689E
:10A1E000615A53994C99999999999945494B1B787A
:10A1F0000B2B08D90C2B1CBF0C3B19410846BDE8A2
:10A200003840FFF781BDC3F10C0399400846BDE813
:10A210003840FFF779BD2946FFF786FE2946BDE89D
:10A220003840FFF7A3BE3D4A126802FB011222FA32
:10A2300003F3C7E72128B6D80021FFF775FE2046B3
:10A240000121BDE83840FFF791BE354A126802FB94
:10A25000011222FA03F3B5E73249334A0B604FF497
:10A260005173136038BD3149314A0B604FF451735B
:10A27000136038BD2F49304A0B6040F244431360ED
:10A2800038BD2E492E4A0B6040F24443136038BD5E
:10A290002C492D4A0B6040F24443136038BD2B49D2
:10A2A0002B4A0B6040F24443136038BD29492A4AC7
:10A2B0000B6040F24443136038BD2849284A0B60C4
:10A2C00040F24443136038BD2649274A0B6040F2F0
:10A2D0004443136038BD2549254A0B6040F244438E
:10A2E000136038BD2349244A0B604FF45173136047
:10A2F00038BD2249224A0B604FF45173136038BDB8
:10A30000212C3FF650AF7F29D4BF002101212046E8
:10A3100093E700BF9491FF1F08800340089003401B
:10A3200008800B4010800B4048A0044018800B4070
:10A330004CA004401880034008B004401080034043
:10A3400004B004404080034018C0044038800340FB
:10A3500014C004402880034010B004402080034013
:10A360000CB004403080034010C0044048800340DB
:10A370001CC00440189003403490044010900340E7
:10A380003090044038B1102828BF1020044AC3B2CE
:10A39000107813707047024A0123107813707047C9
:10A3A0009491FF1F2DE9F8430E4680463249334D04
:10A3B000304603F071FA47F6122300281ABF1D46F3
:10A3C0004FF002094FF00109002425FA04F003F0D0
:10A3D0006DF84FF05E51074603F0C0F80146304675
:10A3E00003F06EFA30B90134072CEED1E80903F01E
:10A3F0005DF807463146384603F064F94FF07C516A
:10A4000002F0A2FF03F096FA4FF6FF729042A8F115
:10A41000030328BF1046012B29D9B8F1170F17D80D
:10A42000174B23FA08F303F0010383F0010223B969
:10A43000B8F1190F0FD0BDE8F883124B124D134934
:10A440001A6044EAC9042A6008601C60BDE8F88309
:10A45000B8F1200FECD10E4B0E4D0F49002244EA0B
:10A46000C9041A602A6008601C60BDE8F8830B4BC1
:10A470000B4D0C49F2E700BF001BB740006CDC023B
:10A480006006F00000800340048003400880034021
:10A4900000800B4004800B4008800B40009003407C
:10A4A0000490034008900340212801D8FFF73CBDE9
:10A4B000704700BF212806D8044B53F8303093F87A
:10A4C0000002C0B270470020704700BFB005010015
:10A4D000212801D8FFF74ABD704700BF72B60C496A
:10A4E0000C4B0D4A1B680868126862B6520102D50F
:10A4F000322B88BF01300949C3F5BB334FF47A7260
:10A50000FF33A1FB031302FB00F000EB9310704735
:10A510001C9EFF1F18E000E004ED00E0ABAAAAAA11
:10A520002DE9F843054672B6204F214B214A1B689E
:10A530003C68126862B6520102D5322B88BF0134E2
:10A5400095B3C3F5BB331C4EDFF86490DFF864802D
:10A55000FF334FF47A72A6FB031302FB04F404EBFF
:10A56000931472B6D9F800103A68D8F800E062B6D1
:10A57000C1F5BB33FF33A6FB03031EF0806FC4EBB2
:10A5800093134FF47A7002D0322988BF013200FB56
:10A590000233B3F57A7F04D3013D05D004F57A7414
:10A5A000DFE701F021FEDCE7BDE8F8831C9EFF1F1A
:10A5B00018E000E004ED00E0ABAAAAAAF8B52D4B24
:10A5C0002D49DFF8D0E0DFF8D0C02C4E2C4D2D4CBB
:10A5D0002D4A2E4F4FF4000018604FF08070186025
:10A5E0004FF0007018604FF0806018604FF000600E
:10A5F00018600020086028234BF6FF71CCF800108B
:10A60000CEF80030336013602B6023603B60B36290
:10A610009362092245F8242CC4F8D80F05F57F650C
:10A62000C7F8D41F07F5FF2707F5FA67C6F8F83F04
:10A630002B6006F5FF26C4F8D42F05F5FD2504F59B
:10A64000FF24386006F2F4761148316005F5FF65A5
:10A6500004F5FD642B6023600260FFF733FA1920D4
:10A66000FFF75EFF00F0B6FF40F21310BDE8F840C0
:10A67000FFF756BF08E100E0048003401480034068
:10A68000248003402C8003401C800340348003401E
:10A6900000800B400C800340088003402DE9F84FF8
:10A6A000214B1B6807460BB101221A70DFF8889016
:10A6B0001E4D99F80040DFF884801D4E0134272C90
:10A6C0008ABF4FF0000A5FFA84FA5446AB462B78F3
:10A6D000A34216D1FFF708FC40281FDC33791B0684
:10A6E000F5D59BF800300133272B86BF0022134697
:10A6F000DAB218F80330DBB2F3712A702B78A34278
:10A70000E8D00C490A4BFFB208F804700120AC22D3
:10A71000087089F800A0DA70BDE8F88FFF28D6DD50
:10A7200001F062FDD3E700BF949EFF1F919EFF1FC3
:10A7300000C00640909EFF1F989EFF1F289EFF1F8F
:10A740001C4BDFF894C01A681B49F0B542F48052E4
:10A750001A4D1A60DFF884E0194F1A4E1A4C002384
:10A760008CF800304FF451722B701F2840F21335D3
:10A770008EF800303B70337025600A6012D819469D
:10A780000124124A124D11701248547000212C27D6
:10A79000402693724FF4003491701174D7702E706C
:10A7A0000460F0BDC0F34431C0F3471400F01F0350
:10A7B000E7E700BF348004400CC00440259EFF1F23
:10A7C000919EFF1F909EFF1F08C0044000C00640DE
:10A7D00031E400E004E100E0249EFF1F989EFF1F8B
:10A7E000034B1B68DB0401D5FFF758BF704700BF60
:10A7F0003480044010B5044C237823B101F0F4FCFC
:10A800002378002BFAD110BD909EFF1F054A064BFE
:10A8100010781B78C0B2DBB2984238BF4030C01A03
:10A82000704700BF249EFF1F259EFF1F30B42B4B97
:10A830001A7994061FD52A48DA7903782949013311
:10A840003F2B0978C8BF00238B42D2B203D0264CDD
:10A85000D9B2E2540170254A116861B1244A1278D4
:10A86000D2B2934236BFC2F140029B1A9B18272BEB
:10A87000C4BF01230B70194AD378DBB2180611D478
:10A880005A060DD5154B1B795B0609D5194B1A498C
:10A890001B6800220A7003B11A70104B2C22DA7068
:10A8A00030BC704711790906EAD5144910480C7874
:10A8B0000178C9B28C420DD04A1C272A84BF0021DE
:10A8C0000A460F4D054C98BFD1B2AA5CD2B2E271D4
:10A8D0000170D5E76C21D170D2E700BF00C00640FF
:10A8E000249EFF1F259EFF1F509EFF1F209EFF1FBF
:10A8F000919EFF1F949EFF1F909EFF1F989EFF1F1B
:10A90000289EFF1F21282FD8184B195CFF292BD018
:10A91000174B184ADFF870C003EBC000F0B543686E
:10A92000DFF868E0144F154D154E00241C60DEF86A
:10A930000030012043F020038840CEF8003014603E
:10A940004FF4A07338602E60C2F800C0013BFDD107
:10A9500013689B05FCD42023013BFDD1094B09B2B0
:10A9600033F8110080B2F0BD00207047C00601002E
:10A97000B005010000500440085004400450044059
:10A98000000002030051044080014A003880044066
:10A99000431E032B14D872B60A4951F8230068B13C
:10A9A00070B4094C058834F81320466841F82360D8
:10A9B000521B24F8132062B670BC704762B6704711
:10A9C00000207047F49EFF1F58A1FF1F0138032885
:10A9D0000BD872B6074B53F8203043B100205B68A8
:10A9E0000130002BFBD162B670470020704718463B
:10A9F000F9E700BF489FFF1F30B472B62B4A1378A7
:10AA00001D0706D52A4B196A002936D0996A0029F4
:10AA100041D053781C0706D5254B196C00293ED030
:10AA2000996C002939D09378190705D5204B196EF8
:10AA3000002936D0996E89B1D3781B0707D51C4BF6
:10AA4000D3F880207AB3D3F8882011213AB162B6C6
:10AA5000184B00221A7030BC00F048BE0D21154C76
:10AA6000154D227843F8315003EBC1030830013A09
:10AA70005860227062B630BC704704220D4C0F4DF6
:10AA8000217843F8325003EBC20308304A1E586065
:10AA9000227062B6EFE70521E1E70921DFE708222E
:10AAA000ECE70C22EAE71022E8E700BFE806010025
:10AAB0000080FF1F719FFF1FC800400088004000FA
:10AAC000431E032B1DD81B4A400140F0100030B438
:10AAD000104472B6184CE25C032A1BD8DFE802F07F
:10AAE0000212151703220D88E25410F0080F14BF4C
:10AAF000C823882343EA054308310360416062B6F6
:10AB000030BC704708300222EDE70522EBE7083041
:10AB10000422E8E7094A52F8230038B1084A52F8FB
:10AB20002300416042F8231062B6E9E742F823109F
:10AB3000034AF7E70080FF1F809FFF1F489FFF1F0A
:10AB4000589FFF1F00BE70472DE9F04FDFF818B384
:10AB5000DFF818A387B044E0AD4F4FEA930807EB46
:10AB6000C809013ED9F8042003F00803F6B2A2F1A7
:10AB7000080003F0FF04002B40F0018157F8383043
:10AB80001B0C99B222F8081C002B00F0EF80A14B9F
:10AB900022F8064C42F8044C53F82620002A00F014
:10ABA000CF819D4D55F8263058609C4C45F82600C5
:10ABB00034F81630194424F8161000F077FD0028F8
:10ABC00000F0C281964A974B19F0080F00F1080077
:10ABD00018BF1346C9F8040047F8383008238BF82B
:10ABE00000309BF80040E4B265071CD58E4B1B7803
:10ABF000B3B18E490A7802F0FF0322B1013BDBB208
:10AC00000B7003B900BE8A490A7802F0FF032AB12B
:10AC1000013BDBB20B70002B00F0688100F064FE9A
:10AC200004238BF8003004F0080303F0FF02002B2C
:10AC300000F0C9809AF80030DBB21E098CD19A0866
:10AC4000DFF8CC9159F8321009EBC200C1F383014F
:10AC5000013940680C2900F28580DFE801F07A7A3A
:10AC60008383838383834683838307000168714DD5
:10AC70004068714F714E6860296088B240F281610E
:10AC80000024674B49F832304FF0010E88423C6097
:10AC9000C9F81040C9F8184086F800E05C4A00F294
:10ACA000E780B0F5D06F80F01B82B0F5817F00F0B7
:10ACB000D98100F26981802800F02A82822840F040
:10ACC000D781A98801F07F01042900F2D1815C4875
:10ACD0005C4A890008441470547001788C0740F174
:10ACE000608382F800E0022173E1534F3A682AB38F
:10ACF000554B524E554819883478057840298E4670
:10AD000045F0020828BF4FF0400E002C84F00104EB
:10AD10003470CEEB01010CBF8824C82409EBC806AF
:10AD200089B285F0010544EA0E447260198049F841
:10AD3000384072440570002965D03A603D4B1A884E
:10AD4000B2F5A06F0ED100219A785970404B1A705D
:10AD500008E038493F4C0D68A54200F09880304922
:10AD600049F832103C4A0123137037E72C4A2D4B27
:10AD700019F0080F18BF134647F838302EE700F0D7
:10AD8000B5FC364A364952F82630002B00F0E380F5
:10AD900058688C5D42F8260003F10802C9F80420C7
:10ADA000032C05D8DFE804F02C02292602228A555C
:10ADB0001A8819F0080F0CBF8823C82343EA0243FE
:10ADC00047F838300AE7E00700F19380210600F1E8
:10ADD000D180A20706D5234A234913780220DBB28B
:10ADE00013700870E30602D51F4B10221A7007B0CB
:10ADF000BDE8F08F04228A55DAE705228A55D7E7A5
:10AE000003228A55D4E7BEF1400F18BF002294E711
:10AE10000080FF1FF49EFF1FA09EFF1F58A1FF1F71
:10AE2000C8004000880040007C9FFF1F059FFF1F57
:10AE3000F09FFF1F689FFF1F9C9EFF1F049FFF1F27
:10AE4000C0200740749FFF1FB09EFF1F709FFF1F11
:10AE5000982007402109000394200740489FFF1FC6
:10AE6000809FFF1F882007408020074090200740D8
:10AE7000B0F5106F00F07C8140F2A38040F6211203
:10AE8000904240F07B82A54A012313706AE74C6828
:10AE9000A3498C427FF463AF0178A9297FF45FAFA7
:10AEA000417845297FF45BAF8178C2297FF457AFA1
:10AEB000C1786B297FF453AF9A489B4E0178347860
:10AEC00081F00105002C41F0020105700CBF8820C3
:10AED000C82084F0010449F8310009EBC10193480E
:10AEE0003470002505244D60047038E700F062FFDF
:10AEF00094E68F4B89488B491A614FF0020E80F817
:10AF000000E08C4F0A708C49196099608B4E8C4D13
:10AF10008C4C9A610D213970FF213170DFF84CE2C1
:10AF200029702270884D894A8EF800109F270124CD
:10AF300006F8047C5D600470DA6007B0BDE8F08F4D
:10AF400043F82600824D30E6824A47F838001378ED
:10AF50000133137042E68B5D032B00F2BA8001A22D
:10AF600052F823F0DDAB0000DDAB0000BDAF000008
:10AF7000B7AF00006F49724B80220D2008701A7025
:10AF8000A2077FF52FAF26E740F20232904240F051
:10AF9000ED81AA8802F07F02042A69D86D88002D0D
:10AFA00066D16449CDF804E0920011440A7842F079
:10AFB00002020A70C1E101238B550FE600238B5575
:10AFC0000CE6B0F5086F53D16349644A09781170F3
:10AFD0007146ED888D4280F0E88252480478402D19
:10AFE000AE4644F0020C28BF4FF0400E02EB0E03B9
:10AFF00009EBCC01029301234A604FEA0E48CEEBE5
:10B00000050101930025C82242EA080384F00102E9
:10B0100049F83C3035700270DFF814C1424BDFF85C
:10B02000048149BBBEF1400F7FF42DAF42F0020C0A
:10B0300009EBCC03029ADFF8F8E05A608DBB0D04EF
:10B0400045F088059DF804304EF83C500A443370B2
:10B050000470134640297FF416AF0021404A3B603C
:10B06000118010E7AA8802F07F02042A40F28B8147
:10B07000304A0F23137006E74029D7D942F0020265
:10B080000CEBC200029E4660BDB19DF804503548ED
:10B090001D703346403988F8004040334CF8320088
:10B0A000DCE79DF8043033700D04029B047045F01A
:10B0B000C8050B444EF83C50CCE79DF804501D7079
:10B0C000029B1D4888F80040403940334CF832005C
:10B0D000C4E719F0080F0CBF022303238B557DE54D
:10B0E00021494A68002AC3D06C88B5F804E003E01F
:10B0F0000C314A68002ABBD00B88A342F8D14B8898
:10B100007345F5D1240A032C0CBF1178098960E737
:10B11000124A0221147054705BE700BF942007406C
:10B1200001000400709FFF1F049FFF1F059FFF1F6A
:10B130000080FF1FC0200740880040008820074093
:10B140008020074098200740B49EFF1F089FFF1FE4
:10B15000A09EFF1F719FFF1F7C9FFF1F749FFF1FFB
:10B16000B09EFF1FC8004000EC0601008C20074085
:10B17000B248116AAC7804700C0600F19881D9F8D5
:10B180002820AF49100600F1DB81D9F83020AC4906
:10B19000120600F1D081D9F83820A949130600F130
:10B1A000C581D9F84020A649150600F1BA81D9F821
:10B1B0004820A349140600F1AF81D9F85020A049D6
:10B1C000100600F1A481D9F858209D49120600F11B
:10B1D0009981D9F860209A49130600F18E81D9F837
:10B1E00068209749150600F18381D9F870209449A9
:10B1F000140600F17881D9F878209149100600F101
:10B200006D81D9F880208E49120600F16181D9F84C
:10B2100088208B49130600F15581D9F89020884980
:10B22000150600F14981D9F898208549140600F1E6
:10B23000FF808448844A854901908548854D864C25
:10B24000049700230596029580460F4616461D4634
:10B250000394306828B1446800F048FA2046002C76
:10B26000F9D100233360029B38681A46002342F864
:10B27000253028B1446800F039FA2046002CF9D175
:10B2800000223A60019A98F800301146002241F8F5
:10B29000042B039A0191023B4FF0000122F8151094
:10B2A000032B07D8DFE803F05D025D024FF00103D6
:10B2B00088F800300135042D06F1040607F1040773
:10B2C00008F10108C5D1654C654D2278654B049F96
:10B2D000059E0021100729701A7000F192806249C2
:10B2E00062780A700021C9F83010C9F838101107C7
:10B2F000DFF84C816ED4A2785C49DFF844810A7093
:10B3000000211207C9F85010C9F858104BD4E27840
:10B3100057494B4C0A7013074FF00001C9F87010E1
:10B32000C9F8781000F1AE8033780193002283F0E1
:10B330000105C9F89020C9F898200021029188469B
:10B340008E460A464B48047844F0020C09EBCC03C5
:10B350000393019B002B039B5A600CBF8822C822D9
:10B3600052E64FF0000388F80030A3E7B0F5A06F75
:10B370007FF47EAE012300250193DEE740F6212213
:10B380009042F7D074E66D88002D7FF471AE3A4993
:10B39000CDF804E0920011440A7822F002020A700B
:10B3A000CBE7022115E600F081F9002800F0EB80E0
:10B3B0000830324AC8F86400C8F8602000F076F916
:10B3C000002800F0DA8008302D4AC9F86C00C9F86E
:10B3D00068209CE700F06AF9002800F0E08008305F
:10B3E000264AC8F84400C8F8402000F05FF9002859
:10B3F00000F0CF800830224AC9F84C00C9F8482034
:10B4000079E700F053F9002800F0A58008301B4AC6
:10B41000C9F82400C9F8202000F048F9002800F0FD
:10B4200094800830164AC9F82C00C9F8282056E73D
:10B43000D1F89C00083800F059F9FAE67C9FFF1F0C
:10B440000080FF1F589FFF1FF49EFF1F489FFF1F94
:10B45000809FFF1FA09EFF1F58A1FF1FE80601004D
:10B46000719FFF1FC4200740C8200740CC20074021
:10B47000D0200740709FFF1FC02007408800400079
:10B48000C800400000F012F9002870D008304F4A80
:10B49000C4F88400C4F8802000F008F9002860D0C7
:10B4A00008304B4AC9F88C00C9F888203CE7506A3C
:10B4B000083800F01BF962E6D1F89400083800F073
:10B4C00015F9B0E6D1F88C00083800F00FF9A4E6C1
:10B4D000D1F88400083800F009F998E6C86F0838F8
:10B4E00000F004F98DE6486F083800F0FFF882E6B6
:10B4F000C86E083800F0FAF877E6486E083800F0B1
:10B50000F5F86CE6C86D083800F0F0F861E6486DB3
:10B51000083800F0EBF856E6C86C083800F0E6F89A
:10B520004BE6486C083800F0E1F840E6C86B083894
:10B5300000F0DCF835E6486B083800F0D7F82AE66A
:10B54000C86A083800F0D2F81FE62A78C9F828003F
:10B5500001322A70C3E62A78C9F8200001322A7025
:10B560005AE72A78C9F8880001322A70DCE62A787E
:10B57000C4F8800001322A708EE72A78C9F8680082
:10B5800001322A70C3E62A78C8F8600001322A70B6
:10B5900014E72A78C9F8480001322A70ABE62A7805
:10B5A000C8F8400001322A701FE740298E4628BFA4
:10B5B0004FF0400E02EB0E0302930123CEEB01018C
:10B5C0004FEA0E4800250193BCE600BF880040000A
:10B5D000C8004000F8B500F0A7FF294B29482A4CC5
:10B5E0002A4F2B4DDFF8BCC0DFF8BCE0294E00220B
:10B5F0001A605A609A60DA601A615A619A61DA6177
:10B600001A625A629A62DA621A635A639A63DA6356
:10B610001A645A649A64DA641A655A659A65DA6536
:10B620001A665A669A66DA661A675A679A67DA6716
:10B63000C3F880200168C3F8842041F480210160B0
:10B64000C3F307212170C3F30740134938701B0E61
:10B650002B70FF238CF80030104D8EF8003010480E
:10B660000B700123337084F8642070264FF400744B
:10B67000102207F82C3C2E70046081F8F820F8BDE9
:10B680000080FF1F348004409C200740B02007400A
:10B69000B4200740942007401020074049E400E010
:10B6A00008E100E0802007408820074072B60D487E
:10B6B0000268B2FA82F30F2B10DC4FF00041D94040
:10B6C00022EA0102026062B6074803EBC303DB0013
:10B6D000C2180021C15010465160704762B6002068
:10B6E000704700BF9891FF1FBC83FF1F0D4B0E4A90
:10B6F000C31AA2FB03231B090F2B0CD80B4A127889
:10B7000052B972B60A484FF00041026821FA03F3B9
:10B710001A43026062B67047064A1278002AF0D0D7
:10B72000FFF76AB9BC83FF1F398EE338719FFF1F93
:10B730009891FF1F7C9FFF1F38B50E4B0E4C1B6866
:10B74000218805468BB1B1F5917F05D20B4A4B1C80
:10B7500055549BB2238038BD0022084898470021E9
:10B76000064A55540123238038BDB1F5917FEDD3AE
:10B7700038BD00BFA89FFF1F62A1FF1F68A1FF1F68
:10B780002DE9F843214E224F3168012380463B705A
:10B79000B1B1204D4B8801EB8302013300240F2B04
:10B7A000C2F808802C7004D84B8000233B70BDE8A1
:10B7B000F88340230B800320FFF782F93460F4E71D
:10B7C000DFF8549099F80030002BF0D0114D45F679
:10B7D000215408E0013C12D02B7883B900F004FD1D
:10B7E00099F800307BB10320FFF7F0F80528F1D875
:10B7F000FFF75CFF014630600028EBD0CAE7012369
:10B800002B70BDE8F883BDE8F88300BFC49FFF1F1D
:10B81000989FFF1FC89FFF1F7C9FFF1F1201F8B555
:10B82000D5B2A1B3012943D04378044600781B0662
:10B8300043EA004040F4704045F004068F1E304358
:10B84000FFF79EFF022F04F1020314D9053414F808
:10B85000023C14F8032C14F8010C1B0443EA0223E5
:10B86000334343EA0060033FFFF78AFF022F23467A
:10B8700004F10304EBD8022F23D0012F0DD045F49F
:10B88000774040F00500BDE8F840FFF779BF144865
:10B890002843BDE8F840FFF773BF187845F47705F3
:10B8A00045F0060545EA0020BDE8F840FFF768BF0F
:10B8B00003780C4845EA03452843BDE8F840FFF704
:10B8C0005FBF1A78587845F0774545F0070545EA97
:10B8D000022545EA0040BDE8F840FFF751BF00BF30
:10B8E00006F0F70007F000F738B5084B1C7824B9CC
:10B8F000074D296809B14B8803B938BD9B000B80FF
:10B900000320FFF7DDF82C6038BD00BF989FFF1FB4
:10B91000C49FFF1F2DE9F041AD4E33680746002B51
:10B9200000F092801D885A88910803EB810104324F
:10B93000AA428C6842D25A8004F00F064FEA1428BB
:10B94000A449A6F1080208F00F00C4F30313062A65
:10B9500000F101050B701AD9B31E012B5FFA88F0B4
:10B960004ED9052E48D0042E00F0A481731F022B5F
:10B970007FD90F2E0ED1F72842D8F02802D0964B4F
:10B980001B883BB1FFF7D8FE0020BDE8F08127B14E
:10B99000BD4202D00020BDE8F081082EC4F303337D
:10B9A00000F08780092E11D00A2E40F094800A2BD7
:10B9B000F0D18A4B8A4A1B68A02181E01846FFF724
:10B9C00095FE0420FEF7E4FF3060B5E7092BE1D1D6
:10B9D000270E00F07B81834B814A1B689021C4F3C2
:10B9E00007461170EDB2FCB2002B00F09D8022469C
:10B9F00031462846984797E0F02843D9F72841D0A8
:10BA0000F1380E28C6D801A353F820F0C3BB0000BC
:10BA1000A7BB000095BB000095B9000095B90000D8
:10BA200087BB000095B9000067BC000095B9000015
:10BA300031BC00004BBC00006FBB000095B900009A
:10BA400057BB00003BBB0000674B1B78002BA1D00D
:10BA50000420FEF79DFF0346306000289AD0058839
:10BA6000002D7FF460AFFFF741FE35602846BDE84A
:10BA7000F081FFF761FEC4F30740FFF75DFE072E7C
:10BA800002D1200EFFF758FE534B584A19885848E8
:10BA90001468584D524A017000270E0AF0201F808A
:10BAA0002E7010700CB301225348A0470120BDE84E
:10BAB000F081082B7FF46EAF504B494A1B68802100
:10BAC000C4F307461170EDB2240E6BB3284622462C
:10BAD0003146984728E00B2E11D10B2B7FF45AAF3B
:10BAE000474B3F4A1B68B021EAE7464B1B68002BD7
:10BAF00000F0FB80404898470120BDE8F0810C2E03
:10BB000040F000810C2B7FF445AF3F4B344A1B685B
:10BB1000C0211170EDB2C4F30746002B00F0C880BD
:10BB200028463146240E98473849314A314B0D702A
:10BB300016701C700120BDE8F081354B1B68002B8E
:10BB400000F0D6809847C4F30746254BEDB2240E8B
:10BB500083F80080E8E72F4B1B68002BF2D12E4BB7
:10BB60001B68A3B1FE209847C4F30746EDE72B4BB3
:10BB70001B68002BE6D1284B1B6843B1FC2098477B
:10BB8000C4F30746E1E7264B1B68002BDAD1C4F368
:10BB90000746DAE7234B1B68C4F30746002BD4D0D3
:10BBA00030469847D1E7204B1A68002AEFD0260C80
:10BBB000630C06F07F0003F47E531843F6B29047FF
:10BBC000C3E71A4B1B68C4F30746002BE8D1BCE758
:10BBD000D09FFF1F66A1FF1F62A1FF1FAC9FFF1F29
:10BBE00060A1FF1FE09FFF1F7C9FFF1FA89FFF1FFB
:10BBF00064A1FF1F65A1FF1F68A1FF1FD89FFF1F42
:10BC0000DC9FFF1FC09FFF1F9C9FFF1F67A1FF1F9F
:10BC1000889FFF1F8C9FFF1F909FFF1FCC9FFF1FC0
:10BC2000BC9FFF1FD49FFF1FA49FFF1FB89FFF1F34
:10BC30003F4B1B68002B85D13E4B1B68002BA6D0C9
:10BC4000FA209847C4F307467FE73B4B1B68002B5D
:10BC50007FF478AF374B1B68002B98D0FB209847B8
:10BC6000C4F3074671E7354B1B68002B7FF46AAFBE
:10BC7000304B1B68002B8AD0F8209847C4F3074646
:10BC800063E70E2B7FF486AE2D4A2E4B1268E0211F
:10BC90001970002A47D0260C610C06F07F0301F4CE
:10BCA0007E511943EDB2A1F5005128469047F6B2F6
:10BCB000240E39E7FFF740FDC4F30740FFF73CFDD2
:10BCC000200EFFF739FD0020BDE8F0811E4B1D4A14
:10BCD0001B6880211170EDB2C4F3074683B1314671
:10BCE00028463A4698473C461EE70120BDE8F081C9
:10BCF000104B1B68002B3FF44AAFFF20984746E7E4
:10BD00001C4611E70D2EBCD10D2B7FF443AE0F4B1B
:10BD10000C4A1B68D0211170EDB2C4F30746002B0A
:10BD20007FF4FEAEC4E7C4F30746EDB2240EFBE693
:10BD3000B49FFF1F909FFF1F949FFF1F849FFF1FB3
:10BD4000A09FFF1F60A1FF1FD89FFF1FB09FFF1F75
:10BD500038B5164D2868E0B101884488A14213DD4A
:10BD600003191B7A83B104F10803C2180C1B0023CA
:10BD700002E012F8011F21B10133A342F9D120469C
:10BD800038BD1C46204638BDFFF7B0FC00202860B7
:10BD900038BD074B1B780BB9002038BD0220FEF7D9
:10BDA000F7FD28600028D7D1F6E700BFEC9FFF1F02
:10BDB0007C9FFF1F0D4B1B78BBB910B50C4C216845
:10BDC00003F0FF024B883F2B07DC07330B4401F1E4
:10BDD000470003F8012F8342FBD140230B80012051
:10BDE000FEF76EFE0023236010BD7047E49FFF1F27
:10BDF000E89FFF1F10B4EFF3108272B6437F33B990
:10BE0000017F012907D003290FD00123437702B90D
:10BE100062B610BC7047124C2168A1B11149436150
:10BE20000B68836108605861EFE70F4C216881B1AE
:10BE30000E4943610B688361086058610C4B4FF0F9
:10BE400080511960E1E7074B416181612060186012
:10BE5000DBE7064B4161816120601860EEE700BFBF
:10BE600004A0FF1F00A0FF1FF49FFF1FF89FFF1FEC
:10BE700004ED00E070B5EFF3108272B60C4C206850
:10BE800080B10C4E00254369236073B19D6102B9F6
:10BE900062B6457783689847EFF3108272B62068E0
:10BEA0000028F0D102B962B670BD3360EFE700BF81
:10BEB000F49FFF1FF89FFF1FFFF7DCBF184A30B445
:10BEC0001468002C27D0036821688B420ED2CB1A4D
:10BED00000218460C1602360E0601060022303756C
:10BEE00030BC704711688B42144608D3A2685B1AB5
:10BEF0000360002AF6D18260C460A060EEE7D268D9
:10BF0000C2608460E060C568CB1A0222A86023602A
:10BF1000027530BC70478460C4601060DEE700BF0B
:10BF2000FC9FFF1FF8B5224E34682CB32368002B0A
:10BF30003AD1204F1D4604E03468ECB12368002B51
:10BF400032D1A36803B1DD602069336003682575D1
:10BF50001B68BB4221D1037F4560022BC46020D007
:10BF6000FFF748FF6368002BE6D023602046FFF709
:10BF7000A5FF3468002CE1D1EFF3108372B60E4AAE
:10BF800000211068116003B962B628B18468FFF718
:10BF900095FF20460028F9D1F8BD22460021984798
:10BFA000E0E783689847DDE7013B2360E4E700BFF3
:10BFB000FC9FFF1FD58000000CA0FF1F024A1368E2
:10BFC00001331360FFF7AEBF1C9EFF1F704700BF19
:10BFD0000368F0B4FBB1002501249D60DC601B4CBC
:10BFE0001A601C44241104F144056A1103269200CE
:10BFF0009E60174F0679174B47F8241002F16042F4
:10C0000002F5614205F01F05012000FA05F5E6542E
:10C010001560F0BC7047104C236843F400032360A4
:10C0200000BF0E4B0E4DA4F58734A4F59E74012677
:10C030001E60234604609C68002CD0D01033AB42B5
:10C040000360F8D1002303601846E2E7008FFCBFCD
:10C050009C91FF1F44E400E03C80044000700340DA
:10C06000407103400168A9B10B4BF0B40B441B11A4
:10C070000A4E0B4F0B4D46F8237003F1440202F0B9
:10C080001F0401235211A340002445F822308C6084
:10C090000460F0BC704700BF008FFCBF9C91FF1F85
:10C0A000CDBF000080E100E0024A034B0121116096
:10C0B0001B6818470C7103409C91FF1F024A034BF9
:10C0C000012111605B6818471C7103409C91FF1FA0
:10C0D000024A034B012111609B6818472C710340F1
:10C0E0009C91FF1F024A034B01211160DB68184736
:10C0F0003C7103409C91FF1FF8B50E4671B17AB1B7
:10C100000746144600253B6816F8011B1B68384695
:10C110009847013C0544F6D12846F8BD0846F8BDCD
:10C120001046F8BD00B5064A036812885B6883B004
:10C1300001A9ADF804200222984703B05DF804FB82
:10C14000E4060100F0B507468BB0002A33D0012A7F
:10C1500008BF0A2251B3212400E0F4B2B1FBF2F58A
:10C1600002FB1511C8B2092900F1300198BFC8B20D
:10C170000AA988BF3730214488BFC0B201F8240C17
:10C18000661E2946002DE8D133B1013CE4B20AAB6A
:10C1900023442D2203F8242C3B6801AA11195B6863
:10C1A0003846C4F1220298470BB0F0BD30228DF81A
:10C1B00025202124E8E70368C9B21B6898470BB023
:10C1C000F0BD00BF0029BABF49422D2300230A2237
:10C1D000FFF7B8BF08B5F4F751FAF5F765FD00F0C1
:10C1E00003F8FAE7704700BF38B5224C237803B153
:10C1F00038BD01232370FFF7ABFD70BB00F068F87A
:10C2000040BB00F0FBF810BBFEF700FBE0B90023D9
:10C210002370EFF30583002BEAD1EFF3108172B6A0
:10C22000154B1868E0B1154C2278CAB945691D60F4
:10C2300001232370C5B1AA6101B962B60025457713
:10C24000836898472570D3E700F0B4F9DFE700F082
:10C25000AFF9D9E700F0AAF9D3E7FFF7C3FFCDE7BD
:10C260000029C5D162B638BD054B1D600029E5D156
:10C27000E3E700BF10A0FF1F04A0FF1F08A0FF1FDF
:10C2800000A0FF1FF0B44D1E2E46002400E0013434
:10C29000B0FBF2F302FB1300092800F130078ABF5C
:10C2A0003730F8B2C0B206F8010F1846002BEED1B5
:10C2B0000A1953704CB1107815F8016F28700133CA
:10C2C000E01A834202F80169F5DB0846F0BC7047CA
:10C2D000054A064B10781B78C0B2DBB2984238BFD3
:10C2E0004030C01A704700BF18A0FF1F19A0FF1FE1
:10C2F000F0B4384B1A7912F0300F2CD072B6997D09
:10C3000001F0FF0200293DD062B6334F334938783F
:10C310000D78334E1C46C0B2EDB2431C402BE17980
:10C3200028BF0023AB4202F1FF32C9B21CBFF15457
:10C33000184612F0FF02F0D12A4B1B68C2B23A70C5
:10C340004BB1A84236BFC5F14005401B4019272814
:10C35000C4BF01221A701F49CA78D2B2150616D47A
:10C3600052060DD51B4B1B795B0609D51E4B1F4989
:10C370001B6800220A7003B11A70164B3C22DA7057
:10C38000F0BC70474022D9795A7462B6E3E70B7962
:10C390001C06E5D5164B174E1C783378E4B2DBB299
:10C3A0009C420ED0144D01E0A3420AD00133402B31
:10C3B00028BF00230879E85CC0B2C871087D07284F
:10C3C000F2D9DBB2034933700B79180644BF7C23E2
:10C3D000CB70C5E700A0064018A0FF1F19A0FF1FE3
:10C3E0005CA0FF1F14A0FF1FA0A0FF1F9CA0FF1FA9
:10C3F000A4A0FF1F9DA0FF1F1CA0FF1F054A064B06
:10C4000010781B78C0B2DBB2984238BF4030C01AF7
:10C41000704700BF18A1FF1FADA0FF1FF0B4384B3D
:10C420001A7912F0300F2CD072B6997D01F0FF020C
:10C4300000293DD062B6334F334938780D78334EFA
:10C440001C46C0B2EDB2431C402BE17928BF00234B
:10C45000AB4202F1FF32C9B21CBFF154184612F0D0
:10C46000FF02F0D12A4B1B68C2B23A704BB1A8420E
:10C4700036BFC5F14005401B40192728C4BF012223
:10C480001A701F49CA78D2B2150616D452060DD5B5
:10C490001B4B1B795B0609D51E4B1F491B680022ED
:10C4A0000A7003B11A70164B3C22DA70F0BC704768
:10C4B0004022D9795A7462B6E3E70B791C06E5D5B8
:10C4C000164B174E1C783378E4B2DBB29C420ED088
:10C4D000144D01E0A3420AD00133282B28BF0023CA
:10C4E0000879E85CC0B2C871087D0728F2D9DBB2D0
:10C4F000034933700B79180644BF7C23CB70C5E722
:10C5000000B0064018A1FF1FADA0FF1FD8A0FF1F5D
:10C51000A8A0FF1F1CA1FF1FACA0FF1F20A1FF1F91
:10C5200019A1FF1FB0A0FF1F70B584B072B6194BE0
:10C53000194D1A48702241260F2480211A702E703E
:10C540001A460470197013781B06FCD5144B186832
:10C5500062B6144B144C984298BF00EB800001A9BE
:10C5600098BF40000A22FFF78DFE01A92046002354
:10C5700011F8012B01333AB10A2B20F8022FF7D121
:10C580001623237004B070BD5B00DBB2237004B0CF
:10C5900070BD00BF000002400700024006000240DC
:10C5A000080002407F9698007492FF1F704700BFFA
:10C5B000704700BF704700BF2DE9F043DFF8EC8003
:10C5C0008BB006460F4600F073F898F9003001333F
:10C5D00004460D4637D03046394600F0DFF90028D2
:10C5E00031D02BA3D3E900233046394600F026FE94
:10C5F000814668BB28A3D3E900233046394600F0C2
:10C60000FFFD00B398F90030254ACDF820900424AE
:10C6100000200021022BCDE90467CDE902670094D8
:10C620000192CDE906012CD0684600F0BDF940B377
:10C63000089B1BB101F0AAF9089B0360DDE9060124
:10C640000BB0BDE8F083204629460BB0BDE8F0836F
:10C65000134A98F90030019203210022CDE90467C2
:10C66000CDE90267009108922BB90E4B4FF0604262
:10C67000CDE90623D8E70C490020022BCDE90601BD
:10C68000D2D101F083F922230360D1E7AFF3008018
:10C69000EF39FAFE422E864051302DD5104987C021
:10C6A00058070100FFFFEF470000F07F8A92FF1F4D
:10C6B0002DE9F04FB04F21F00042BA4283B00C4652
:10C6C0004FEAD17605460DD9AC4FBA4225D9C1F310
:10C6D0001303034340F0EF800EB10020014603B086
:10C6E000BDE8F08FA64B9A4200F2CC80A54B9A424F
:10C6F00000F2DE808AA3D3E9002300F05DF9002276
:10C70000A14B00F09BFD002800F005812846214642
:10C7100000229D4B00F050F9E1E783A3D3E9002309
:10C7200000F08CFD002840F0CB802846214680A3F5
:10C73000D3E9002300F064FD0028CED1934B2846B6
:10C7400003EBC60821467CA3D3E9002300F0E6FAF8
:10C75000D8E9002300F030F900F07AFD804600F0BF
:10C7600077FA77A3D3E9002306460F4600F0D6FAFE
:10C7700002460B462846214600F01CF972A3D3E975
:10C780000023CDE900013046394600F0C7FA824661
:10C790008B4652465B46DDE9000100F00BF9054689
:10C7A0000C462A4623462846214600F0B7FA68A3DD
:10C7B000D3E9002306460F4600F0B0FA66A3D3E99A
:10C7C000002300F0F7F832463B4600F0A7FA64A3D6
:10C7D000D3E9002300F0F0F832463B4600F09EFA21
:10C7E00061A3D3E9002300F0E5F832463B4600F0B0
:10C7F00095FA5FA3D3E9002300F0DEF832463B460A
:10C8000000F08CFA02460B462846214600F0D2F88A
:10C8100006460F462846214632463B46B8F1000FF1
:10C8200056D000F07BFA324604460D463B460020C7
:10C830004FF0804100F0BEF802460B4620462946E4
:10C8400000F096FB02460B465046594600F0B2F8FF
:10C85000DDE9002300F0AEF80B4602464A4900200D
:10C8600000F0A8F86FF47F7398454FDA08F57A78EE
:10C8700001EB085100224FF0B87300F04FFA03B0FB
:10C88000BDE8F08F424B9A423FF658AF414BF4005F
:10C890002344D3E9002300F08DF83F4BC6F1010893
:10C8A0001C44CDE90001D4E900ABC6EB080870E7F1
:10C8B0004FF0000875E702460B4600F07DF80EE7E2
:10C8C00017A3D3E900231046194600F027FA06E71C
:10C8D00000F024FA0022804689464FF0804330461B
:10C8E000394600F067F802460B464046494600F0DC
:10C8F0003FFB2A46234600F05DF802460B46002027
:10C90000214900F057F803B0BDE8F08F01EB085162
:10C9100003B0BDE8F08F804643E700BFAFF300806F
:10C920009C7500883CE4377EEF39FAFE422E864043
:10C9300051302DD5104987C0FE822B654715F73F32
:10C940000000E0FE422EE63F763C7935EF39EA3DC5
:10C95000D0A4BE726937663EF16BD2C541BDBB3E05
:10C960002CDE25AF6A56113F93BDBE166CC1663FE3
:10C970003E5555555555C53F412E8640FFFFEF7F2B
:10C98000422ED63FFFFF2F3E0000F03F6007010020
:10C99000B1A2F03F800701007007010041F00041A3
:10C9A00001F58010C00F70470020704781F00041F2
:10C9B00002E000BF83F0004330B54FEA41044FEA84
:10C9C000430594EA050F08BF90EA020F1FBF54EA1F
:10C9D000000C55EA020C7FEA645C7FEA655C00F0BB
:10C9E000E2804FEA5454D4EB5555B8BF6D420CDD8C
:10C9F0002C4480EA020281EA030382EA000083EA0F
:10CA0000010180EA020281EA0303362D88BF30BDAE
:10CA100011F0004F4FEA01314FF4801C4CEA113104
:10CA200002D0404261EB410113F0004F4FEA033363
:10CA30004CEA133302D0524263EB430394EA050FEE
:10CA400000F0A780A4F10104D5F1200E0DDB02FA5D
:10CA50000EFC22FA05F2801841F1000103FA0EF2F1
:10CA6000801843FA05F359410EE0A5F120050EF1B7
:10CA7000200E012A03FA0EFC28BF4CF0020C43FAE8
:10CA800005F3C01851EBE37101F0004507D54FF0F5
:10CA9000000EDCF1000C7EEB00006EEB0101B1F545
:10CAA000801F1BD3B1F5001F0CD349085FEA30008B
:10CAB0004FEA3C0C04F101044FEA445212F5800F96
:10CAC00080F09A80BCF1004F08BF5FEA500C50F133
:10CAD000000041EB045141EA050130BD5FEA4C0C16
:10CAE000404141EB010111F4801FA4F10104E9D19F
:10CAF00091F0000F04BF01460020B1FA81F308BF96
:10CB00002033A3F10B03B3F120020CDA0C3208DD61
:10CB100002F1140CC2F10C0201FA0CF021FA02F13C
:10CB20000CE002F11402D8BFC2F1200C01FA02F1AC
:10CB300020FA0CFCDCBF41EA0C019040E41AA2BFD1
:10CB400001EB0451294330BD6FEA04041F3C1CDA99
:10CB50000C340EDC04F11404C4F1200220FA04F0B9
:10CB600001FA02F340EA030021FA04F345EA030163
:10CB700030BDC4F10C04C4F1200220FA02F001FA25
:10CB800004F340EA0300294630BD21FA04F02946A7
:10CB900030BD94F0000F83F4801306BF81F4801140
:10CBA0000134013D4EE77FEA645C18BF7FEA655CB3
:10CBB00029D094EA050F08BF90EA020F05D054EA85
:10CBC000000C04BF1946104630BD91EA030F1EBF8A
:10CBD0000021002030BD5FEA545C05D1400049418E
:10CBE00028BF41F0004130BD14F580043CBF01F581
:10CBF000801130BD01F0004545F0FE4141F4700167
:10CC00004FF0000030BD7FEA645C1ABF1946104641
:10CC10007FEA655C1CBF0B46024650EA013406BF42
:10CC200052EA033591EA030F41F4002130BD00BF01
:10CC300090F0000F04BF0021704730B54FF48064BE
:10CC400004F132044FF000054FF0000150E700BF3F
:10CC500090F0000F04BF0021704730B54FF480649E
:10CC600004F1320410F0004548BF40424FF000018B
:10CC70003EE700BF42004FEAE2014FEA31014FEACE
:10CC800002701FBF12F07F4393F07F4F81F060511D
:10CC9000704792F0000F14BF93F07F4F704730B58C
:10CCA0004FF4607401F0004521F0004120E700BF1F
:10CCB00050EA010208BF704730B54FF000050AE0A6
:10CCC00050EA010208BF704730B511F0004502D5A7
:10CCD000404261EB41014FF4806404F132045FEAA9
:10CCE000915C3FF4DCAE4FF003025FEADC0C18BF4E
:10CCF00003325FEADC0C18BF033202EBDC02C2F144
:10CD0000200300FA03FC20FA02F001FA03FE40EAD5
:10CD10000E0021FA02F11444C1E600BF70B54FF0D5
:10CD2000FF0C4CF4E06C1CEA11541DBF1CEA1355B7
:10CD300094EA0C0F95EA0C0F00F0DEF82C4481EA1F
:10CD4000030621EA4C5123EA4C5350EA013518BF3F
:10CD500052EA033541F4801143F4801338D0A0FB2C
:10CD600002CE4FF00005E1FB02E506F00042E0FBD9
:10CD700003E54FF00006E1FB03569CF0000F18BFDF
:10CD80004EF0010EA4F1FF04B6F5007F64F5407487
:10CD900004D25FEA4E0E6D4146EB060642EAC6211A
:10CDA00041EA55514FEAC52040EA5E504FEACE2E87
:10CDB000B4F1FD0C88BFBCF5E06F1ED8BEF1004F8A
:10CDC00008BF5FEA500E50F1000041EB045170BD06
:10CDD00006F0004646EA010140EA020081EA03014A
:10CDE000B4EB5C04C2BFD4EB0C0541EA045170BD46
:10CDF00041F480114FF0000E013C00F3AB8014F1C0
:10CE0000360FDEBF002001F0004170BDC4F1000408
:10CE1000203C35DA0C341BDC04F11404C4F1200589
:10CE200000FA05F320FA04F001FA05F240EA0200E4
:10CE300001F0004221F0004110EBD37021FA04F61A
:10CE400042EB06015EEA430E08BF20EAD37070BDD4
:10CE5000C4F10C04C4F1200500FA04F320FA05F033
:10CE600001FA04F240EA020001F0004110EBD37035
:10CE700041F100015EEA430E08BF20EAD37070BDA5
:10CE8000C4F1200500FA05F24EEA020E20FA04F37E
:10CE900001FA05F243EA020321FA04F001F000412D
:10CEA00021FA04F220EA020000EBD3705EEA430E9E
:10CEB00008BF20EAD37070BD94F0000F0FD101F0CD
:10CEC0000046400041EB010111F4801F08BF013C06
:10CED000F7D041EA060195F0000F18BF704703F044
:10CEE0000046520043EB030313F4801F08BF013DCB
:10CEF000F7D043EA0603704794EA0C0F0CEA135587
:10CF000018BF95EA0C0F0CD050EA410618BF52EA40
:10CF10004306D1D181EA030101F000414FF0000046
:10CF200070BD50EA410606BF1046194652EA430654
:10CF300019D094EA0C0F02D150EA013613D195EAC8
:10CF40000C0F05D152EA03361CBF104619460AD110
:10CF500081EA030101F0004141F0FE4141F470011A
:10CF60004FF0000070BD41F0FE4141F4780170BD0A
:10CF700070B54FF0FF0C4CF4E06C1CEA11541DBF6F
:10CF80001CEA135594EA0C0F95EA0C0F00F0A7F871
:10CF9000A4EB050481EA030E52EA03354FEA01319E
:10CFA00000F088804FEA03334FF0805545EA1313B1
:10CFB00043EA12634FEA022245EA111545EA106579
:10CFC0004FEA00260EF000419D4208BF964244F110
:10CFD000FD0404F5407402D25B084FEA3202B61A2F
:10CFE00065EB03055B084FEA32024FF480104FF403
:10CFF000002CB6EB020E75EB030E22BFB61A754677
:10D0000040EA0C005B084FEA3202B6EB020E75EB09
:10D01000030E22BFB61A754640EA5C005B084FEA71
:10D020003202B6EB020E75EB030E22BFB61A75463E
:10D0300040EA9C005B084FEA3202B6EB020E75EB49
:10D04000030E22BFB61A754640EADC0055EA060E0A
:10D0500018D04FEA051545EA16754FEA06164FEA4D
:10D06000C30343EA52734FEAC2025FEA1C1CC0D1F9
:10D0700011F4801F0BD141EA00014FF000004FF086
:10D08000004CB6E711F4801F04BF01430020B4F147
:10D09000FD0C88BFBCF5E06F3FF6AFAEB5EB030CFF
:10D0A00004BFB6EB020C5FEA500C50F1000041EBFC
:10D0B000045170BD0EF0004E4EEA113114EB5C04C9
:10D0C000C2BFD4EB0C0541EA045170BD41F480119C
:10D0D0004FF0000E013C90E645EA060E8DE60CEAA4
:10D0E000135594EA0C0F08BF95EA0C0F3FF43BAFC1
:10D0F00094EA0C0F0AD150EA01347FF434AF95EA78
:10D100000C0F7FF425AF104619462CE795EA0C0F5B
:10D1100006D152EA03353FF4FDAE1046194622E728
:10D1200050EA410618BF52EA43067FF4C5AE50EA02
:10D1300041047FF40DAF52EA43057FF4EBAE12E7F2
:10D140004FF0FF3C06E000BF4FF0010C02E000BFD3
:10D150004FF0010C4DF804CD4FEA410C7FEA6C5CB6
:10D160004FEA430C18BF7FEA6C5C1BD001B050EA59
:10D17000410C0CBF52EA430C91EA030F02BF90EA44
:10D18000020F0020704710F1000F91EA030F58BF03
:10D19000994208BF90422CBFD8176FEAE37040F065
:10D1A000010070474FEA410C7FEA6C5C02D150EA03
:10D1B000013C07D14FEA430C7FEA6C5CD6D152EABE
:10D1C000033CD3D05DF8040B704700BF8446104683
:10D1D00062468C461946634600E000BF01B5FFF782
:10D1E000B7FF002848BF10F1000F01BD4DF808ED52
:10D1F000FFF7F4FF0CBF012000205DF808FB00BF23
:10D200004DF808EDFFF7EAFF34BF012000205DF87C
:10D2100008FB00BF4DF808EDFFF7E0FF94BF0120C9
:10D2200000205DF808FB00BF4DF808EDFFF7CEFFCA
:10D2300094BF012000205DF808FB00BF4DF808ED09
:10D24000FFF7C4FF34BF012000205DF808FB00BFDA
:10D250004FEA410212F5001215D211D56FF478731E
:10D26000B3EB625212D94FEAC12343F0004343EAC1
:10D27000505311F0004F23FA02F018BF404270479C
:10D280004FF00000704750EA013005D111F0004026
:10D2900008BF6FF0004070474FF00000704700BFBC
:10D2A0004FEA4102B2F1E04324BFB3F5001CDCF1C8
:10D2B000FE5C0DD901F0004C4FEAC0024CEA507000
:10D2C000B2F1004F40EB830008BF20F0010070472F
:10D2D00011F0804F21D113F13872BCBF01F0004032
:10D2E000704741F480114FEA5252C2F11802C2F164
:10D2F000200C10FA0CF320FA02F018BF40F00100E5
:10D300004FEAC1234FEAD32303FA0CFC40EA0C0096
:10D3100023FA02F34FEA4303CCE77FEA625307D1D3
:10D3200050EA01331EBF4FF0FE4040F4400070470A
:10D3300001F0004040F0FE4040F40000704700BFA4
:10D3400080F0004002E000BF81F0004142001FBFBA
:10D350005FEA410392EA030F7FEA226C7FEA236CC3
:10D360006AD04FEA1262D2EB1363C1BFD2184140B8
:10D3700048404140B8BF5B42192B88BF704710F04E
:10D38000004F40F4000020F07F4018BF404211F0F1
:10D39000004F41F4000121F07F4118BF494292EA59
:10D3A000030F3FD0A2F1010241FA03FC10EB0C0085
:10D3B000C3F1200301FA03F100F0004302D5494212
:10D3C00060EB4000B0F5000F13D3B0F1807F06D3BF
:10D3D00040084FEA310102F10102FE2A51D2B1F1B7
:10D3E000004F40EBC25008BF20F0010040EA0300AC
:10D3F0007047490040EB000010F4000FA2F1010259
:10D40000EDD1B0FA80FCACF1080CB2EB0C0200FAE2
:10D410000CF0AABF00EBC25052421843BCBFD04030
:10D420001843704792F0000F81F4000106BF80F4AA
:10D4300000000132013BB5E74FEA41037FEA226C6D
:10D4400018BF7FEA236C21D092EA030F04D092F038
:10D45000000F08BF0846704790EA010F1CBF00206C
:10D46000704712F07F4F04D1400028BF40F00040C9
:10D47000704712F100723CBF00F50000704700F0E9
:10D48000004343F0FE4040F4000070477FEA226210
:10D4900016BF08467FEA23630146420206BF5FEAE1
:10D4A000412390EA010F40F4800070474FF00003E1
:10D4B00004E000BF10F0004348BF40425FEA000CA8
:10D4C00008BF704743F0964301464FF000001CE050
:10D4D00050EA010208BF70474FF000030AE000BFA6
:10D4E00050EA010208BF704711F0004302D54042E4
:10D4F00061EB41015FEA010C02BF84460146002056
:10D5000043F0B64308BFA3F18053A3F50003BCFA70
:10D510008CF2083AA3EBC25310DB01FA02FC63441D
:10D5200000FA02FCC2F12002BCF1004F20FA02F224
:10D5300043EB020008BF20F00100704702F1200217
:10D5400001FA02FCC2F1200250EA4C0021FA02F278
:10D5500043EB020008BF20EADC7070474FF0FF0C7D
:10D560001CEAD0521EBF1CEAD15392EA0C0F93EA78
:10D570000C0F6FD01A4480EA010C400218BF5FEA1A
:10D5800041211ED04FF0006343EA501043EA51118D
:10D59000A0FB01310CF00040B1F5000F3EBF490087
:10D5A00041EAD3715B0040EA010062F17F02FD2A8B
:10D5B0001DD8B3F1004F40EBC25008BF20F001006E
:10D5C000704790F0000F0CF0004C08BF49024CEA85
:10D5D000502040EA51207F3AC2BFD2F1FF0340EA17
:10D5E000C250704740F400004FF00003013A5DDC88
:10D5F00012F1190FDCBF00F000407047C2F10002C9
:10D60000410021FA02F1C2F1200200FA02FC5FEAB5
:10D61000310040F1000053EA4C0308BF20EADC70FF
:10D62000704792F0000F00F0004C02BF400010F471
:10D63000000F013AF9D040EA0C0093F0000F01F01E
:10D64000004C02BF490011F4000F013BF9D041EA40
:10D650000C018FE70CEAD15392EA0C0F18BF93EA42
:10D660000C0F0AD030F0004C18BF31F0004CD8D16C
:10D6700080EA010000F00040704790F0000F17BFF3
:10D6800090F0004F084691F0000F91F0004F14D039
:10D6900092EA0C0F01D142020FD193EA0C0F03D191
:10D6A0004B0218BF084608D180EA010000F0004094
:10D6B00040F0FE4040F40000704740F0FE4040F46F
:10D6C000400070474FF0FF0C1CEAD0521EBF1CEA0E
:10D6D000D15392EA0C0F93EA0C0F69D0A2EB03022C
:10D6E00080EA010C49024FEA402037D04FF08053C6
:10D6F00043EA111143EA10130CF000408B4238BF8B
:10D700005B0042F17D024FF4000C8B4224BF5B1A98
:10D7100040EA0C00B3EB510F24BFA3EB510340EAE6
:10D720005C00B3EB910F24BFA3EB910340EA9C0094
:10D73000B3EBD10F24BFA3EBD10340EADC001B0104
:10D7400018BF5FEA1C1CE0D1FD2A3FF650AF8B42A8
:10D7500040EBC25008BF20F0010070470CF0004CB5
:10D760004CEA50207F32C2BFD2F1FF0340EAC250E0
:10D77000704740F400004FF00003013A37E792F0A1
:10D78000000F00F0004C02BF400010F4000F013AFF
:10D79000F9D040EA0C0093F0000F01F0004C02BFFA
:10D7A000490011F4000F013BF9D041EA0C0195E763
:10D7B0000CEAD15392EA0C0F08D142027FF47DAFFC
:10D7C00093EA0C0F7FF470AF084676E793EA0C0FEC
:10D7D00004D14B023FF44CAF08466EE730F0004CEA
:10D7E00018BF31F0004CCAD130F000427FF45CAF7A
:10D7F00031F000437FF43CAF5FE700BF4FF0FF3CE8
:10D8000006E000BF4FF0010C02E000BF4FF0010C3A
:10D810004DF804CD4FEA40024FEA41037FEA226C03
:10D8200018BF7FEA236C11D001B052EA530C18BF25
:10D8300090EA010F58BFB2EB030088BFC81738BF8A
:10D840006FEAE17018BF40F0010070477FEA226C78
:10D8500002D15FEA402C05D17FEA236CE4D15FEA74
:10D86000412CE1D05DF8040B704700BF84460846A8
:10D870006146FFE70FB5FFF7C9FF002848BF10F169
:10D88000000F0FBD4DF808EDFFF7F4FF0CBF0120AE
:10D8900000205DF808FB00BF4DF808EDFFF7EAFF38
:10D8A00034BF012000205DF808FB00BF4DF808EDF3
:10D8B000FFF7E0FF94BF012000205DF808FB00BFE8
:10D8C0004DF808EDFFF7D2FF94BF012000205DF86E
:10D8D00008FB00BF4DF808EDFFF7C8FF34BF01207B
:10D8E00000205DF808FB00BF4FEA4002B2F1FE4F96
:10D8F0000FD34FF09E03B3EB12620DD94FEA002312
:10D9000043F0004310F0004F23FA02F018BF4042EA
:10D9100070474FF00000704712F1610F01D14202D1
:10D9200005D110F0004008BF6FF0004070474FF085
:10D930000000704742000ED2B2F1FE4F0BD34FF001
:10D940009E03B3EB126209D44FEA002343F0004375
:10D9500023FA02F070474FF00000704712F1610F98
:10D9600001D1420202D14FF0FF3070474FF000006A
:10D97000704700BF0B460146184600F001B800BFD3
:10D9800013460A460146022000F0ACBE014B18685F
:10D99000704700BFB896FF1F70B50F4E0F4D761B36
:10D9A000B61018BF002405D0013455F8043B984741
:10D9B000A642F9D10A4E0B4D761B02F0EBFEB610D3
:10D9C00018BF002406D0013455F8043B9847A642FE
:10D9D000F9D170BD70BD00BFA0070100A007010014
:10D9E000B4070100A0070100024B0146186800F0CF
:10D9F0000BB800BFB896FF1F024B0146186800F035
:10DA000035BF00BFB896FF1F2DE9F04F01F10B05A0
:10DA1000162D83B0064640F29F8035F0070500F1D1
:10DA2000BF80A94200F2BC8000F058FBB5F5FC7F36
:10DA3000C0F09C826B0A00F0BA80042B00F2838154
:10DA4000A80900F1390E4FEA4E033830C44F07EBF6
:10DA50008303A3F108015C68A14207D1ACE0002A6E
:10DA600080F2AC80E468A14200F0A680636823F0F5
:10DA700003035A1B0F2AF2DDB9493C6901F1080E74
:10DA8000744500F0B381636823F003035A1B0F2A27
:10DA900000F39981002AC1F814E0C1F810E080F287
:10DAA0009E80B3F5007F80F06781DB0803F1010CF5
:10DAB00001229B1002FA03F34A6851F83C80C4F833
:10DAC000088001EBCC091A43A9F10803E3604A601E
:10DAD00041F83C40C8F80C40831001249C4094421B
:10DAE00000F28A80144206D120F003006400144240
:10DAF00000F10400FAD007EBC009CC468046DCF800
:10DB00000C108C4507D173E1002A80F28181C9682D
:10DB10008C4500F06D814B6823F003035A1B0F2ADC
:10DB2000F2DD0C46D1F80CC054F8088F4B1945F0C3
:10DB300001054D6042F00101C8F80CC03046CCF838
:10DB400008807B613B61C3F80CE0C3F808E05960D2
:10DB50009A5000F0C5FA1FE0102921D800F0BEFA53
:10DB60001025062302207E4F07EB8303A3F1080252
:10DB70005C68944200F045816368E168A56823F021
:10DB80000303234430465A68E96042F001028D6085
:10DB90005A6000F0A5FA0834204603B0BDE8F08FC3
:10DBA00000240C232046336003B0BDE8F08F8023AF
:10DBB0004FF0400E3F2049E770465DE72344E1689F
:10DBC0005A68A56842F00102E96030468D605A60EB
:10DBD00000F086FA0834204603B0BDE8F08F2344F5
:10DBE00030465A6842F001025A6000F079FA08346F
:10DBF000204603B0BDE8F08FBC68636823F00308DB
:10DC0000A84504D3C5EB08030F2B00F38C80554BBC
:10DC1000DFF860911A68D9F8003001332A4404EB28
:10DC2000080A00F0608102F580520F3222F47F6210
:10DC300022F00F0211463046019200F04BFCB0F189
:10DC4000FF3F8346019A00F05881824500F2FC8034
:10DC5000454B1968DA451144196000F05381D9F831
:10DC60000000DFF810E101301BBFCAEB0B0A514482
:10DC7000CEF800B019601BF0070100F01781C1F168
:10DC80000800C1F58051834408315A44C2F30B02A5
:10DC9000C2EB010949463046019300F01BFC431CCE
:10DCA000019B00F03F81CBEB00024A4442F00102AD
:10DCB0001968C7F808B04944BC42CBF80420196081
:10DCC000DFF8A49016D0B8F10F0F40F2FD80626823
:10DCD000A8F10C0323F00703E01802F001024FF053
:10DCE000050E1A430F2B6260C0F804E0C0F808E08C
:10DCF00000F21C811D4BBC681A68914288BF1960F4
:10DD00001B4B1A689142626888BF196022F00302B7
:10DD10009542A2EB050301D80F2B04DC304600F03E
:10DD2000DFF9002438E7621943F0010345F00105EB
:10DD300065603046BA60536000F0D2F9083420467E
:10DD400003B0BDE8F08F142B71D9542B00F2A480DE
:10DD5000280B00F16F0E4FEA4E036E3076E600BFDF
:10DD6000BC96FF1F2CA1FF1F30A1FF1F28A1FF1F82
:10DD700024A1FF1FC89AFF1F5A0A042A5ED9142A39
:10DD800000F2B38002F15C0149005B3207EB810CC9
:10DD900057F82110DFF8DC81ACF1080C8C4500F05D
:10DDA00088804A6822F00302934202D289688C4537
:10DDB000F7D1D1F80CC07A68C4F80CC0A160CCF8D7
:10DDC0000840CC6088E6631942F0010745F0010580
:10DDD000656030464B610B61C3F80CE0C3F808E0A6
:10DDE0005F609A50083400F07BF9D5E64A6873E624
:10DDF00008F1010818F0030F0CF1080C7FF47FAE56
:10DE000030E0DC68A34208BF02303FF435AEB3E631
:10DE10000B440C465A68C96854F8085F42F0010286
:10DE20005A603046E9608D6000F05AF9B4E603F1BB
:10DE30005C0E03F15B004FEA4E0307E69A0902F11C
:10DE4000390149003832A1E7BC424A4B3FF400AFE8
:10DE50009C68626822F003025AE759F8083999452C
:10DE600040F0828010F0030F00F1FF30F5D17B68A5
:10DE700023EA04037B6064009C423FF6BDAE002CA5
:10DE80003FF4BAAE1C4240467FF435AE64001C42FB
:10DE900000F10400FAD02EE6B3F5AA7F18D8E80BFB
:10DEA00000F1780E4FEA4E037730CFE54FF4805102
:10DEB000EBE60121D8F80430921001FA02F21A437D
:10DEC000C8F80420614677E70123CBF8043025E742
:10DED00040F25452934220D8A80C00F17D0E4FEA34
:10DEE0004E037C30B2E51032A4E6542A26D81A0B31
:10DEF00002F16F0149006E3248E7BC68626822F0A7
:10DF0000030205E7CAF30B0000287FF4A8AE4244E1
:10DF1000BB6842F001025A60ECE6FE234FF07F0E30
:10DF20007E2093E501224FF00009C1E604F10801CB
:10DF3000304600F09BFCD9F80010DBE6B2F5AA7F72
:10DF400005D8DA0B02F17801490077321EE740F27A
:10DF500054518A4205D89A0C02F17D0149007C3265
:10DF600014E7FE217E2211E77B6884E7E808431C62
:10DF70005B00F8E5BC96FF1F8842F0B50DD98B1801
:10DF800098420AD28118002A51D09A1A13F8014DEA
:10DF900001F8014D9342F9D1F0BD0F2A48D941EA69
:10DFA00000039B0746D100F1100401F11003154650
:10DFB00053F8106C44F8106C53F80C6C44F80C6C6B
:10DFC00053F8086C44F8086C103D53F8046C44F89E
:10DFD000046C0F2D03F1100304F11004E8D8A2F132
:10DFE000100323F00F0302F00F0E1033BEF1030FE6
:10DFF0001944034421D91E1F0D467446043C55F8AC
:10E00000047B46F8047F032CF8D8AEF1040424F016
:10E01000030404342344214402F0030262B1013BAF
:10E020000A4411F8014B03F8014F8A42F9D1F0BDBF
:10E030000346F3E70346F2E7F0BD7246EEE700BFA2
:10E0400070B4840746D0541E002A41D0CDB2034696
:10E0500002E0621EE4B3144603F8015B9A07F8D1AC
:10E06000032C2ED9CDB245EA05250F2C45EA0545EE
:10E0700019D903F110022646103E0F2E42F8105C0B
:10E0800042F80C5C42F8085C42F8045C02F11002B1
:10E09000F2D8A4F1100222F00F0204F00F041032A3
:10E0A000032C13440DD91E462246043A032A46F88F
:10E0B000045BFAD8221F22F003020432134404F056
:10E0C00003042CB1C9B21C4403F8011BA342FBD1C9
:10E0D00070BC704714460346C2E700BF704700BFDC
:10E0E000704700BF024B0A460146186800F002B8AC
:10E0F000B896FF1F2DE9F04F174683B0002900F0B6
:10E10000C1800E46814607F10B05FFF7E7FF56F881
:10E1100004EC162D2EF00304A6F1080840D81022B6
:10E120001546AF4241D8944275DAC94B996808EB5D
:10E1300004008842416800F0D98021F001030344C3
:10E140005B68DB077DD51EF0010F35D039464846A8
:10E15000FFF75AFC0746E0B156F8043C23F00103F0
:10E160004344A0F108029A4200F04481221F242A6D
:10E1700000F23181132A00F204810346324611680D
:10E1800019605168596092689A603146484600F0BB
:10E190006DFB4846FFF7A4FF384603B0BDE8F08F9B
:10E1A00025F00705002D2A46BBDA0C230020C9F80C
:10E1B000003003B0BDE8F08F56F8083CC3EB080A06
:10E1C000DAF8043023F0030C04EB0C039342BDDBBC
:10E1D0005746DAF80C1057F8080F221F242AC1609E
:10E1E000886000F21781132A40F212813168CAF860
:10E1F00008107168CAF80C101B2A00F22B8108362F
:10E200000AF110023168116071685160B168916063
:10E210003E461C46D046631B0F2B1DD8D8F8043051
:10E2200003F0010323434444C8F80430636843F017
:10E23000010363604846FFF753FF304603B0BDE873
:10E24000F08F21F003012144914221DBC3688268F1
:10E250000C46D3609A60DEE7D8F8042008EB05018D
:10E2600002F00102154343F001020B44C8F80450C8
:10E270004A605A6842F0010208315A60484600F08C
:10E28000F5FAD7E7114603B0BDE8F04FFFF7BCBB86
:10E290001EF0010F7FF45AAF56F8083CC3EB080A92
:10E2A000DAF8043023F0030C01EB0C0E96458BDBFF
:10E2B000C36882685746D3609A6057F8081FDAF837
:10E2C0000C30CB60221F242A996000F29980132A17
:10E2D00062D93368CAF808307368CAF80C301B2A50
:10E2E00000F2A08008360AF1100356E021F0030B7B
:10E2F000A34405F11000834559DA1EF0010F7FF4A5
:10E3000025AF56F8081CC1EB080ADAF8041021F012
:10E31000030CE34458453FF757AF5746DAF80C1063
:10E3200057F8080F221F242AC160886000F2B480C9
:10E33000132A40F2A5803168CAF808107168CAF83B
:10E340000C101B2A00F2AF8008360AF11002316867
:10E35000116071685160B16891600AEB0501C5EB0D
:10E360000B0242F0010299604A60DAF8043003F0CF
:10E3700001031D434846CAF80450FFF7B1FE384672
:10E380005CE733680360736843601B2A27D800F199
:10E39000080306F10802F2E63B4632681A6072682A
:10E3A0005A60B2689A603E467446D04633E708EB3E
:10E3B0000501C5EB0B0B4BF0010299604A6056F862
:10E3C000043C03F001031D43484646F8045CFFF794
:10E3D00087FE304632E73146FFF7CEFDD5E6B3681B
:10E3E0008360F368C360242A28D000F1100306F18B
:10E3F0001002C4E650F8043C23F003031C440AE76F
:10E40000314638467446D046FFF7B6FD3E4602E731
:10E410003A46F7E6314638461C46D046FFF7ACFD93
:10E420003E46F8E6B368CAF81030F368CAF814300C
:10E43000242A1BD010360AF11803AEE733690361B2
:10E440007369436106F1180200F1180397E600BFF3
:10E45000BC96FF1FB168CAF81010F168CAF8141012
:10E46000242A0FD010360AF11802CBE63369CAF815
:10E4700018307369CAF81C3018360AF120038CE78B
:10E480003A4664E73269CAF818207269CAF81C2053
:10E4900018360AF12002B5E6314638460193FFF7F7
:10E4A0006BFD019B59E7B168CAF81010F168CAF812
:10E4B0001410242A03D010360AF1180247E73269F3
:10E4C000CAF818207269CAF81C2018360AF120020E
:10E4D0003DE700BF38B5074C0023054608462360DA
:10E4E000FBF7EAFC431C00D038BD2368002BFBD0AF
:10E4F0002B6038BD8CA2FF1FFFFFFFFFFFFFFFFF58
:10E5000090F800F06DE9024520F007016FF0000C73
:10E5100010F0070491F820F040F049804FF000041B
:10E520006FF00700D1E9002391F840F000F10800F6
:10E5300082FA4CF2A4FA8CF283FA4CF3A2FA8CF32E
:10E540004BBBD1E9022382FA4CF200F10800A4FA95
:10E550008CF283FA4CF3A2FA8CF3E3B9D1E90423E9
:10E5600082FA4CF200F10800A4FA8CF283FA4CF320
:10E57000A2FA8CF37BB9D1E9062301F1200182FADA
:10E580004CF200F10800A4FA8CF283FA4CF3A2FAE0
:10E590008CF3002BC6D0002A04BF04301A4612BAEE
:10E5A000B2FA82F2FDE8024500EBD2007047D1E9F1
:10E5B000002304F00305C4F100004FEAC50514F080
:10E5C000040F91F840F00CFA05F562EA05021CBF51
:10E5D00063EA050362464FF00004A9E7002A41D030
:10E5E00040EA010313F00303F0B425D1032A23D931
:10E5F00004680D68AC421FD1043A35D0A4F101354E
:10E6000025EA040414F0803F31D1071D0D1D0DE0F3
:10E6100057F8043B0E68A3F10134B34224EA030423
:10E620000AD1043A20D014F0803F23D1032A29468E
:10E63000384605F10405EBD803780C789C4202F1CA
:10E64000FF320CD182B114B916E06AB17BB110F877
:10E65000013F11F8014FA34202F1FF32F5D0181B20
:10E66000F0BC7047104670471046F0BC7047184623
:10E67000F0BC70470020F3E72046F1E740EA0103D1
:10E680009B0770B42BD1032A29D90C460346214697
:10E6900054F8046BA6F1013525EA060515F0803F14
:10E6A00006D1043A032A43F8046B2146EFD8A2B1FD
:10E6B0000C781C70013A013301313CB16AB111F898
:10E6C000014B03F8014B013A002CF7D12AB11A444F
:10E6D000002103F8011B9A42FBD170BC704703462E
:10E6E000E5E700BF2DE9F047254C2568D5F84841FE
:10E6F0000646884692469946C4B360681F2817DCD0
:10E70000431C76B104EB80050122C5F888A0D4F83B
:10E71000881182401143022EC4F88811C5F808916F
:10E720001ED00230636044F820800020BDE8F087EE
:10E73000144B03B34FF4C870FFF756F90446D0B139
:10E74000D5F84831002780E88800C5F848413846A8
:10E750000123C4F88871C4F88C71002EE1D0D1E790
:10E76000D4F88C110A43C4F88C21DAE705F5A674B5
:10E77000C5F84841C1E74FF0FF30BDE8F08700BF62
:10E7800090070100E9D90000024B13B1024800F0E4
:10E7900005B8704700000000A9E70000002301460B
:10E7A0001A461846FFF79EBF38B5074D074C2C1B7D
:10E7B000A41005D0013C55F8043D9847002CF9D130
:10E7C000BDE8384001F0F6BF000000000000000086
:10E7D000F8B5234F0C460646FFF780FCBB685D6822
:10E7E00025F00305291B01F6EF7121F47F6121F06B
:10E7F0000F01A1F58054B4F5805F07DB002130469E
:10E80000FFF768FEBB682B44984204D03046FFF700
:10E8100067FC0020F8BD61423046FFF75BFE013027
:10E820000DD0104BBA6819682D1B45F00105304614
:10E83000091B55601960FFF753FC0120F8BD00214A
:10E840003046FFF747FEBA68831A0F2BDEDD064C11
:10E850000449246843F00103001B53600860D5E7B6
:10E86000BC96FF1F30A1FF1FC89AFF1F002945D08B
:10E870002DE9F0410D468046FFF730FC55F8047C49
:10E880006A4927F00103A5F10804E2188E68506870
:10E89000B24220F0030062D0FE0750600BD455F85E
:10E8A000087CE41B01F1080EA56875453B446FD058
:10E8B000E768EF60BD6015186D68ED0742D543F05D
:10E8C00001026260E350B3F5007F18D2DB085A1CE6
:10E8D0004D6851F83270A76001209B1000FA03F3D5
:10E8E00001EBC2001D430838E0604D6041F8324042
:10E8F000FC604046BDE8F041FFF7F2BB70475A0AA2
:10E90000042A53D89A0902F139077F0002F1380529
:10E9100001EB870051F827204449083890424DD038
:10E92000516821F003018B4202D292689042F7D1E4
:10E93000D068E060A2608460D4604046BDE8F041E9
:10E94000FFF7CEBB95683A4FBD4203443FD0D06835
:10E95000E86043F0010285606260E350B3E7FF07BF
:10E96000034407D455F8082CA41A1344A068E2689D
:10E97000C26090602F4A126843F0010093426060C9
:10E980008C60B6D32C4B40461968FFF721FFB0E7E7
:10E9900011184968C90744D49168D268CA60034411
:10E9A00043F0010091606060E350A2E7142A17D899
:10E9B00002F15C077F0002F15B05A9E7AA104B6832
:10E9C000012505FA02F213434B600246B1E743F01A
:10E9D00001024C610C61E560A5606260E35088E76C
:10E9E000542A06D81A0B02F16F077F0002F16E0558
:10E9F0008EE7B2F5AA7F06D8DA0B02F178077F001E
:10EA000002F1770584E740F25450824206D89A0C0E
:10EA100002F17D077F0002F17C0579E7FE277E2564
:10EA200076E743F001026260E35062E7BC96FF1FA5
:10EA3000C496FF1FC49AFF1F2CA1FF1F0000CC101B
:10EA4000581BFC21AC26C62A7C2E3831F4334C36B8
:10EA5000A438983A5A3C543D803E7A3FFF3FFFFF2E
:10EA60000000FF03FF07FF0BFF0FFF13FF17FF1B44
:10EA7000FF1FFF23FF27FF2BFF2FFF33FF37FF3B36
:10EA8000FF3FFFFF0000D007100E88133219AA1EA7
:10EA9000282374275C2B442F643284354038663A2F
:10EAA0008C3C803EFF3FFFFF0000900120031405D7
:10EAB000D0075A0AAC0DCC10B4146A18E81C3421E3
:10EAC00080252A2B70301437FF3FFFFF00005802CB
:10EAD00046056608540BD80E5C12E015FA19141E90
:10EAE0006022AC265C2B0C30BC34023AFF3FFFFFA7
:10EAF0000000C800F4018403140508072E091C0C4B
:10EB0000D80EF811AE159619401F1C25F22B58345B
:10EB1000FF3FFFFF00006400C8009001BC021A0420
:10EB2000DC059E07F609800CA00F2413A2174C1DCC
:10EB30005424442FFF3FFFFF00005802460566089B
:10EB4000540BD80E5C127017FC21F82A7030583420
:10EB5000DC37663A8C3C803EFF3FFFFF00005802E6
:10EB600046056608540BA00FD4172823F82A442F13
:10EB7000643284354038663A8C3C803EFF3FFFFF6C
:10EB800000007805220B0410B4143219B01DFC21CA
:10EB90004826FE29822D383126344637663A223DF2
:10EBA000FF3FFFFF0000540BEC13FA1908201C254F
:10EBB0003629EC2C0C302C33E8357238663AF63BAB
:10EBC000863D163FFF3FFFFF3CEA0000A4EB00003C
:10EBD00084EA000080EB000060EA0000CCEA00005C
:10EBE000A8EA0000F0EA000014EB000038EB000097
:10EBF0005CEB000010ED0000FCEB00000000D00713
:10EC0000800CD80E0010C012EC130C17FA19141E49
:10EC10006022AC265C2B0C30BC34023AFF3FFFFF75
:10EC200000000000CDCC4C3DCDCCCC3D9A99193E96
:10EC3000CDCC4C3E0000803E9A99993E3333B33E92
:10EC4000CDCCCC3E6666E63E00000000070000002A
:10EC50000C0000001000000013000000160000006F
:10EC60001800000000000000070000000C00000079
:10EC700013000000180000001F0000002400000026
:10EC8000000000000C00000018000000240000003C
:10EC9000300000003C0000004800000000000000C0
:10ECA000FBFFFFFFF4FFFFFFEFFFFFFFE8FFFFFFAA
:10ECB000E3FFFFFFDCFFFFFF00000000F4FFFFFFAA
:10ECC000E8FFFFFFDCFFFFFFD0FFFFFFC4FFFFFFF8
:10ECD000B8FFFFFF2C011301FA00E100C800AF00EC
:10ECE00096007D0064004B00320019004006780554
:10ECF000B004E80384032003BC025802F40190012D
:10ED00002C01FA00C8009600640032001900FFFFD1
:10ED1000000078053408540B800C3C0F5C12E015A1
:10ED2000FA19141E6022AC265C2B0C30BC34023A5B
:10ED3000FF3FFFFFA4ED0000329CFF1F0000FF0F0C
:10ED4000549DFF1F0000FF0F8935000070ED00008B
:10ED5000A49CFF1F32005E010000000000000000C4
:10ED60002935000054485200534E53004D4158007D
:10ED7000544F5543482053454E534500455854522F
:10ED80004120434F4E54524F4C4C4552000000001E
:10ED900050495443482042454E440000424954459E
:10EDA0000000000042524541544800FF7CED000045
:10EDB000FE9CFF1FF401A00F6A9CFF1FF401A00F2F
:10EDC000353500009CED0000E49CFF1FBC025C1286
:10EDD0002E9CFF1FBC025C126D35000090ED000000
:10EDE0003A9DFF1FF401A00FA09CFF1FF401A00F8C
:10EDF00051350000C4F50000CCF50000B8F5000066
:10EE0000BCF50000C0F500005CF400007CF50000DB
:10EE100098F500009CF50000A0F50000A4F50000A6
:10EE2000A8F50000ACF50000B0F5000084F5000086
:10EE3000B4F500005CF4000058F400008CF500000C
:10EE400090F5000094F500005CF400007CF50000F3
:10EE500080F5000084F5000088F5000068F50000EA
:10EE60006CF5000070F5000074F5000078F5000006
:10EE700058F500005CF5000060F5000080FA000025
:10EE800064F50000D4F50000D8F50000DCF50000C2
:10EE9000E0F50000E4F50000E8F50000ECF5000006
:10EEA000F0F50000F4F50000F8F50000FCF50000B6
:10EEB00000F6000004F600000100000008F6000063
:10EEC000070000000000000001000000E94200000F
:10EED0000000000000000000000000000000000032
:10EEE0000000000000000000000000000000000022
:10EEF0000000000000000000000000000000000012
:10EF00000000000000000000000000000000000001
:10EF100000000000000000000000000000000000F1
:10EF200000000000000000000000000000000000E1
:10EF300000000000000000000000000000000000D1
:10EF400000000000000000000000000000000000C1
:10EF500000000000000000000000000000000000B1
:10EF600000000000000000000000000000000000A1
:10EF70000000000000000000000000000000000091
:10EF80000000000000000000000000000000000081
:10EF90000000000000000000000000000000000071
:10EFA0000000000000000000000000000000000061
:10EFB0000000000000000000000000000000000051
:10EFC0000000000000000000000000000000000041
:10EFD0000000000000000000000000000000000031
:10EFE0000000000000000000000000000000000021
:10EFF000000000000001FFFFFFE3600007736000F6
:10F00000000000000001FFFFFFE360000EE360006E
:10F010000000000000018000000360001DC36000CC
:10F02000000000000001BFFFFFE360003B836000C1
:10F03000000000000001BFFFFFE3600077036000F5
:10F04000000000000001B00000036000EE0360005B
:10F05000000000000001B00000036001DC0360005C
:10F06000000000000001B00000036003B80360006E
:10F07000000000200001B000000360077003600082
:10F08000000000600001BFFFFFE3600EE0036000CE
:10F09000000000600001BFFFFFE3601DC0036000CF
:10F0A00000030060000180000003603B80036000FB
:10F0B000000300E00001BFFFFFE360770003600092
:10F0C000000300C00001BFFFFFE360EE000360002B
:10F0D000000380C00001B000000361DC0003600099
:10F0E000000780C00001B000000363B800036000A7
:10F0F0000007C0C00001B00000036770000360009B
:10F100000006C0C00001B00000036EE00003600014
:10F11000000660C10101B00000037DC00003600073
:10F12000000630C30301BFFFFFE37B8000036000E4
:10F13000000C30C30701BFFFFFE37700000360004E
:10F14000000C1CC30601800000030E0000036000D9
:10F15000000C0CC20E01FFFFFFE3FC000003600087
:10F16000000C0EC61E01FFFFFFE3F8000003600065
:10F17000000C07C61E000000000000000000000098
:10F18000000C03C676000000000000000000000034
:10F19000000C01C7E60000000000000000000000B5
:10F1A000000C00C7C60000000000000000000000C6
:10F1B000000C00030600000000000000000000003A
:10F1C000000C000000000000000000000000000033
:10F1D000000C000000000000000000000000000023
:10F1E000000000000000000000000000000000001F
:10F1F000000000000000000000000000000000000F
:10F2000000000000000000000000000000000000FE
:10F2100000000000000000000000000000000000EE
:10F2200000000000000000000000000000000000DE
:10F2300000000000000000000000000000000000CE
:10F2400000000000000000000000000000000000BE
:10F2500000000000000000000000000000000000AE
:10F26000000000000000000000000000000000009E
:10F27000000000000000000000000000000000008E
:10F28000000000000000000000000000000000007E
:10F29000000000000000000000000000000000006E
:10F2A000000000000000000000000000000000005E
:10F2B000000000000000000000000000000000004E
:10F2C000000000000000000000000000000000003E
:10F2D000194200000600000009000000E88EFF1F30
:10F2E0000000000080F8000074F80000289DFF1F57
:10F2F0000000300000000000ED4F0000D54000008D
:10F3000000000000F8F60000000001010800000005
:10F31000808EFF1F6CF60000000002010A00000052
:10F32000308FFF1F0000000050F800005CF8000064
:10F33000609CFF1F0000010001000000E945000083
:10F34000193F0000000000000100000074F70000F9
:10F350000600000008F60000000004050800000098
:10F36000288BFF1F010000006CF70000090000005F
:10F370000000000001000000C55B0000010000006B
:10F3800094F70000030000000000000098F800005F
:10F3900074F80000249DFF1F0000300000000000F2
:10F3A000ED4F0000D540000000000000000000000C
:10F3B00001000000594C0000000000009CF7000014
:10F3C000A4F700007E9CFF1F010010000600000053
:10F3D000F1570000393F0000F14900000000000033
:10F3E00068F8000074F800002A9DFF1F000030003C
:10F3F00000000000ED4F0000D540000000000000BC
:10F4000040F8000000000301060000001C8DFF1FF3
:10F4100000000000A4F8000074F80000009DFF1F29
:10F420000000300000000000DD4F0000293F000018
:10F43000000000000000000064F6000030F600004C
:10F440007A9CFF1F00000900000000000D4600002C
:10F45000593F0000000000004F4E00004F4646009C
:10F4600055534200424154004C4F572000000000C9
:10F470004D454E552020202020202020205858582F
:10F4800020592E595600000058000000524F5400D9
:10F490004D454C0044594E006D73000042544800E5
:10F4A000424954004C5652004E524D0052455600AF
:10F4B000312F0000415400004D4F440050424400A1
:10F4C00045434200454353004C564C004C565000B7
:10F4D000474C440045434800762E0000312E342E20
:10F4E0003600000053455400434C52004E754556BB
:10F4F000490000006669726D7761726520762E00A2
:10F5000055534220706F776572000000416C6B614B
:10F510006C696E6520626174746572790000000028
:10F5200030202520617420004E694D4820626174AE
:10F5300074657279000000004C69506F206261743C
:10F540007465727900000000444F4E27540000009B
:10F5500050414E4943000000455749004557580067
:10F560005341580045565200484D53003554480009
:10F570004F43540035444E004F444E004D57000059
:10F58000465000004346000053500000535700000F
:10F5900053454C005345450042520000564C000074
:10F5A000455800004D572B0042522B00564C2B0063
:10F5B00045582B00554E4F00414C4B004E4D4800D6
:10F5C0004C495000425254480000000050544348F7
:10F5D000000000002D3400002D3300002D3200000B
:10F5E0002D3100004C494E002B3100002B32000021
:10F5F0002B3300002B340000533100005332000045
:10F600005A3100005A3200005649425241544F00CC
:10F61000444952454354494F4E000000434F4E5415
:10F62000524F4C00535155454C4348204200000076
:10F630004C4556454C00000053454E53452042541E
:10F6400045000000535155454C4348204C000000F4
:10F6500053454E5345204C565200000052455455D8
:10F66000524E000044455054480000005345545544
:10F6700050204354524C53004C4556454C20434374
:10F680000000000050494E4B59204B4559000000E6
:10F690004445474C49544348000000004841524DFE
:10F6A0002053454C0000000053455249455300008B
:10F6B00045584354204841524D0000004841524DA6
:10F6C0002052414E474500004558435420434320B3
:10F6D00042000000455843542043432041000000AD
:10F6E000504954434842454E44000000504F525444
:10F6F0002F474C44000000005345545550204252BF
:10F70000454154480000000056454C20424F4F539D
:10F710005400000056454C2044454C41590000001F
:10F72000435552564500000056454C4F43495459E5
:10F73000000000004252454154482041540000005E
:10F74000434320422052495345000000425254484E
:10F7500020434320420000004252544820434320AB
:10F760004100000041424F5554000000455854529A
:10F7700041530000524F5441544F52005345545589
:10F78000502043544C0000005345545550204252E1
:10F790000000000041444A55535400004D4944497B
:10F7A000204348004D4944492043484E4C00000046
:10F7B000424154205459504500000000574C20430A
:10F7C00048414E00574C20504F5745520000000012
:10F7D0004641535420424F4F5400000044414320BF
:10F7E0004F55540042434153204D4F4445000000C3
:10F7F000335244205452494C4C000000535045436E
:10F80000204B4559000000004741544520484F4CCB
:10F81000440000004C45474143592042520000003B
:10F820004C45474143592050420000004F4354414A
:10F83000564500005452414E53504F53450000006E
:10F84000524F5441544F52205345545550000000DC
:10F850005052494F52495459000000004D4F4E4FED
:10F86000205052494F000000524F5441544520341B
:10F870000000000053454D49544F4E4553000000D1
:10F88000524F54415445203300000000524F544120
:10F890005445203200000000524F5441544520315D
:10F8A00000000000504152414C4C454C00FFFFFF0E
:10F8B0000100000088F70000040000006CF7000061
:10F8C000000005010B000000348DFF1F2C0100001B
:10F8D000000000008CF8000074F80000269DFF1F57
:10F8E0000000300000000000ED4F0000D540000097
:10F8F00000000000010000007CF70000050000008F
:10F900000000000020F7000020F70000A69CFF1F69
:10F9100000000C000300000011570000493F0000E8
:10F92000000000000100000064F700000800000073
:10F930000021110202000000002111020504FFFF56
:10F94000003E7FFF4E754556496330310000000090
:10F950007676764E75455649636363007676764EC5
:10F960007545564963303465657676767676767673
:10F9700076000000496E76616C696420636F6E6684
:10F98000696720666F726D6174000000496E766170
:10F990006C696420636865636B73756D00000000BB
:10F9A000496E76616C696420636F6E666967207367
:10F9B000697A6500496E76616C696420636F6E6672
:10F9C00069672076657273696F6E0000496E7661B3
:10F9D0006C6964206D6573736167652E00000000BB
:10F9E000653030006330300053656E64696E6720A7
:10F9F000636F6E6669672E2E2E000000436F6E6681
:10FA000069672073656E742E000000006330330058
:10FA100053656E64696E672076657273696F6E2ECA
:10FA20000000000063303200526563656976696EDC
:10FA30006720636F6E6669672E2E2E004E657720F5
:10FA4000636F6E6669672073617665642E000000DF
:10FA5000556E6B6E6F776E206D6573736167652E83
:10FA60000000000065303100436F6E666967206DED
:10FA7000676D7400506F776572206F6666204E75F3
:10FA800045564900746F2065786974005265616459
:10FA9000792E00FF34800440400000001211FFFF67
:10FAA000FF02020000001310FFFFFF02020000002F
:10FAB0001800000034800440800000001EFFFFFF9B
:10FAC000FF02000000001DFFFFFFFF02000000001A
:10FAD000190000000000000000000000E5770000B1
:10FAE000A97700005D770000A5770000617700002E
:10FAF0006D7700008D770000000103070F1F3F7F27
:10FB00002200FF2100FFFFFF0080C0E0F0F8FCFEB4
:10FB1000000000000000000001970000F9C0000094
:10FB20005D7700006981000001820000CD8F000038
:10FB3000818F0000B58F00008D8F0000A18F000025
:10FB40009D8E0000CD8F0000F58F0000ED8300003A
:10FB50002D8C0000C98B0000C5900000D18F0000E3
:10FB600029910000C9910000000060000000000021
:10FB7000000000000000000000E0000000000000A5
:10FB80000000000000000001E00000000000000094
:10FB900000000000000001F0000000000000000074
:10FBA000000000000003F000000000000000000062
:10FBB0000000000007F0000000000000000000004E
:10FBC00000000007F8000000000000000000000036
:10FBD00000000FF800000003C0007E000001E000FC
:10FBE0007F0FF800000003C000FE000001E000FFEE
:10FBF000EFF800000003C000FE000001E000FFFF7E
:10FC0000F800000003C000F00000000F007FFE7F3E
:10FC1000C0000003C000F00000000F003FFE7FF8AE
:10FC20003FF1FBCFFCFEF3BC3DEFE01FFE7FFF7F0B
:10FC3000FBFFDFFEFEFFBC3DEFE01FC6FFFF7FFBCB
:10FC4000FFDFFEFEFFBC3DEFE00FE3C7FE787BC3A6
:10FC5000DE1EF0FFBC3DEF0007FF87FC787BC3DEB4
:10FC60001EF0F83C3DEF0001FFFFF0007BC3C01E1B
:10FC7000F0F03C3DEF0001F37FE03FFBC3CFFEF02F
:10FC8000F03C3DEF0003E33F807FFBC3DFFEF0F07D
:10FC90003C3DEF0007E73C00787BC3DE1EF0F03C04
:10FCA0003DEF0007FFBE00787BC3DE1EF0F03C3D59
:10FCB000EF0007FFFE00787BC3DE1EF0F03C3DEF57
:10FCC000000FFFFE007FFBFFDFFEF0F03FFDEFE0E7
:10FCD0000FFFFF007FFBFFDFFEF0F03FFDEFE00FC7
:10FCE000F9FF003E79F9CF9EF0F01F3DE7E01FF1EC
:10FCF000FF0000000000000000000000001F80FF67
:10FD0000007FFFFFFFFFFFFFFFFFFFE01C007F0002
:10FD10007FFFFFFFFEB46D888D18E000001F007F9D
:10FD2000FFFFFFFE95AD7DB577E000000F007FFF80
:10FD3000FFFFFEA5AD9D8D19E0000006007FFFFFCF
:10FD4000FFFEB5ADEDB57EE0AED580A8D300408D09
:10FD50002000A1C8DB40A4A62EAFFFFF00000000DA
:10FD6000000180000000000000000000038000008F
:10FD70000000000000000007C000000000000000BC
:10FD8000000007C00000000000000000000FC000DD
:10FD900000000000000000001FE000000000000064
:10FDA0000000001FE00000000000000000003FE035
:10FDB0000000000000000000003FF0000000000014
:10FDC000000000007FF0000000000000001FF87F2E
:10FDD000F0000000000000003FFE7FF00000000087
:10FDE0000000003FFF7FF0000000000000001FFF48
:10FDF000FBE0000000000000000FFFF9FFC0000062
:10FE0000000000000FFFF9FFF800000000000007ED
:10FE1000FFF1FFFF00000000000003FC73FFFF8004
:10FE2000000000000001FE3FFFFF80000000000016
:10FE300000FF1E0FFF000000000000007FFE1FFCFF
:10FE4000000000000000003FFFFFF800000000007D
:10FE500000000FDFFFE0000000000000001F19FF9E
:10FE6000C0000000000000003F3CFF000000000058
:10FE70000000007E7CF800000000000000007FFE13
:10FE80007C0000000000000000FFFFFC00000000FC
:10FE900000000000FFFFFE0000000000000000FF67
:10FEA000FFFE0000000000000001FFEFFE00000068
:10FEB0000000000001FFCFFE000000000000000372
:10FEC000FF07FE0000000000000003FC07FE00002A
:10FED000000000000003F003FE000000000000002E
:10FEE000018000FE000000000000000000007E0015
:10FEF0000000000000000000003E000000000000C4
:10FF0000000000000C000000000000078000FC0062
:10FF10000003C0000000078001FC000003C00000D7
:10FF200000078001FC000003C0000000078001E022
:10FF30000000001E000000078001E00000001E001D
:10FF40007FE3F79FF9FDE7787BDFC0FFF7FFBFFD99
:10FF5000FDFF787BDFC0FFF7FFBFFDFDFF787BDF94
:10FF6000C0F0F787BC3DE1FF787BDE00F0F787BC8F
:10FF70003DE1F0787BDE0000F787803DE1E0787BB3
:10FF8000DE007FF7879FFDE1E0787BDE00FFF787EB
:10FF9000BFFDE1E0787BDE00F0F787BC3DE1E07873
:10FFA0007BDE00F0F787BC3DE1E0787BDE00F0F718
:10FFB00087BC3DE1E0787BDE00FFF7FFBFFDE1E0BD
:10FFC0007FFBDFC0FFF7FFBFFDE1E07FFBDFC07C11
:10FFD000F3F39F3DE1E03E7BCFC000000000000056
:10FFE0000000000000FFFFFFFFFFFFFFFFFFFFC05B
:10FFF000FFFFFFFFFD68DB111A31C0FFFFFFFFFDB0
:020000021000EC
:100000002B5AFB6AEFC0FFFFFFFFFD4B5B3B1A3330
:10001000C0FFFFFFFFFD6B5BDB6AFDC0000000005F
:100020000000000001970000F9C000005D770000AB
:1000300069810000E59E0000CD8F0000818F0000E7
:10004000B58F00008D8F0000A18F00009D8E0000F5
:10005000CD8F0000F58F0000F18F00001990000097
:1000600071900000C5900000D18F00002991000020
:10007000C991000000000000003E5B4F5B3E3E6BFC
:100080004F6B3E1C3E7C3E1C183C7E3C181C577D32
:10009000571C1C5E7F5E1C00183C1800FFE7C3E77E
:1000A000FF0018241800FFE7DBE7FF30483A060E90
:1000B0002629792926407F050507407F05253F5AD7
:1000C0003CE73C5A7F3E1C1C08081C1C3E7F142247
:1000D0007F22145F5F005F5F06097F017F006689F2
:1000E000956A606060606094A2FFA29408047E0438
:1000F0000810207E201008082A1C08081C2A08085E
:100100001E101010100C1E0C1E0C30383E3830061D
:100110000E3E0E06000000000000005F0000000719
:10012000000700147F147F14242A7F2A1223130847
:10013000646236495620500008070300001C224123
:10014000000041221C002A1C7F1C2A08083E0808C7
:100150000080703000080808080800006060002077
:10016000100804023E5149453E00427F400072495A
:100170004949462141494D331814127F10274545FE
:1001800045393C4A49493141211109073649494914
:1001900036464949291E0000140000004034000082
:1001A00000081422411414141414004122140802EB
:1001B000015909063E415D594E7C1211127C7F495E
:1001C0004949363E414141227F4141413E7F4949B3
:1001D00049417F090909013E414151737F080808DF
:1001E0007F00417F41002040413F017F08142241B0
:1001F0007F404040407F021C027F7F0408107F3E0A
:100200004141413E7F090909063E4151215E7F0976
:10021000192946264949493203017F01033F4040DD
:10022000403F1F2040201F3F4038403F63140814C8
:100230006303047804036159494D43007F41414100
:100240000204081020004141417F040201020440E1
:1002500040404040000307080020545478407F2865
:100260004444383844444428384444287F3854545B
:10027000541800087E090218A4A49C787F0804047E
:100280007800447D40002040403D007F102844001D
:1002900000417F40007C047804787C0804047838AE
:1002A00044444438FC1824241818242418FC7C08DE
:1002B000040408485454542404043F44243C40405B
:1002C000207C1C2040201C3C4030403C442810280E
:1002D000444C9090907C4464544C44000836410057
:1002E0000000770000004136080002010204023CD1
:1002F0002623263C1EA1A161123A4040207A3854A0
:100300005455592155557941225454784221555418
:10031000784020545579400C1E527212395555556B
:1003200059395454545939555454580000457C4156
:100330000002457D420001457C407D1211127DF096
:10034000282528F07C545545002054547C547C0AC0
:10035000097F4932494949323A4444443A324A4889
:1003600048303A4141217A3A42402078009DA0A08D
:100370007D3D4242423D3D4040403D3C24FF2424DF
:10038000487E4943662B2FFC2F2BFF0929F620C0FE
:10039000887E090320545479410000447D4130484F
:1003A000484A32384040227A007A0A0A727D0D1992
:1003B000317D2629292F28262929292630484D40F4
:1003C00020380808080808080808382F10C8ACBAF0
:1003D0002F102834FA00007B000008142A1422226F
:1003E000142A14085500550055AA55AA55AAFF55B8
:1003F000FF55FF000000FF00101010FF0014141440
:10040000FF001010FF00FF1010F010F0141414FC87
:10041000001414F700FF0000FF00FF1414F404FCA4
:10042000141417101F10101F101F1414141F001085
:100430001010F0000000001F101010101F101010FE
:1004400010F010000000FF1010101010101010100D
:10045000FF10000000FF140000FF00FF00001F104D
:10046000170000FC04F414141710171414F404F407
:100470000000FF00F714141414141414F700F714F8
:100480001414171410101F101F141414F414101047
:10049000F010F000001F101F0000001F14000000EB
:1004A000FC140000F010F01010FF10FF141414FFE3
:1004B000141010101F00000000F010FFFFFFFFFFDE
:1004C000F0F0F0F0F0FFFFFF0000000000FFFF0F72
:1004D0000F0F0F0F3844443844FC4A4A4A347E0216
:1004E000020606027E027E02635549416338444497
:1004F0003C04407E201E2006027E020299A5E7A54C
:10050000991C2A492A1C4C7201724C304A4D4D30BC
:100510003048784830BC625A463D3E494949007EE1
:100520000101017E2A2A2A2A2A44445F4444405178
:100530004A444040444A51400000FF0103E080FF2C
:10054000000008086B6B083612362436060F090FB8
:1005500006000018180000001010003040FF0101D4
:10056000001F01011E00191D1712003C3C3C3C00FD
:1005700000000000050E08090D0C06070F0400130B
:100580000393050E08090D0C06070F04FFFFC58530
:10059000848687C4FFFF001303931A9217FFFFFF9F
:1005A0006FF07F030370037813F0800FFBD0704768
:1005B0004008FE4340A004404408FE4344A00440D9
:1005C0000018FE4300C004403000FE433090044059
:1005D0003400FE43349004401C18FE431CC0044009
:1005E0001018FE4310C004400818FE4308C0044021
:1005F0000C18FE430CC004400C10FE430CB0044029
:100600001010FE4310B004401810FE4318B0044010
:100610001C10FE431CB004401410FE4314B00440F0
:100620000418FE4304C004400010FE4300B0044020
:100630000008FE4300A004400408FE4304A0044058
:100640000C08FE430CA004400808FE4308A0044028
:100650001418FE4314C004401818FE4318C0044088
:100660000410FE4304B004400810FE4308B00440E8
:100670001400FE43149004404C08FE434CA0044078
:100680000420FE4304D004402410FE4324B0044060
:100690002010FE4320B004402810FE4328B0044040
:1006A0002C10FE432CB004400020FE4300D0044038
:1006B0004808FE4348A004401000FE431090044048
:1006C000090AFFFFFFFFFFFFFFFFFFFFFFFFFF0D17
:1006D00000060807FFFF0E0FFF0CFFFFFFFFFFFFE5
:1006E0000B05FFFF0D0AFFFF15191519000100008A
:1006F000AC91FF1F1200000000020000D891FF1F04
:1007000073000000002201004C92FF1F2100000036
:10071000002101003492FF1F0900000000030000C7
:100720007092FF1F0000000001030904C091FF1F29
:1007300000000000020309042089FF1F00000000E0
:10074000030309047492FF1F000000000000000072
:10075000000000000000000065787000FFFFFFFF50
:10076000000000000000E03F000000000000E0BFCB
:10077000763C7935EF39EA3D763C7935EF39EABD9B
:100780000000E0FE422EE63F0000E0FE422EE6BF03
:100790009092FF1FF8B500BFF8BC08BC9E4670479A
:1007A00089E7000035040000E134000095500000A6
:0407B000E9730000E9
:0407B400F8B500BFD5
:1007B80038B5084B1C681C6054B1074D94FAA4F373
:1007C800B3FA83F355F823309847631E1C40F5D1DC
:1007D80038BD00BFA0D004408C91FF1F38B5084B2E
:1007E8001C681C6054B1074D94FAA4F3B3FA83F360
:1007F80055F823309847631E1C40F5D138BD00BF1B
:10080800A0C004406C91FF1F38B5084B1C681C60E1
:1008180054B1074D94FAA4F3B3FA83F355F823308F
:100828009847631E1C40F5D138BD00BFA0B00440F6
:100838003C91FF1F38B5084B1C681C6054B1074D2C
:1008480094FAA4F3B3FA83F355F823309847631E58
:100858001C40F5D138BD00BFA0A00440EC90FF1F9C
:1008680038B5084B1C681C6054B1074D94FAA4F3C2
:10087800B3FA83F355F823309847631E1C40F5D12B
:1008880038BD00BFA0900440B490FF1F00000000D6
:1008980016034E00750045005600490020004D0023
:1008A8004900440049000000002000000001020740
:1008B8000B0102070B4A140032000000010000007F
:1008C800002000000020000000100000AB0A00001B
:1008D80000080000660600005505000092040000AC
:1008E800000400008E03000033030000E80200004B
:1008F800AB020000240000000020000002000200FB
:10090800FBFFFFFF000000000000000000000000E7
:1009180000000000000000000000000000000000CF
:10092800000000000C000000140500000C0000008E
:100938000000F0410200FFFFFFFF000034ED00005F
:10094800C4ED0000DCED0000ACED00004CED000053
:100958000000000010F6000010F60000509DFF1F78
:10096800000001000100000000000000000000007D
:100978000000000000000000F0F70000F0F70000A1
:100988009A9CFF1F03000400000000000000000004
:100998000000000000000000000000001CF600003D
:1009A8001CF60000C69BFF1F0000020001000000AB
:1009B800000000000000000000000000000000002F
:1009C80044F6000030F60000B489FF1F01001E0045
:1009D800000000000000000000000000000000000F
:1009E8000100000000000000ECF60000ECF600003A
:1009F800689CFF1F000004000100000000000000C8
:100A08000000000000000000000000009CF600004C
:100A1800A8F60000949CFF1F0000040001000000DD
:100A280000000000000000000000000000000000BE
:100A380078F6000078F60000E69BFF1F00007F00B4
:100A4800010000000000000000000000000000009D
:100A58000000000038F6000030F600008E89FF1F05
:100A6800010011000000000000000000000000006C
:100A7800000000000000000034F7000034F7000018
:100A8800BC9CFF1F000001000100000000000000E6
:100A98000000000000000000288AFF1F34F4000056
:100AA800588FFF1FE089FF1F6C8BFF1F4C8AFF1FA9
:100AB800E08AFF1F5C8EFF1F0000000058F700004F
:100AC80058F70000C89BFF1F00000A000100000043
:100AD800000000000000000000000000000000000E
:100AE80050F6000030F600008C89FF1F01000C0052
:100AF80000000000000000000000000000000000EE
:100B08000000000014F8000014F80000589CFF1FB3
:100B180000000100010000000000000000000000CB
:100B2800000000000000000014F7000014F70000A7
:100B3800C09CFF1F00001E00010000000000000014
:100B480000000000000000000000000040F7000066
:100B580040F70000D69BFF1F01000A0001000000BB
:100B6800000000000000000000000000000000007D
:100B7800D0F70000D0F70000469DFF1F00000100DD
:100B8800000000000000000000000000000000005D
:100B980000000000E4F70000E4F70000FC9CFF1FE1
:100BA800000001000000000000000000000000003C
:100BB8000000000000000000E0F60000E0F6000081
:100BC800CE9CFF1F00000C00000000000000000089
:100BD800000000000000000000000000FCF700001A
:100BE800FCF70000F49CFF1F00000100010000005A
:100BF80000000000000000000000000000000000ED
:100C0800BCF70000BCF70000AC8FFF1F04005000C9
:100C180000000000000000000000000000000000CC
:100C280000000000C4F70000C4F70000DC9DFF1FAF
:100C380000000300000000000000000000000000A9
:100C4800000000000000000034F8000034F8000044
:100C58000A9DFF1F000018000000000000000000AF
:100C680000000000000000000000000008F700007D
:100C780008F70000C49BFF1F0000090001000000E6
:100C880000000000000000000000000010F4000058
:100C980088F30000D0F80000E0F20000DCF3000068
:100CA80024F30000848DFF1F908BFF1F388EFF1FD9
:100CB800688CFF1F048AFF1F208CFF1FB08FFF1F47
:100CC800F08DFF1FFC8BFF1FB08CFF1F8C8CFF1F4C
:100CD80000000000B0F60000BCF600003E9DFF1FBB
:100CE80000000600010000000000000000000000F5
:100CF800000000000000000020F8000020F80000BC
:100D0800FA9CFF1F00000100010000000000000025
:100D180000000000000000000000000084F6000051
:100D280084F60000349CFF1F00001E000000000035
:100D380000000000000000000000000000000000AB
:100D4800D4F60000D4F60000F89CFF1F0000040051
:100D5800010000000000000000000000000000008A
:100D680000000000B0F70000B0F70000389DFF1F3A
:100D78000000020001000000000000000000000068
:100D880000000000000000002CF800002CF8000013
:100D98005C9CFF1F0000060000000000000000002F
:100DA80000000000000000000000000008F800003B
:100DB80008F800008C9CFF1F0000010001000000E3
:100DC800000000000000000000000000000000001B
:100DD80024F6000030F60000BC89FF1F01001E0049
:100DE80000000000000000000000000000000000FB
:100DF800488BFF1FA08EFF1FD88BFF1F048BFF1F80
:100E08000C8FFF1F00F90000B48BFF1FF88CFF1F29
:100E1800000000004CF700004CF70000CA9CFF1FC0
:100E280000007F000100000000000000000000003A
:100E3800000000000000000090F6000090F600009E
:100E4800529DFF1F00004600000000000000000047
:100E58000000000000000000D48CFF1F148EFF1F4C
:100E6800B8F300007CF30000B0F80000F4F80000CC
:100E780048F3000064F3000024F9000000000000BB
:100E880028F7000028F700004E9DFF1F00007F0094
:100E98000100000000000000000000000000000049
:100EA800748AFF1FCC8DFF1F888FFF1F608DFF1F67
:100EB800988AFF1FB8EE0000C48EFF1FA88DFF1F81
:100EC800BC8AFF1F448CFF1F000000005CF6000076
:100ED80030F60000C489FF1F000004000000000075
:100EE80000000000000000000000000000000000FA
:100EF800010000000000000000000000C8F600002B
:100F0800C8F60000B49BFF1F00007F00010000002E
:100F180000000000000000000000000004000000C5
:100F280000000000DCF70000DCF70000A29CFF1FB7
:100F380000000100000000000000000000000000A8
:100F480000000000DCFA000000000000E8030000D8
:100F5800000000000060064094FA00000000000055
:100F68000000000000000000000000000000000079
:100F78000000000000000000000000000000000069
:100F88000000000000000000000000000000000059
:100F98000000000000000000000000000000000049
:100FA8000000000000000000000000000000000039
:100FB800DCFA000000000000E80300000000000068
:100FC80000700640B4FA00000000000000000000B5
:100FD8000000000000000000000000000000000009
:100FE80000000000000000000000000000000000F9
:100FF80000000000000000000000000000000000E9
:1010080000000000000000000000000000000000D8
:101018000000000000000000000000000A040000BA
:1010280090A2FF1F259F0000259F0000259F00001C
:10103800259F0000259F0000259F0000259F000098
:10104800259F0000259F0000259F0000259F000088
:10105800259F0000259F0000259F0000259F000078
:10106800259F0000259F0000259F0000259F000068
:10107800259F0000259F0000259F0000259F000058
:10108800259F0000259F0000259F0000259F000048
:10109800259F0000259F0000259F0000259F000038
:1010A800259F0000259F0000259F0000259F000028
:1010B800259F0000259F0000259F0000259F000018
:1010C800259F0000259F0000259F0000259F000008
:1010D800259F0000259F0000259F0000259F0000F8
:1010E800259F0000259F0000259F0000259F0000E8
:1010F800259F0000259F0000259F0000259F0000D8
:10110800259F000008000000FFFFFFFFCDBF000083
:10111800CDBF0000CDBF0000CDBF000012011001FF
:1011280000000040C016850475020102030100009A
:1011380018035400650065006E00730079006400B0
:10114800750069006E006F0009027300020100C09B
:1011580032090400000201030000072401000125F0
:1011680000062402010100062402020200092403E9
:10117800010301020100092403020401010100091D
:10118800050402400000000005250101010905834E
:1011980002400000000005250101030904010002C6
:1011A8000300000009211101000122210007058127
:1011B80003400001070502032000020006C9FF09D9
:1011C80004A15C7508150026FF0095400975810289
:1011D80095200976910295040976B102C0000000B5
:1011E800040309040C0300000000000000000000D4
:1011F80000000000000000000000010000000000E6
:10120800000000007C95FF1FE495FF1F4C96FF1F10
:1012180000000000000000000000000000000000C6
:1012280000000000000000000000000000000000B6
:1012380000000000000000000000000000000000A6
:101248000000000000000000000000000000000096
:101258000000000000000000000000000000000086
:101268000000000000000000000000000000000076
:101278000000000000000000000000000000000066
:101288000000000000000000000000000000000056
:101298000000000000000000000000000000000046
:1012A8000000000000000000010000000000000035
:1012B8000E33CDAB34126DE6ECDE05000B000000FA
:1012C8000000000000000000000000000000000016
:1012D8000000000000000000000000000000000006
:1012E80000000000000000000000000000000000F6
:1012F80000000000000000000000000000000000E6
:1016280000000000000000009092FF1F0000000072
:1016380000000000BC96FF1FBC96FF1FC496FF1F4A
:10164800C496FF1FCC96FF1FCC96FF1FD496FF1F92
:10165800D496FF1FDC96FF1FDC96FF1FE496FF1F42
:10166800E496FF1FEC96FF1FEC96FF1FF496FF1FF2
:10167800F496FF1FFC96FF1FFC96FF1F0497FF1FA1
:101688000497FF1F0C97FF1F0C97FF1F1497FF1F4E
:101698001497FF1F1C97FF1F1C97FF1F2497FF1FFE
:1016A8002497FF1F2C97FF1F2C97FF1F3497FF1FAE
:1016B8003497FF1F3C97FF1F3C97FF1F4497FF1F5E
:1016C8004497FF1F4C97FF1F4C97FF1F5497FF1F0E
:1016D8005497FF1F5C97FF1F5C97FF1F6497FF1FBE
:1016E8006497FF1F6C97FF1F6C97FF1F7497FF1F6E
:1016F8007497FF1F7C97FF1F7C97FF1F8497FF1F1E
:101708008497FF1F8C97FF1F8C97FF1F9497FF1FCD
:101718009497FF1F9C97FF1F9C97FF1FA497FF1F7D
:10172800A497FF1FAC97FF1FAC97FF1FB497FF1F2D
:10173800B497FF1FBC97FF1FBC97FF1FC497FF1FDD
:10174800C497FF1FCC97FF1FCC97FF1FD497FF1F8D
:10175800D497FF1FDC97FF1FDC97FF1FE497FF1F3D
:10176800E497FF1FEC97FF1FEC97FF1FF497FF1FED
:10177800F497FF1FFC97FF1FFC97FF1F0498FF1F9C
:101788000498FF1F0C98FF1F0C98FF1F1498FF1F49
:101798001498FF1F1C98FF1F1C98FF1F2498FF1FF9
:1017A8002498FF1F2C98FF1F2C98FF1F3498FF1FA9
:1017B8003498FF1F3C98FF1F3C98FF1F4498FF1F59
:1017C8004498FF1F4C98FF1F4C98FF1F5498FF1F09
:1017D8005498FF1F5C98FF1F5C98FF1F6498FF1FB9
:1017E8006498FF1F6C98FF1F6C98FF1F7498FF1F69
:1017F8007498FF1F7C98FF1F7C98FF1F8498FF1F19
:101808008498FF1F8C98FF1F8C98FF1F9498FF1FC8
:101818009498FF1F9C98FF1F9C98FF1FA498FF1F78
:10182800A498FF1FAC98FF1FAC98FF1FB498FF1F28
:10183800B498FF1FBC98FF1FBC98FF1FC498FF1FD8
:10184800C498FF1FCC98FF1FCC98FF1FD498FF1F88
:10185800D498FF1FDC98FF1FDC98FF1FE498FF1F38
:10186800E498FF1FEC98FF1FEC98FF1FF498FF1FE8
:10187800F498FF1FFC98FF1FFC98FF1F0499FF1F97
:101888000499FF1F0C99FF1F0C99FF1F1499FF1F44
:101898001499FF1F1C99FF1F1C99FF1F2499FF1FF4
:1018A8002499FF1F2C99FF1F2C99FF1F3499FF1FA4
:1018B8003499FF1F3C99FF1F3C99FF1F4499FF1F54
:1018C8004499FF1F4C99FF1F4C99FF1F5499FF1F04
:1018D8005499FF1F5C99FF1F5C99FF1F6499FF1FB4
:1018E8006499FF1F6C99FF1F6C99FF1F7499FF1F64
:1018F8007499FF1F7C99FF1F7C99FF1F8499FF1F14
:101908008499FF1F8C99FF1F8C99FF1F9499FF1FC3
:101918009499FF1F9C99FF1F9C99FF1FA499FF1F73
:10192800A499FF1FAC99FF1FAC99FF1FB499FF1F23
:10193800B499FF1FBC99FF1FBC99FF1FC499FF1FD3
:10194800C499FF1FCC99FF1FCC99FF1FD499FF1F83
:10195800D499FF1FDC99FF1FDC99FF1FE499FF1F33
:10196800E499FF1FEC99FF1FEC99FF1FF499FF1FE3
:10197800F499FF1FFC99FF1FFC99FF1F049AFF1F92
:10198800049AFF1F0C9AFF1F0C9AFF1F149AFF1F3F
:10199800149AFF1F1C9AFF1F1C9AFF1F249AFF1FEF
:1019A800249AFF1F2C9AFF1F2C9AFF1F349AFF1F9F
:1019B800349AFF1F3C9AFF1F3C9AFF1F449AFF1F4F
:1019C800449AFF1F4C9AFF1F4C9AFF1F549AFF1FFF
:1019D800549AFF1F5C9AFF1F5C9AFF1F649AFF1FAF
:1019E800649AFF1F6C9AFF1F6C9AFF1F749AFF1F5F
:1019F800749AFF1F7C9AFF1F7C9AFF1F849AFF1F0F
:101A0800849AFF1F8C9AFF1F8C9AFF1F949AFF1FBE
:101A1800949AFF1F9C9AFF1F9C9AFF1FA49AFF1F6E
:101A2800A49AFF1FAC9AFF1FAC9AFF1FB49AFF1F1E
:0C1A3800B49AFF1F00000200FFFFFFFF38
:00000001FF
